:100000000C9487120C94B8120C94B8120C94B81279
:100010000C94B8120C94B8120C94B8120C94B81238
:100020000C94B8120C94B8120C94B8120C94B81228
:100030000C94B8120C94B8120C94B8120C94B81218
:100040000C94B8120C94B8120C94B8120C94B81208
:100050000C94B8120C94B8120C94B8120C94A7AF6C
:100060000C94B8120C94648E0C943A8E0C94B812C2
:100070000C94B8120C94B8120C94B8120C94B812D8
:100080000C94B8120C94B8120C94B8120C94B812C8
:100090000C94108E0C94E68D0C94B8120C9458238A
:1000A0000C94B8120C94B8120C94B8120C94B812A8
:1000B0000C94B8120C94B8120C94B8120C94B81298
:1000C0000C94B8120C94B8120C94B8120C94BC8D09
:1000D0000C94928D0C94B8120C94688D0C943E8DF7
:1000E0000C94B81207634236B79BD8A71A396856E2
:1000F00018AEBAAB558C1D3CB7CC5763BD6DEDFD4A
:10010000753EF6177231BF000000803F0800000006
:10011000BE922449123EABAAAA2ABECDCCCC4C3EFC
:1001200000000080BEABAAAAAA3E00000000BF00EB
:100130000000803F0000000000084178D3BB4387E7
:10014000D1133D190E3CC3BD4282AD2B3E68EC82FB
:1001500076BED98FE1A93E4C80EFFFBE01C4FF7F80
:100160003F00000000000C944B330C947D150C9460
:10017000E85B0C9424150C949D140C9434910C940D
:10018000ED310C9433380C9463360C9401200C94AC
:10019000D79B0C9480140C94DD510C94E1800C944A
:1001A000556B0C940F320C9442A10C940B380C94A8
:1001B000F42F0C94A0C60C9411200C946F140C9482
:1001C00054310C94857B0C9443330C9427810C940C
:1001D00017160C94CA170C9479440C94C3A80C9469
:1001E000BB670C9421370C9418180C94CD4D0C94CB
:1001F0003F1F0C940C910C947F1D0C94779B0C94D6
:100200000F820C94E7540C94BD540C94BFA80C942A
:1002100073440C94F11E0C947BC10C94EF380C9435
:1002200054A10C947C4E0C9491170C943D190C9491
:100230002C830C94AF170C94B5A80C948EC10C941D
:10024000D6150C94D34C0C94E6440C949D180C9445
:100250005D370C94DD740C9461140C94D0120C94E2
:100260002A1A0C94EA380C9443380C945D310C949F
:10027000A0380C946E360C948D140C9424160C94A7
:10028000F5120C9499A80C946A410C94F2320C94D7
:10029000EA120C94253B0C94F9190C94D3700C942D
:1002A00033160C94F0350C94D4120C94A7C10C9412
:1002B000E61B0C949B140C948F220C9407380C941E
:1002C000912D0C9460300C9444150C9472C00C94D5
:1002D0009E1C0C9481A80C94D0A00C9479890C9449
:1002E000ADA80C94AB6A0C947A7F0C94C3380C9430
:1002F00095A80C943E370C9470360C946C160C94A4
:100300002D1F0C94EF680C94046D0C94A3A80C940E
:1003100061520C9472140C94D31B0C94D0380C942E
:10032000C0140C94C8370C94C5810C94096B0C94C0
:10033000E44C0C94FB670C9414830C94A8140C9458
:10034000A9380C94FC310C945F390C949ABA0C9433
:1003500031360C94CF680C94151F0C9442C20C9447
:1003600027220C94BA130C9406370C94CC680C9486
:1003700023B20C94301E0C94FA760C94E8520C9430
:10038000DA800C94DA680C9495800C948B4C0C9465
:1003900034340C94F6170C9428390C946A4C0C9451
:1003A000E6310C94BC1D0C94BA9B0C94AC140C94C8
:1003B00051310C944C880C9462310C94B3320C94EF
:1003C0005A310C94F9400C9473810C9449330C9479
:1003D000F27F0C94B2680C9481820C94C1B80C9496
:1003E00060530C943B370C94386C0C94B0A00C9474
:1003F000994D0C9475320C94D07F0C9434680C9405
:1004000057310C9447680C94326D0C943BBB0C94A0
:10041000886B0C9496160C9465150C9419520C94D8
:1004200028190C94A62E0C941C340C94DD680C94A2
:10043000FE6C0C946A150C9467150C94C16B0C94AB
:100440000B320C943E4E0C94261A0C9412150C94FC
:10045000D9830C94FB370C94C0680C9495320C949F
:10046000C7310C948DA10C94BD680C94AB4E0C94C8
:10047000613F0C9465330C947B7F0C94DE380C94B4
:10048000A7A80C94CEBC0C94B0160C94F4820C94D7
:10049000B1A80C9403330C94A9310C94A0310C94A2
:1004A000C17F0C94A86B0C944D160C94C2450C940F
:1004B000EB2F0C947B530C94C4130C9420680C9475
:1004C00061150C94F9350C9489140C94A0140C94B7
:1004D00078830C9457320C94687F0C945C530C9482
:1004E000281A0C9468820C94EA800C94F3C10C9442
:1004F000919B0C944E2A0C94E9730C9445360C9401
:10050000721A0C9418210C9453370C945F340C9489
:100510000A6D0C946A440C942F890C94EA220C9472
:10052000E4800C9482380C94FF6B0C94F2810C9450
:1005300018750C94B0140C94DDC10C948D9B0C9424
:10054000993E0C9433330C944E150C94B4240C94B3
:1005500048800C94C0150C94C6A80C94E47F0C94AD
:100560008B1C0C94BAC10C948BA80C94C0310C94C5
:10057000794C0C942A390C94DF6A0C946D380C94E5
:10058000FD380C94B8310C9460200C94B9A00C94F4
:1005900075140C94709B0C9416530C945A380C944C
:1005A000C7A80C9458220C94541B0C948FA80C943C
:1005B000BD130C941F6C0C9474C10C9426340C94D1
:1005C000ED210C94BF220C94E3810C94BA120C948C
:1005D00091140C94B9160C9447330C9496830C9494
:1005E000AA520C9467300C949FA80C94E4B30C941A
:1005F000BB540C941E360C9497200C9459360C94D2
:10060000E3200C945A810C943E820C9438530C9441
:10061000622B0C94F52C0C9490150C9467740C942C
:100620007B200C9437210C94F3310C942DC20C9444
:1006300052140C9407530C944D2A0C949FA00C94C4
:10064000EE2F0C94BBA80C949CB70C941E170C9422
:100650002C6D0C9487A80C94941F0C94371D0C944B
:1006600030820C94DE370C942C1A0C9403360C94C4
:10067000C2160C948D350C947F390C947A820C94AC
:10068000CFC10C940C360C940F1A4E414E494E4972
:100690005459494E46CDCCCC3D0AD7233C17B7D14F
:1006A0003877CC2B329595E6241FB14F0A000020F5
:1006B000410000C84200401C4620BCBE4CCA1B0E74
:1006C0005AAEC59D746364696E6F70737578585BBC
:1006D00000454F46003D00494E3A000000200023EF
:1006E00000260029002C002F00320000010000032A
:1006F0000106010901416374697661746520696EC0
:100700002000416374697661746520696E20002D54
:100710003E00200023002D3E00200050656E6465E1
:10072000643A2023002D3E00456D69743A002D3E49
:1007300000456D69743A002D3E00456D69743A00BC
:100740002D3E00456D69743A003D004C45474143DC
:100750005920494E3A0020666F7220286D73293A5D
:10076000004354524C3A205363686564756C6520AD
:10077000636D642000206D730020666F722000435B
:1007800054524C3A2041726D6564200020446973D4
:1007900061726D6564004354524C3A2000207469C4
:1007A0006D653A004354524C3A205265733A004307
:1007B00054524C3A206D6F6D656E7461727920658C
:1007C00076656E74002054533A0020543A00544821
:1007D00045524D3A00436C65616E696E6720616CED
:1007E00061726D20003D0050696E3A004354524CD6
:1007F0003A20436F6D6D616E6420626C6F636B6550
:100800006420627920647269766572004354524CA8
:100810003A204F4E3A416C726561647920416374AD
:100820006976650A004354524C3A2048414C543A88
:10083000416C726561647920496E616374697665A3
:100840000A004354524C3A20584F4E3A20446973A0
:1008500061626C65640A004354524C3A20584F4E12
:100860003A416C7265616479204163746976650A06
:10087000004354524C3A20584F464620736B6970DF
:100880007065642E205072657620636D643A004373
:1008900054524C3A205475726E6564206F6666201F
:1008A00066726F6D3A004354524C3A20526573742D
:1008B0006F7265642066726F6D3A004354524C3A11
:1008C0002049676E6F7265642C206368616E6E6587
:1008D0006C20636D643D0020457865633A004354A5
:1008E000524C3A204163746976653A004354524C45
:1008F0003A2048414C543A416C7265616479204910
:100900006E6163746976650A004354524C3A20580C
:100910004F4E3A2044697361626C65640A00435427
:10092000524C3A20584F4E3A416C726561647920BE
:100930004163746976650A004354524C3A20584F1B
:10094000464620736B69707065642E205072657620
:1009500020636D643A004354524C3A205475726ED1
:100960006564206F66662066726F6D3A004354526C
:100970004C3A20526573746F7265642066726F6DB5
:100980003A0044697361726D696E67206E6F7420FE
:10099000617574686F72697A6564004354524C3AA9
:1009A00020636F6D6D616E64206A75737420666F6D
:1009B0007220004354524C3A204E6F7420656E6F83
:1009C000756768206D656D6F727920666F7220673C
:1009D000726F7570206F7065726174696F6E004917
:1009E0006E76616C69642061726700496E76616C35
:1009F00069642061726700496E76616C6964206188
:100A00007267004354524C3A20556E6B6E6F776E8E
:100A10002073756666697800536B697070696E67DC
:100A2000207363686564756C65642067726F7570A8
:100A30002065786563004354524C3A206368616EC8
:100A40006E656C2066726F7A656E004354524C3A44
:100A5000206368616E6E656C2066726F7A656E00E9
:100A6000536B697070656420686F6D69652073747D
:100A7000756666002000205375623D00204974654C
:100A80006D3D004354524C3A2052414D3D00435479
:100A9000524C3A204F75744F664D656D6F72793ABE
:100AA0002000282D292000282B2920002076616C89
:100AB0007565206973200020756E6B6E6F776E0A06
:100AC000005D3D005B0020696E76616C696400200A
:100AD000004143544956453A00206F6B003A0020CC
:100AE0006661696C6564003A005265747279696E7A
:100AF0006720434D440A004354524C2F706F6C6C76
:100B00003A204F75744F664D656D6F72793A2000CB
:100B1000207365632072656D61696E696E6700534D
:100B200074617475732064656666657265640A0035
:100B30002D3E005075623A20002D3E005075623AFD
:100B400020002D3E005075623A2000000000000099
:100B5000636D640000736574000076616C0000646E
:100B6000656C000048535600005247420000666121
:100B70006E00006D6F6465006374726C006875656B
:100B80000000736174000074656D7000726177001D
:100B9000002D3E005075623A20002D3E00507562D7
:100BA0003A200053454E445354415455533A20552E
:100BB0006E6B6E6F776E20636D64200A000000001C
:100BC000000000000000004F4E0000000000000088
:100BD000004F4646000000000000005245535400FC
:100BE0000000000000544F47474C450000000048FB
:100BF000414C54000000000000584F4E000000001F
:100C0000000000584F4646000000000000494E43D7
:100C10005245415345000044454352454153450028
:100C200000454E41424C45000000004449534142BA
:100C30004C45000000554E465245455A4500004679
:100C40005245455A45000000004155544F000000F0
:100C500000000046414E5F4F4E4C59000048494746
:100C6000480000000000004D454449554D0000007B
:100C7000004C4F5700000000000000484541545F01
:100C8000434F4F4C004845415400000000000043D2
:100C90004F4F4C000000000000445259000000007B
:100CA0000000005247420000000000000048535678
:100CB00000000000000000444D580000000000004B
:100CC000444D58524742570000444D585247420045
:100CD000000050574D0000000000004D42555344A5
:100CE000494D0000544845524D4F00000052454CBC
:100CF00041590000000047524F5550000000005677
:100D00004354454D500000004D425553564300009A
:100D1000004143484149455200005350494C454425
:100D20000000004D4F544F52000000005049440055
:100D300000000000004D42555300000000005541E6
:100D40005254425244470052454C415950574D006D
:100D5000444D5852474257570056454E5453000091
:100D60000000454C455641544F5200434F554E5498
:100D70004552000048554D0000000000004D45520E
:100D800043555259000020002D3E00436F6E76659A
:100D90007274696E6720002D3E0057726F6E672077
:100DA00041737369676E6D656E74200052474278B7
:100DB0003A20004853562064697361626C65640090
:100DC00020764C6576656C3A0020436F6E76563A15
:100DD0000020436F6E76533A0020486F743A004308
:100DE0006F6C643A0020436F6E76657274656420A0
:100DF000563A00436F6E76657274656420533A000C
:100E00002D3E0057726F6E672041737369676E6D78
:100E1000656E7420002D3E0057726F6E672041731F
:100E20007369676E6D656E74200020537566663A4F
:100E3000002041543A0053746F7070696E67204906
:100E40006E7075747300206973200044656C65745E
:100E5000696E6720636F6E662E2052414D20776168
:100E6000733A0053746F70706564006E6F746869D4
:100E70006E6720746F2073746F700053746F70709E
:100E8000696E67206368616E6E656C73202E2E2E0E
:100E90000043616E206E6F7420636C65616E202D5F
:100EA000206C6F636B656400436F6E6669672063D7
:100EB00068616E676564206C6F63616C6C792C206F
:100EC000706F7274616C2064697361626C65640038
:100ED0002F636F6E6669672E6A736F6E007265624C
:100EE0006F6F742000436D643A20002F636F6D6D47
:100EF000616E642F002F72616D2F002F6974656D14
:100F00002F002F6974656D2F0022687474703A2F5A
:100F10002F6C617A79686F6D652E72752F707761AD
:100F200022004C6F636174696F6E3A20687474704C
:100F30003A2F2F003F6D61633D002669703D00260A
:100F4000706F72743D00266E616D653D002F00204C
:100F5000004D5154543A20436F6D706C6574652E8A
:100F60002052656D6F766520746F70696320002470
:100F7000636F6D6D616E64004D5154543A20436C43
:100F800065616E55702072657461696E6564207468
:100F90006F7069632000220022004F75744F664D08
:100FA000656D6F727921005D20003A5B004D5154F0
:100FB000543A005D00456D7074793A205B000A0078
:100FC0003A004D41433A00554450205379736C6FB9
:100FD0006720696E697469616C697A65642E0A00BC
:100FE0005379736C6F6720706172616D733A004D55
:100FF0005154543A20736574206669727374206288
:10100000726F6B65720043757272656E74204C412D
:101010004E20636F6E6669672869702C646E732C4E
:1010200067772C7375626E6574293A000A5573658B
:1010300020746865736520636F6D6D616E64733ACB
:10104000202768656C7027202D20746869732074D0
:101050006578740A276D61632064653A61643A6259
:10106000653A65663A66653A3030272073657420C4
:10107000616E642073746F7265204D41432D61640D
:10108000647265737320696E20454550524F4D0A56
:10109000276970205B69705B2C646E735B2C6777CB
:1010A0005B2C7375626E65745D5D5D5D27202D2020
:1010B000736574207374617469632049500A2773DF
:1010C00061766527202D20736176652063757272C5
:1010D000656E7420636F6E66696720696E204E5678
:1010E00052414D3B204F4E7C4F4646202D20656E91
:1010F00061626C652F64697361626C6520617574EF
:101100006F736176650A2767657427205B636F6E6E
:1011100066696720616464725D27202D20676574AD
:1011200020636F6E6669672066726F6D20707265EE
:101130002D636F6E666967757265642055524C2029
:10114000616E642073746F726520616464722C2018
:101150004F4E7C4F4646202D20656E61626C652F98
:1011600064697361626C6520646F776E6C6F616433
:10117000206F6E20737461727475700A276C6F61D2
:101180006427202D206C6F616420636F6E66696731
:101190002066726F6D204E5652414D0A277077645B
:1011A00027202D20646566696E6520616E6420735A
:1011B000746F7265204D5154542070617373776F52
:1011C00072640A276F746170776427202D2064652C
:1011D00066696E6520616E642073746F7265204865
:1011E000545450204150492070617373776F72647A
:1011F0000A276C6F67205B73657269616C5F6C6F47
:10120000676C6576656C5D205B7564705F6C6F679D
:101210006C6576656C5D27202D20646566696E655A
:10122000206C6F67206C6576656C2028302E2E3719
:10123000290A276B696C6C27202D20746573742034
:101240007761746368646F670A27636C65617227EE
:10125000202D20636C65617220454550524F4D0A28
:10126000277265626F6F7427202D207265626F6F21
:101270007420636F6E74726F6C6C657200536F666E
:1012800074207265626F6F74696E672E2E2E005225
:10129000414D3D000A5379736C6F6720000A6D71F0
:1012A000747420000A696E7075747320000A697482
:1012B000656D7320000A436F6E66696775726564B9
:1012C0003A002F00496E3A2000496E697469616CDA
:1012D000697A696E6720496E70757473003B003DD2
:1012E0000050696E3A003B003D4C4F570054686512
:1012F000726D6F3A0042726F6B65727320636F6E2E
:10130000666967757265643A004170706C79696EE0
:101310006720636F6E666967004C6F616465642067
:10132000455441473A004E6F2073746F72656420D4
:10133000636F6E666967004C6F61646564206672F6
:101340006F6D20454550524F4D006C6F61642066B3
:1013500061696C6564004A534F4E2064657465632F
:10136000746564004C6F6164696E6720436F6E66DC
:1013700069672066726F6D20454550524F4D00439E
:101380006F6E666967206175746F736176653A0088
:101390000A5379736C6F67206465627567206C65AA
:1013A00076656C3A0053657269616C20646562759C
:1013B00067206C6576656C3A0053617665640A0057
:1013C0005365742064796E616D69632049500A0029
:1013D0004F54412050617373776F7264207570644D
:1013E000617465640A004E6F204950206164726523
:1013F000737300205361766564004C6F6164696E9D
:1014000067204854545020636F6E666967206F6E82
:1014100020737461727475703A000000000000005F
:10142000000000004F4E00000000000000004F468A
:101430004600000000000000524553540000000028
:101440000000544F47474C450000000048414C54B1
:10145000000000000000584F4E0000000000000097
:10146000584F4646000000000000494E4352454197
:101470005345000044454352454153450000454E05
:1014800041424C450000000044495341424C450054
:101490000000554E465245455A45000046524545C6
:1014A0005A45000000004155544F00000000000064
:1014B00046414E5F4F4E4C59000048494748000096
:1014C000000000004D454449554D000000004C4FC0
:1014D0005700000000000000484541545F434F4F53
:1014E0004C0048454154000000000000434F4F4C61
:1014F00000000000000044525900000000000000FD
:10150000524742000000000000004853560000000F
:1015100000000000636F756C64206E6F7420706152
:101520007273653A2000557064617465640A004501
:101530004550524F4D20636C65617265640A004DE1
:101540005154542050617373776F726420757064C6
:10155000617465640A002B002D00455461673A20D0
:101560000047657420455441473A20004854545080
:101570002F312E310025733A2025730D0A002048A3
:101580005454502F312E310D0A486F73743A202570
:10159000730D0A4163636570743A202A2F2A0D0A7D
:1015A000436F6E6E656374696F6E3A20636C6F7320
:1015B000650D0A0025730020000D0A004745540000
:1015C0006661696C656420746F20636F6E6E65631D
:1015D000740A004552524F523A2053657276657232
:1015E0002072657475726E65642000436F6E666963
:1015F00067206E6F74206368616E6765640A0044DB
:101600006F6E652E0A00436F6E66696720706172A7
:1016100073696E67206661696C65640A004765746A
:101620002061626F7274656400676F7420436F6E2F
:101630006669670A006874747020726574636F6409
:10164000652000667265652000436F6E66696720DD
:101650005552493A20687474703A2F2F002044651F
:101660006661756C7420636F6E666967207365725E
:1016700076657220757365643A20006C617A7968CA
:101680006F6D652E7275000A282D294352595054EA
:10169000000A282D2950554C5345206F6E20504983
:1016A0004E3132000A282D2943414E000A282D29A7
:1016B0004D455243555259000A282D294D554C5439
:1016C0004956454E54000A282B2950574D5F524524
:1016D0004C4159000A282D294D444E53000A282D0B
:1016E0002955415254425249444745000A282B2962
:1016F0005359534C4F47000A282D29504944000A9A
:10170000282D294D43503233303137000A282D29F6
:101710004152544E4554000A282B294F5441000A87
:10172000282D29535049204C4544000A282D294D85
:101730004F544F5220435452000A282B2941432032
:101740004841494552206F6E2053657269616C3380
:10175000000A282D2943435338313120262048449C
:101760004331303830000A282B2952455354415216
:10177000545F4C414E5F4F4E5F4D5154545F455244
:10178000524F5253000A282D294841524452455382
:1017900045542C207573696E6720736F6674000A58
:1017A000282D29434F554E544552000A282D2944CF
:1017B0004854000A282D294F57495245000A282D20
:1017C0002949504D4F44425553000A282D294D4F69
:1017D00044425553000A282D29444D58000A282B0D
:1017E0002957697A6E657435783030000A282B29BC
:1017F0004672656552616D207072696E74696E67BC
:10180000000A282B295741544348444F47006C6134
:101810007A79686F6D652E7275000A436F6E66691E
:1018200067207365727665723A0032303137303333
:101830004C0020432B2B2076657273696F6E3A0043
:10184000303864656436325F323032362D30312DB7
:101850003039000A4C617A79686F6D652E72752097
:101860004C6967687448756220636F6E74726F6C40
:101870006C65722000204F464600204F4E002042EB
:10188000595041535300536176656420746F20456D
:101890004550524F4D00536176696E6720636F6EFD
:1018A00066696720746F20454550524F4D2E2E00BB
:1018B000203C3C200041433A0041433A20536572AA
:1018C00069616C2075736564206279204143202D25
:1018D0002064697361626C696E6720736572696107
:1018E0006C206C6F6767696E6720616E6420636D42
:1018F000640041433A204F7574206F66206D656D1A
:101900006F72790041433A20496E69743A20004170
:10191000433A2044652D496E69743A20004552527D
:101920000041433A20426164204352430041433A1C
:10193000204F4B00203E3E200041433A0041433AB5
:1019400020506F6C6C696E670041433A20556E6D94
:1019500075746500000000000000000000004F4E9C
:1019600000000000000000004F464600000000009C
:10197000000052455354000000000000544F4747F8
:101980004C450000000048414C540000000000009D
:10199000584F4E00000000000000584F464600001F
:1019A00000000000494E4352454153450000444564
:1019B0004352454153450000454E41424C450000CD
:1019C000000044495341424C45000000554E4652E8
:1019D00045455A450000465245455A45000000001D
:1019E0004155544F00000000000046414E5F4F4EED
:1019F0004C590000484947480000000000004D4590
:101A00004449554D000000004C4F570000000000B5
:101A10000000484541545F434F4F4C0048454154F6
:101A2000000000000000434F4F4C00000000000089
:101A300044525900000000000000524742000000DC
:101A400000000000485356000000000000007261D2
:101A500077007175656974007377696E67006C6FE4
:101A6000636B0020696E69740070696E2300726593
:101A70006C61794374723A20002073746F70005265
:101A8000656C61792D4F757420230072656C6179E6
:101A90004374723A200069646C65006F6666006882
:101AA000656174696E670066616E00647279696E63
:101AB0006700636F6F6C696E6700616374696F6E56
:101AC0000020697320004F7574200072656C617985
:101AD0004374723A2000556E6B6E6F776E2073758B
:101AE00066666978200072656C61794374723A2089
:101AF00000556E6B6E6F776E20636D6420007265AB
:101B00006C61794374723A2000616374696F6E008E
:101B100072656C61794374723A20005B305D3A20E3
:101B200000202D202D202D20EFBBBF003E003E3198
:101B3000202D20005B305D3A2000202D202D202D0F
:101B400020EFBBBF003E003E31202D2000537973B3
:101B50006C6F6720726573756D6564005379736C83
:101B60006F6720726573756D6564005379736C6F70
:101B7000672073757370656E646564000000000013
:101B800000636D640000736574000076616C000092
:101B900064656C00004853560000524742000066DE
:101BA000616E00006D6F6465006374726C0068752F
:101BB000650000736174000074656D700072617778
:101BC000000020002E00696E00735F6F7574006D59
:101BD00079686F6D65004354524C2F657865633AA0
:101BE000204F75744F664D656D6F72793A200020F5
:101BF0002D3E20004D5154543A2000202D3E20000F
:101C0000456D69743A203C00202D3E2000497465E2
:101C10006D436D643A2000202D3E20004974656DAF
:101C20003A20003E3E2000496E76616C6964206374
:101C30006F6D6D616E64003E3E3E004E6F204D4103
:101C40004320636F6E666967757265643A207365D9
:101C500074206669726D776172652773204D414308
:101C60000A00454550524F4D207369676E61747587
:101C70007265206F6B00496E697469616C697A697D
:101C80006E6720454550524F4D2E00476F742049D6
:101C90005020616464726573733A00276970205B39
:101CA00069705B2C646E735B2C67775B2C73756259
:101CB0006E65745D5D5D5D27202D207365742073F6
:101CC00074617469632049500A004661696C6564F7
:101CD00020746F20636F6E66696775726520457446
:101CE0006865726E6574207573696E672044484339
:101CF000502E20596F752063616E207365742069C2
:101D000070206D616E75616C6C792100204D4153BE
:101D10004B3A002047573A0020444E533A004C6F4C
:101D2000616465642066726F6D20666C6173682003
:101D300049503A000A7573657320444843500A00BD
:101D40005374617274696E67206C616E0041424326
:101D50004445464748494A4B4C4D4E4F50515253CB
:101D60005455565758595A61626364656667686985
:101D70006A6B6C6D6E6F707172737475767778794B
:101D80007A303132333435363738392B2F3D0042F3
:101D90006173696320003A004F544120696E697491
:101DA00069616C697A65640A0044454641554C5442
:101DB0002070617373776F726420666F72204F5466
:101DC00041204150492E20557365206F7461707712
:101DD0006420636F6D6D616E6420746F2073657431
:101DE0000070617373776F7264004D5154543A20E0
:101DF00074727969796E67206E656E78742062728C
:101E00006F6B6572004D5154543A20546F6F206DC2
:101E1000616E7920636F6E6E656374696F6E2065A5
:101E200072726F72732E2052657374617274204CDB
:101E3000414E002074727920616761696E20696E7D
:101E40002035207365636F6E6473004D5154543AAE
:101E5000206661696C65642C2072633D004D5154AD
:101E6000543A204177616974696E6720666F722009
:101E700072657461696E656420746F706963730064
:101E8000636F6E6E65637465642061732000202E3D
:101E90002E2E0020757365723A003A000A4D515497
:101EA000543A20417474656D7074696E6720636F75
:101EB0006E6E656374696F6E20746F200064697361
:101EC000636F6E6E6563746564005573696E672039
:101ED0004D5154542070617373776F726420667231
:101EE0006F6D20636F6E6669670044657669636530
:101EF000204E616D653A004D5154543A2041742092
:101F00006C6561737420646576696365206E616DCC
:101F10006520616E642062726F6B6572204950208B
:101F20006D75737420626520636F6E666967757284
:101F3000656400757074696D652C667265656865A9
:101F4000617000303864656436325F323032362D6D
:101F500030312D3039004C69676874487562200053
:101F6000246E616D6500526562696E6420737563ED
:101F7000636573732E2049502061646472657373C6
:101F80003A004572726F723A20726562696E64201F
:101F90006661696C0052656E657765642073756370
:101FA000636573732E204950206164647265737396
:101FB0003A004572726F723A2072656E6577656499
:101FC000206661696C000A4E6F206C696E6B00437D
:101FD0006F6E74696E7565207769746820707265BC
:101FE00076696F75736C79206C6F616465642063CA
:101FF0006F6E6669670033307320454550524F4D10
:10200000206973206E6F742072656C6F6164656403
:102010002E205265626F6F74004D5154543A204126
:102020006363657074696E6720636F6D6D616E6464
:10203000732E2E2E0A004E6F204D51545420636F84
:102040006E66696775726564004C6F6164696E677E
:1020500020636F6E6669672066726F6D20706F72A5
:1020600074616C2064697361626C65642E207573A1
:102070006520676574204F4E20746F20656E616225
:102080006C6500436F6E6669672069732076616CCA
:10209000696400436F6E74696E7565207769746852
:1020A0002070726576696F75736C79206C6F6164EE
:1020B000656420636F6E6669670053657475702090
:1020C0004F544100726561647900247374617465D2
:1020D00000757074696D650066726565686561702C
:1020E00000247374617473002045787069726564AC
:1020F0000A00202D746172676574207A6F6E652DF9
:102100000020416C61726D20457870697265640AC7
:102110000020636D643A00204375723A00205365D5
:10212000743A002054696D65723A00204C6F636BFD
:10213000733A0052414D3D00000021002400270069
:102140002A002D00300033000101000004010701C6
:102150000A0100002200250028002B002E0031007B
:10216000340002010000050108010B010505050509
:10217000070508080808020202020A0A08080404FF
:10218000040401010101010101010303030303032D
:102190000303040707070C0C0C0C0C0C0C0C0202BC
:1021A000020206060606060606060B0B0B0B0B0BB9
:1021B0000B0B050505080807070404040A0A0A0AA8
:1021C0000A0A010210202008081020401020408038
:1021D00002010201080402010102040810204080EB
:1021E0008040201008040201800402018040201079
:1021F00008040201080402010102040810204080C2
:10220000010204081020408004408004800810105F
:10221000204004081020408000000B0C030A0D0E23
:102220000F09080405020000000000000000000083
:10223000000000000000000000000000000000009E
:102240000000000013121100000000000000000058
:10225000000000000000000000000000000000007E
:1022600000000000000000000000000000006F639C
:102270007465742F73747265616D006170706C6940
:10228000636174696F6E2F6A736F6E007465787422
:102290002F706C61696E00436F6E74656E742D549F
:1022A0007970653A2000436F6E6E656374696F6E76
:1022B0003A20636C6F7365004163636573732D43EC
:1022C0006F6E74726F6C2D416C6C6F772D4F7269ED
:1022D00067696E3A202A00556E6B6E6F776E004EFE
:1022E0006F74204D6F646966696564004F4B004DE3
:1022F0006F766564207065726D616E656E746C7961
:1023000000496E7465726E616C20536572766572F9
:10231000204572726F72005061796C6F6164205455
:102320006F6F204C61726765004E6F7420666F7529
:102330006E64005757572D41757468656E746963F4
:102340006174653A204261736963207265616C6DE6
:102350003D224163636573732072657374726963B0
:102360007465642200556E617574686F72697A6570
:1023700064005061796C6F61642073697A652077BD
:10238000726F6E6700426164207265717565737467
:1023900000485454502F312E3120002000000000FE
:1023A000000000000000004F4E0000000000000090
:1023B000004F464600000000000000524553540004
:1023C0000000000000544F47474C45000000004803
:1023D000414C54000000000000584F4E0000000027
:1023E000000000584F4646000000000000494E43E0
:1023F0005245415345000044454352454153450031
:1024000000454E41424C45000000004449534142C2
:102410004C45000000554E465245455A4500004681
:102420005245455A45000000004155544F000000F8
:1024300000000046414E5F4F4E4C5900004849474E
:10244000480000000000004D454449554D00000083
:10245000004C4F5700000000000000484541545F09
:10246000434F4F4C004845415400000000000043DA
:102470004F4F4C0000000000004452590000000083
:102480000000005247420000000000000048535680
:102490000000000000000057726F6E6720706179C5
:1024A0006C6164004D5154543A204354524C2F7483
:1024B00078743A204F75744F664D656D6F72793A36
:1024C0002000202D3E2041543A004368616E207464
:1024D0007970653A004E6F2073746F726564207670
:1024E000616C756573202D2064656661756C743A46
:1024F0002000536176656420455441473A00536596
:102500007420455441473A200000A0C623B211244C
:102510001FBECFEFD1E2DEBFCDBF00E00CBF16E0A3
:10252000A0E0B2E0ECE0F8EB01E00BBF02C00790E6
:102530000D92A439B107D9F72DE0A4E9B6E001C0A6
:102540001D92AF34B207E1F712E1C6E8D2E100E034
:1025500006C021970109802FFE010E94D6D3C538FD
:10256000D10780E00807A9F70E9435B20C94F4DB8C
:102570000C940000CF93DF931F92CDB7DEB7698331
:10258000DC01ED91FC910280F381E02D41E050E00F
:10259000BE016F5F7F4F19950F90DF91CF91089526
:1025A000FC01818D928D0895CF93DF931F92CDB75B
:1025B000DEB76983DC01ED91FC910280F381E02DAF
:1025C00041E050E0BE016F5F7F4F19950F90DF91A2
:1025D000CF910895FC019485FB018485981303C075
:1025E00081E0983008F080E00895CF93DF931F9248
:1025F000CDB7DEB76983DC01ED91FC910280F381F8
:10260000E02D41E050E0BE016F5F7F4F19950F90C4
:10261000DF91CF91089585ED8093BC008091BC003F
:1026200084FDFCCF10925107089520912D07260FAD
:102630003327331F21323105ECF420915107FC017F
:1026400090E080E0243069F082E00895A0912D07A9
:102650002191AC01435F584FA40FB52FB11D2C93AE
:102660000196861798F380912D07680F60932D07C8
:1026700080E0089581E008958FEF9FEF08958FEF38
:102680009FEF089580910C0790E0919581959109B5
:102690000895CF93DF93CB01EA01642F0E941513B5
:1026A000CE01DF91CF910895CF93DF931F92CDB7E5
:1026B000DEB7698361E0CE0101960E94151381E0C7
:1026C00090E00F90DF91CF91089590E0FC01E459E4
:1026D000FE4DE491F0E0EE0FFF1FEE5AFE4DA59186
:1026E000B4912C918E539E4DFC018491822391E0F4
:1026F00009F490E0892F0895FC01DC018D9181118E
:10270000FDCF30E020E050E040E08AE09191992355
:1027100001F1443051055CF59E3271F42F3F3105D3
:1027200009F02CF5DB01A40FB51F12962C934F5F17
:102730005F4F30E020E0EACF829FD001839FB00D51
:102740001124292F990F330B205331092A0F3B1FD6
:10275000DDCF2F3F310509F054F4443051053CF4EE
:10276000640F751FFB01228381E090E0089590E0E3
:1027700080E0089590E080E00895DC01ED91FC9107
:102780000284F385E02D1994DF92EF92FF920F936C
:102790001F93CF93DF93EC010C891D89011511055F
:1027A00059F01D8A1C8AC801DF91CF911F910F91AA
:1027B000FF90EF90DF900895EC85FD858E859F85D5
:1027C000DF01A80FB91F2C91243209F055C01196D2
:1027D0002C912B3709F050C00296E80FF91FF12C0D
:1027E000E12CDF01D190DD2009F446C08DE7D81639
:1027F000E9F08FEFE81AF80AF4CF198A188A2C85C5
:102800003D852115310579F08E859F85280F391F6B
:10281000F9012081222321F001969F878E873EC0F7
:102820001D861C86C0CF0FEF1FEFBDCFE114F10452
:1028300019F11C928E859F8502966C857D85680FA7
:10284000791FE881F9810684F785E02DCE0119957D
:10285000998B888B1B8A1A8AEC85FD858E859F85CE
:10286000E80FF91FEE0DFF1DD2828E859F8503961E
:10287000E80EF91EFF86EE86288939892115310573
:1028800009F4BDCF8A899B89280F391FF90120815E
:10289000222309F4B2CF01969B8B8A8B022F220F41
:1028A000110B81CFDC011C96ED91FC911D971E96BA
:1028B0008D919C91E80FF91F8081082E000C990BD7
:1028C0000895DC0115968D919C91009739F0DC01FB
:1028D000ED91FC910680F781E02D1994089583E035
:1028E00090E0089585E090E00895DC011496ED9164
:1028F000FC9180E0309711F085A1817090E00895FF
:102900008FE090E09093CE088093CD0888EC90E023
:102910000895FC01848195810895FC01768765877F
:102920000895DC01ED91FC9102A0F3A1E02D199531
:1029300091E089270895862F089581E086270895DC
:1029400021E0FC018485883008F020E0822F089582
:10295000FC01848595850895FC01848995890895F5
:102960002FE034E0FC0131832083FB014089518951
:1029700062897389FC01428353836483758308955C
:10298000DC01ED91FC91048CF58DE02D1994FC0196
:10299000A7812A2F2E7FC9F081818F7081508330CB
:1029A000A0F4A695A150BB0B2BE531E00E94EDD31E
:1029B00024E630E040E050E00E9481D3DA01C90112
:1029C00087569F4FAF4FBF4F08958FEF9FEF0895EA
:1029D000FC01A681B781109721F118969C91189758
:1029E0009F708EEF890F823010F091111AC01996E6
:1029F0004D935D936D937C931C97A681B781189638
:102A00009C911897907F926018969C930680F7810E
:102A1000E02D8085982F907F903619F48F70806A12
:102A200080870895CF93DF93EC01E881F9810484D6
:102A3000F585E02D199529893A892F5F3F4F3A8B0B
:102A4000298BDF91CF910895CF93DF93EC018E8591
:102A500081110DC081E090E049895A892C853D851E
:102A60004217530708F080E0DF91CF910895E88185
:102A7000F9810484F585E02DCE0119958F3F9105EC
:102A800049F780E090E0F0CFFC01848595856817D8
:102A9000790708F4CB01928B818B0895CF93DF9354
:102AA000FC012685222351F0EC010190F081E02DFC
:102AB0000190F081E02D6FEF19951E86DF91CF9187
:102AC0000895FC0187859089089581E0089590E03C
:102AD00080E00895DC011296ED91FC91309761F051
:102AE0000280F381E02D309739F0862F8295807F28
:102AF00060856F70682B60870895DC011296ED91F8
:102B0000FC91309751F00280F381E02D309729F04D
:102B1000808582958F7090E0089590E080E0089520
:102B2000CF93DF93CDB7DEB760970FB6F894DEBFD3
:102B30000FBECDBF19821A821B821C821D821E828B
:102B40001F8218868A81807F81608A836FEF3E8131
:102B50009F81888529817A815B814C814C873E8762
:102B6000888B372F452F5C857E85892F98896096C5
:102B70000FB6F894DEBF0FBECDBFDF91CF910895A1
:102B80000F931F93CF93DF9300D000D01F921F921B
:102B9000CDB7DEB781E028960FB6F894DEBF0FBE42
:102BA000CDBFDF91CF911F910F910895CF92DF920A
:102BB000EF92FF920F931F93CF93DF9300D000D03B
:102BC000CDB7DEB78C016B017A01FC01808D8830B6
:102BD00010F40E94C0968FE094E09A838983F601F6
:102BE00082819381A481B5818B839C83AD83BE83D5
:102BF000B701CE0101960E947FA7F801808F88302F
:102C0000A0F4F586E486128E118E81E026960FB62A
:102C1000F894DEBF0FBECDBFDF91CF911F910F9112
:102C2000FF90EF90DF90CF90089580E0EFCFCF93AB
:102C3000DF93EC01888D883020F40E94C09688E0F4
:102C4000888FDF91CF910895FC01808D883040F40A
:102C5000218D328D232B21F00E94929590E00895D2
:102C60008FEF9FEF0895CF93DF93FC0124852830E9
:102C700028F08FEF9FEFDF91CF910895EC01019045
:102C8000F081E02D0084F185E02D1995892B89F3E1
:102C90008C850E94929590E0EECFCF93DF93FC015C
:102CA000218D328D2115310529F48FEF9FEFDF91B2
:102CB000CF910895EC01808D4217530708F0A901C8
:102CC0000E94E1951816190684F7298D3A8D281B64
:102CD000390B3A8F298FEBCF0F931F93CF93DF934D
:102CE0001F92CDB7DEB7FC01218D328D232B41F42D
:102CF0008FEF9FEF0F90DF91CF911F910F9108956C
:102D00008C0141E050E0BE016F5F7F4FFC01808D80
:102D10000E94E195181619065CF7F801818D928DD5
:102D20000197928F818F898190E0E4CFCF93DF93D9
:102D30001F92CDB7DEB741E050E0BE016F5F7F4F1D
:102D4000FC0184850E94E1951816190634F48981E6
:102D500090E00F90DF91CF9108958FEF9FEFF9CF23
:102D6000FC018485883010F40C94E19590E080E0BB
:102D70000895FC018485883010F40C94BA9590E095
:102D800080E008950F931F93CF93DF9300D000D07E
:102D90001F921F92CDB7DEB78C01D80159964D9185
:102DA0005C915A974115510551F0ED91FC91048CBD
:102DB000F58DE02D70E060E0C8011995EECFF801C7
:102DC000808D0E94BA95892BB1F148E050E0BE0198
:102DD0006F5F7F4FD80158968C910E94E19518162D
:102DE0001906F4F4D801509684E0FE013196019062
:102DF0000D928A95E1F78D8190E0982F88272E819A
:102E0000820F911DF801958B848B8F81282F30E0E4
:102E1000322F22278885820F932F911D928F818FC9
:102E200028960FB6F894DEBF0FBECDBFDF91CF91CD
:102E30001F910F91089590E080E0F2CFCF92DF9242
:102E4000EF92FF920F931F93CF93DF93CDB7DEB72F
:102E5000AF970FB6F894DEBF0FBECDBF7C016A01FD
:102E60000FE014E01A8309831C861B8688EE93E02A
:102E7000A0E0B0E08D879E87AF87B88B85EE93E0AA
:102E80009A878987188F0F8B198E1A8E1B8E1C8E2E
:102E900088E089A31BA70AA71CA61DA61EA61FA61D
:102EA0008091CE0A9091CF0AA091D00AB091D10A18
:102EB0008EA39FA3A8A7B9A78B839C83AD83BE8352
:102EC00018861F82AE01465D5F4FCE0101960E94BB
:102ED00042AD81309105B1F4D701ED91FC910488A8
:102EE000F589E02D1DA30CA38CA59DA5AEA5BFA5BE
:102EF0008EA39FA3A8A7B9A7A601BE016C5D7F4FB3
:102F0000C7011995AF960FB6F894DEBF0FBECDBFBF
:102F1000DF91CF911F910F91FF90EF90DF90CF90B5
:102F200008950F931F93CF93DF93EC018B01888D4E
:102F3000883010F40E94C096B80182E00E94099780
:102F4000888F883050F41D870C871A8E198E81E087
:102F5000DF91CF911F910F91089580E0F9CF0F93EA
:102F60001F93CF93DF938C01EA01FC0184858830A5
:102F700048F40E943095892B39F481E090E0F80103
:102F800093838283D0E0C0E0CE01DF91CF911F9187
:102F90000F910895EF92FF920F931F93CF93DF93BA
:102FA0007C018091BA08D4E0833309F0D8E00AEAC2
:102FB00018E0C0E0F801219131918F01F70184817F
:102FC00095812817390729F0CF5FDC13F3CF80E014
:102FD00006C08C2F0E94CE968431B1F781E0DF913C
:102FE000CF911F910F91FF90EF900895CF93DF93B2
:102FF000EC018C858830D0F40E94CE96843189F023
:10300000882379F0883169F021E08C3159F4E88126
:10301000F9810084F185E02DCE01199521E0892BFD
:1030200009F420E0822FDF91CF91089580E0FBCF5B
:103030006F927F928F929F92AF92BF92CF92DF92C8
:10304000EF92FF920F931F93CF93DF938C015B015D
:103050007A018091BA08882309F46CC024E0622EBA
:10306000833311F098E0692E8AEAC82E88E0D82EC2
:103070004601712CC0E0D4012D913D914D01F80124
:10308000848195812817390799F48C2F0E94CE9658
:10309000D82F873119F08C3109F040C08C2F0E9455
:1030A000BA95892B29F4DC3119F48C2F0E94B29641
:1030B000CF5F6C12E0CF711008C0D801ED91FC9188
:1030C0000084F185E02DC8011995D0E0F601219129
:1030D00031916F01D80114968D919C912817390771
:1030E00051F48D2F0E94CE96873129F4A701B501A6
:1030F0008D2F0E943095DF5FDC13E8CFC701DF9191
:10310000CF911F910F91FF90EF90DF90CF90BF90E4
:10311000AF909F908F907F906F900895843139F099
:103120008111C6CFF401329711821082C1CF77246A
:103130007394BECFF12CE12CE1CFCF92DF92EF92CE
:10314000FF920F931F93CF93DF93CDB7DEB7AF9767
:103150000FB6F894DEBF0FBECDBF8C016B017A01B4
:103160008FE094E09A8389831B821C821D821E82D9
:103170001C861B8648EE53E060E070E04D875E875A
:103180006F87788B25EE33E03A872987988F8F8B6E
:10319000198E1A8E1B8E1C8E28E029A39BA78AA746
:1031A0001CA61DA61EA61FA6D8011C968C918830B1
:1031B00060F40E94CE96882321F0F80184850E9455
:1031C000B29688E0D8011C968C938091CE0A90919B
:1031D000CF0AA091D00AB091D10A8EA39FA3A8A72D
:1031E000B9A78B839C83AD83BE8318861F82AE01F3
:1031F000465D5F4FB601CE0101960E9442AD009739
:10320000C1F0D801ED91FC910684F785E02D8FE0A7
:1032100094E09DA38CA38CA59DA5AEA5BFA58EA370
:103220009FA3A8A7B9A7A701BE016C5D7F4FC801E6
:103230001995AF960FB6F894DEBF0FBECDBFDF91E4
:10324000CF911F910F91FF90EF90DF90CF90089555
:10325000CF93DF93EC018C85883060F40E94CE968A
:10326000873111F08C3131F48C850E9413958115D2
:10327000984088F3DF91CF910895FC0184858830D0
:1032800010F40C94139590E080E0089565E0FC0143
:10329000828193810E94439B009749F0FC018085C5
:1032A000982F907F21F082958F7090E0089590E0A4
:1032B00080E00895CF92DF92EF92FF926A017B0146
:1032C00063E0FC01828193810E94439BFC01892B76
:1032D000A9F080858D7091F4C094D094E094F0941E
:1032E000CC24CA9481859285A385B4858C219D21A7
:1032F000AE21BF2181879287A387B487FF90EF908B
:10330000DF90CF900895CF92DF92EF92FF926A0103
:103310007B0163E0FC01828193810E94439BFC015D
:10332000892BA9F09085892F8D7089F4907F926008
:103330009087CC24FF2441855285638574854C2970
:103340005D296E297F294187528763877487FF90A3
:10335000EF90DF90CF900895CF92DF92EF92FF929F
:103360006A017B0163E0FC01828193810E94439B9F
:10337000009791F0FC0120852F70223069F461855F
:103380007285838594856C217D218E219F21FF90FC
:10339000EF90DF90CF90089560E070E0CB01F7CF21
:1033A000CF93C62F63E0FC01828193810E94439BEF
:1033B000FC01892B91F09085892F8D7071F4907F9D
:1033C0009260908781859285A385B4858827BB27E5
:1033D0008C2B81879287A387B487CF91089566E568
:1033E00075E1811102C068E575E185E59BE00C940B
:1033F000C8896DE772E185E59BE00E94C889F0E02D
:10340000E0E0199584EF91E0089567EA7AE0811190
:1034100002C062EA7AE086E09CE00C94C889DC0194
:1034200055962C915597273781F4ED91FC91008C9E
:10343000F18DE02D199561ED76E086E09CE00E942B
:10344000C88986E09CE00C94418808950C9483CA56
:103450000C9483CA0C9483CAEF92FF920F931F932C
:10346000CF93DF93EC018B0180910A0790910B07BA
:103470000097A9F0FC0120852F70263081F40E946E
:10348000CB9AFC0190859F70943049F48185928598
:10349000DF91CF911F910F91FF90EF900895EE88EB
:1034A000FF88C70101970D97D0F461E174E0C8016E
:1034B0000E9437D8892B99F48FE2888F85E08E9D02
:1034C000B0018F9D700D11246458744E46E050E099
:1034D000CE0149960E9457CCCE014896D9CF90E0B4
:1034E00080E0D6CFCF93C1E068EE73E080E090E05B
:1034F0000E9479A94AE050E06C2F85E59BE00E948C
:103500004588CF5FC43181F784EF91E0CF91089572
:10351000EF92FF920F931F93CF93DF936115710585
:1035200011F480E090C0EB018C0188858F708230AF
:1035300009F442C08430A9F762E077E086E09CE0BD
:103540000E94C8894AE050E0F801638186E09CE06F
:103550000E94458865E174E086E09CE00E947189E4
:1035600069857A8586E09CE00E94718986E09CE00E
:103570000E944188F801E080F180E114F10489F2B1
:103580006AE174E0C7010E94CB9A8C01009749F26E
:10359000FC0180858F70863021F669857A856115FA
:1035A000710509F44CC0FB018081882309F447C0F0
:1035B000C8010E94CB9A42C065EF76E086E09CE0AD
:1035C0000E94C8894AE050E0F801638186E09CE0EF
:1035D0000E94458865E174E086E09CE00E94718964
:1035E00049855A856B857C852AE030E086E09CE041
:1035F0000E94E78886E09CE00E944188F801E08014
:10360000F180E114F10409F48CCF6AE174E0C701A0
:103610000E94CB9A8C01009709F483CFFC0180852E
:103620008F708550823008F07CCF6985862F9A850F
:10363000892B29F06150C8010E94439B7C01F8014D
:10364000F286E18681E0DF91CF911F910F91FF908B
:10365000EF900895EF92FF920F931F93CF93DF9314
:103660000097C1F0FC0120812223A1F08C0180E5AC
:10367000E82E8BE0F82EC1E0D0E0B701C8010E942F
:1036800020CC892B49F02196F5E0EF0EF11CCE30CD
:10369000D10599F7D0E0C0E0CE01DF91CF911F9125
:1036A0000F91FF90EF900895CF93DF93EC016BE8BB
:1036B0007AE186E09CE00E94C8896FE77AE186E0C3
:1036C0009CE00E94C8896C817D8186E09CE00E941C
:1036D000399F69E77AE186E09CE00E94C88986E02C
:1036E0009CE00E94418860E08C810E94F8A8E881FB
:1036F000F9810484F585E02D60E0CE01199581E023
:1037000090E0DF91CF910895CF93DF9300D000D068
:103710001F921F92CDB7DEB7EFE3FBE0128A118A4A
:1037200080E090E19587848784E890E0948B838B98
:1037300081E0868780E090E2908B878787E7858BA2
:103740001C821B8283E892E09A838983FE83ED8347
:103750008FEF9FEF98878F8366E978E185E59BE09F
:103760000E94C8896091AC067091AD06CE010196A9
:103770000E9476A08FE39BE00E940F1A66E878E132
:1037800085E59BE00E94C88985E59BE00E94418811
:103790000E9472B028960FB6F894DEBF0FBECDBF60
:1037A000DF91CF910895892B71F0FB018281938184
:1037B0000E948A9C6FE375E185E59BE00E94C889C1
:1037C00088EC90E0089590E080E0F2CF0F931F9393
:1037D000CF93DF93EB0102970CF483C00A811B8126
:1037E00064E274E1C8010E9402CC892B51F481E0AB
:1037F0000E941A9F88EC90E0DF91CF911F910F916A
:1038000008956EE274E1C8010E9402CC892B11F484
:1038100080E0EECF6AEF73E185E59BE00E94C88906
:103820000E947A9E672F6095617070E085E59BE04D
:103830000E94399F85E59BE00E9441888091310B71
:103840009091320B892BE9F10A811B810E941B9C0C
:103850008823B9F1F80101900020E9F73197E01BC6
:10386000F10BB09770F582E70E94069C8091310BB6
:103870009091320BDC01ED91FC910088F189E02DF3
:1038800060E270E01995B8018091310B9091320B94
:103890000E9471898091310B9091320BDC01ED9186
:1038A000FC910190F081E02D60E019958091310B41
:1038B0009091320BDC01ED91FC910488F589E02DAB
:1038C00019956A817B8185E59BE00E94718963EF90
:1038D00073E185E59BE00E94C88985E59BE00E9435
:1038E00041888091CD089091CE0802973CF080EFFE
:1038F0009FEF9093CE088093CD087CCF66EE73E166
:103900008FE59BE00E94C8898FE59BE00E9441887B
:1039100084EF91E071CF892B71F0FB01828193815B
:103920000E94D89C60ED73E185E59BE00E94C88908
:1039300088EC90E0089590E080E0F2CFEF92FF9263
:103940000F931F93CF93DF93CDB7DEB72C970FB6AE
:10395000F894DEBF0FBECDBF8C017B018FE094E0F9
:103960009A8389831B821C821D821E8298878F8383
:1039700019861A861B861C8605301105ECF0BE01DF
:10398000695F7F4FF701808591850E947C13892BA9
:1039900099F0CE0107960E947B9DBE01695F7F4F23
:1039A000F701868197810E947C13892B61F0CE01FB
:1039B00007960E94259E0EC0CE0101960E947B9D17
:1039C0000430110554F7CE0101960E94259E033064
:1039D0001105A4F1BE01695F7F4FF70184819581D4
:1039E0000E947C13892B51F1CE0107960E94D09D35
:1039F000BE01695F7F4FF701828193810E947C1332
:103A0000892B19F1CE0107960E94269D69EB73E17F
:103A100085E59BE00E94C88980E00E94119F88ECA8
:103A200090E02C960FB6F894DEBF0FBECDBFDF91AD
:103A3000CF911F910F91FF90EF900895CE010196C5
:103A40000E94D09D023011059CF6CE0101960E9485
:103A5000269D01301105D1F6CE0101960E94269DCA
:103A600060EC73E185E59BE00E94C889CFCF0F939E
:103A70001F93CF93DF938C01EB010297C4F08A81EF
:103A80009B810E94B4CB80932A0299270E94249F95
:103A90000230110549F08C819D810E94B4CB809346
:103AA000290299270E942E9FC8ECD0E002C0C0E9ED
:103AB000D1E065EA73E185E59BE00E94C8894AE0B0
:103AC00050E060912A0285E59BE00E94458860E90C
:103AD00073E185E59BE00E94C8894AE050E060916F
:103AE000290285E59BE00E94458885E59BE00E94D0
:103AF0004188CE01DF91CF911F910F910895CF930F
:103B0000DF93EB010297ACF164E274E18A819B815F
:103B10000E9402CC892B29F40E947A9E7D7F0E940C
:103B2000C19E6EE274E18A819B810E9402CC892B46
:103B300029F40E947A9E72600E94C19E6FE773E131
:103B400085E59BE00E94C8890E947A9E71FB6627EA
:103B500060F971E0672770E085E59BE00E94399F7E
:103B600085E59BE00E94418888EC90E0DF91CF9151
:103B700008950E94841BF8CF0F931F93CF93DF9378
:103B8000FC01738362836115710509F448C08B01E0
:103B9000EC011682CB010E949A9F97FD45C09D8340
:103BA0008C838C819D81009719F08635910524F0D6
:103BB00080E290E09D838C83F801048115810115DA
:103BC000110509F440C0F80180858F708530D9F562
:103BD000C8010E948A9F8230B0F161E0C8010E9452
:103BE000439BFC01892B79F180858F70823021F510
:103BF00061857285838594850E941CD220E030E027
:103C00004AE754E40E947BD20E94DAD46115710520
:103C100081059105E1F06F83788789879A87DF9125
:103C2000CF911F910F9108959195819591099D8351
:103C30008C8381E08E83B5CF833029F461857285D2
:103C400083859485DBCF60E070E0CB01D7CF88E837
:103C500093E1A0E0B0E08F839887A987BA87DFCF90
:103C60000F931F93CF93DF93EC017B836A836115DE
:103C7000710509F442C0FB01A085B185109771F16F
:103C800018968C9118978F70823041F516968D9109
:103C90009C919D838C8380ED98E098878F83FB01B6
:103CA000A481B581109709F18B0118969C91189702
:103CB0009F70923039F09530C1F4CD010E948A9FF7
:103CC000882399F0C8010E949A9F8E83813091F0D9
:103CD00040F0823051F48DE699E005C090E080E03C
:103CE000D8CF89E69BE098878F83DF91CF911F9192
:103CF0000F9108958AE09AE0F6CF1D821C82F5CFDD
:103D00002F923F924F925F926F927F928F929F92EB
:103D1000AF92BF92CF92DF92EF92FF920F93CF9329
:103D2000DF9300D01F92CDB7DEB77C017A83698321
:103D30005C834B83DB011C92FC0160818FEF860F5B
:103D4000883108F04BC034FF49C0FAE06F9FB001E2
:103D5000112463567C4DCD010E9457CCD70111969A
:103D60008C918F7041F04B815C8160EB74E08981B4
:103D70009A810E9447D8E981FA8101900020E9F7F1
:103D8000319729813A81E21BF30B19012E0E3F1E58
:103D90004B815C814E1B5F0B415051095C834B830F
:103DA000D7011196EC911197EF7009F4F5C0E1502D
:103DB000EC3008F0F1C0F0E08827EE51F14E8F4F63
:103DC0000C94D6D3F11E941F012060207B203F1F4E
:103DD0001120112011202D1F151F972029803A80B6
:103DE000DFCFF7018481282F30E050E040E000234E
:103DF00059F030E0A4E6B0E00E94B3D32FEF30E0FA
:103E000040E050E00E9481D35F934F933F932F9304
:103E10008EE194E09F938F93FC81FF932B812F93EE
:103E20003F922F920E947FD8B2C017968C9117971D
:103E30008F9316968C9116978F9315968C91159754
:103E40008F9314968C918F9381E294E09F938F933C
:103E5000BC81BF93EB81EF93E3CF17968C911797BB
:103E60008F9316968C9116978F9315968C91159724
:103E70008F9314968C918F9385E294E0E7CF1496FC
:103E8000CD90DD90ED90FC901797F7FE34C084E65E
:103E9000882E912CA12CB12CC701B601A50194014B
:103EA0000E9481D39B01AC0188279927DC01821BEA
:103EB000930BA40BB50BBF93AF939F938F93662780
:103EC0007727CB016C197D098E099F09A501940103
:103ED0000E9481D35F934F933F932F9389E294E0A5
:103EE0009F938F933C813F934B814F933F922F92AF
:103EF0000E947FD84CC0C701B60124E630E040E004
:103F000050E00E9481D39F938F937F936F935F9331
:103F10004F933F932F938AE294E09F938F939C81DA
:103F20009F93AB81AF93E2CFC7010E94C714BC013E
:103F3000D7011696CC9016971796DC901797D0FA63
:103F4000DD24D0F814969C9114971596FC90EB8084
:103F5000BC80292F30E050E040E077FD35C00111F2
:103F600035C07F936F931F921F921F929F931F9252
:103F7000FF92DF92CF9283E394E09F938F93FC8133
:103F8000FF932B812F933F922F920E947FD80FB6E1
:103F9000F894DEBF0FBECDBF89819A810F900F903C
:103FA0000F900F90DF91CF910F91FF90EF90DF90E6
:103FB000CF90BF90AF909F908F907F906F905F90C9
:103FC0004F903F902F900895002361F0292F30E00B
:103FD000A4E6B0E00E94B3D32FEF30E040E050E021
:103FE0000E9481D35F934F933F932F931F92FF9231
:103FF000DF92CF9286E394E09F938F93BF92EF92EC
:1040000075CF15968C9115971F928F9316969C914C
:10401000169717968C9181708F939F9389E394E004
:1040200015CF14968D909D90AD90BC90179720E081
:1040300030E0A901C501B4010E9415D22401350167
:1040400087FF04C077FA709477F87094C301B201C7
:104050000E94D3D46B01072E000C880B990B0E9491
:104060001CD29B01AC01C301B2010E94F4D320E039
:1040700030E04AE754E40E947BD20E945ED50E9461
:10408000D3D4062F772E20E030E0A901C501B4017A
:104090000E9415D287FF07C07F920F93DF92CF92C5
:1040A0008FE394E0D3CE7F920F93DF92CF9280E4A0
:1040B00094E09F938F933C813F934B814F93B0CE7D
:1040C00014968C9114971F928F9315968C91159737
:1040D0001F928F9316968C911F928F9386E394E094
:1040E0009F938F93BC81BF93EB81EF933F922F926D
:1040F0000E947FD84CCF17968C9117971F928F9361
:1041000014968C9114971F928F9315968C911597F6
:104110001F928F9316968C911F928F9383E394E056
:104120009F938F93BC81BF93EB81EF93DFCE149667
:104130006D917C914B815C81C1010E9465D82CCF2F
:10414000EF92FF920F931F93CF93DF93EC017B01CC
:1041500088859985892BA9F48A819B810E948A9FF1
:10416000082F10E00530110564F40E947D9F9987A7
:104170008887BC018A819B810E945F9F0F5F1F4FD0
:10418000F1CFE885F9853097D9F08085982F9F7019
:10419000A9F4807F82608087E885F9851186128680
:1041A00013861486E885F985F782E682C701DF91D8
:1041B000CF911F910F91FF90EF900895923061F38E
:1041C000F12CE12CF3CFCF93DF93FC0122813381DB
:1041D000232B59F1EC016FE079E186E09CE00E942D
:1041E000C8894AE050E06E8186E09CE00E944588E4
:1041F00086E09CE00E9441888C819D810E9483CA58
:1042000070E060E08A819B810E94A0201D821C8258
:10421000E881F9810484F585E02D60E0CE011995EF
:1042200081E090E0DF91CF91089590E080E0FACFB7
:104230001F93CF93DF93FC01162FC389D489818903
:1042400092899C012F5F3F4F328B218BC80FD91F62
:10425000CE010E9439D3181721F0612FCE010E94A0
:1042600041D381E090E0DF91CF911F910895FC014F
:1042700081899289248535858217930740F42389A3
:104280003489820F931F0E9439D390E008958FEFF5
:104290009FEF0895EF92FF920F931F93CF93DF93B9
:1042A000CDB7DEB760970FB6F894DEBF0FBECDBFB7
:1042B0007B01CA01B9012AE0AE014F5F5F4F0E9446
:1042C000C4CCA801BE016F5F7F4FC7010E9497AAAF
:1042D00060960FB6F894DEBF0FBECDBFDF91CF91D1
:1042E0001F910F91FF90EF900895DA01E091570729
:1042F000F0E0FE2FEE27E60FF71F90E0982F8827BB
:10430000A901BD018E0F9F1F0C948592CF93DF935F
:104310001F92CDB7DEB72091570730E0322F22270A
:10432000260F371F90E0982F8827498341E050E0FF
:10433000BE016F5F7F4F820F931F0E9485920F9087
:10434000DF91CF910895CF93DF931F92CDB7DEB762
:1043500041E050E0BE016F5F7F4F0E94FA9189817A
:104360000F90DF91CF9108952091570730E0322FC1
:104370002227620F731F90E0982F8827860F971FC0
:104380000C94A32163E070E00C94B421DA01E09175
:104390005707F0E0FE2FEE27E60FF71F90E0982F6B
:1043A0008827A901BD018E0F9F1F0C94FA9144E04C
:1043B00050E0BC018FE090E00C94859244E050E026
:1043C000BC0185E090E00C94859244E050E0BC0193
:1043D00081E090E00C94859208959F92AF92BF92F5
:1043E000CF92DF92EF92FF920F931F93CF93DF93C1
:1043F0008C015B01942EE52EFC01C688D788F08CD9
:1044000080E591E00E9489A48F2D0E94D694C92D49
:10441000DE2D8C179D0708F4EC019E01A501B60165
:104420008F2D0E945394F801868997898C0F9D1FC8
:10443000978B868BCE01DF91CF911F910F91FF90CB
:10444000EF90DF90CF90BF90AF909F900895CF9363
:10445000FC01C08D80E591E00E9489A460E270E0DB
:104460008C2F0E94EA9162E070E08C2F0E94B421B0
:1044700084FD16C062E070E08C2F0E94B42183FF9F
:104480000AC048E162E070E08C2F0E94862180E043
:1044900090E0CF91089580E591E00E9489A4E3CF58
:1044A00040E162E070E08C2F0E94862181E0F0CF35
:1044B000FF920F931F93CF93DF93EB01FC01178AB9
:1044C000168A2A81211109C02B81211106C02C8155
:1044D000211103C02D81222301F141155105E9F07D
:1044E0008A01FC01F08C80E591E00E9489A4AE0174
:1044F0004E5F5F4F24E030E06CE070E08F2D0E9453
:104500007521B8018F2D0E94DD9681E090E0DF914A
:10451000CF911F910F91FF90089580E0F7CF0F93F7
:104520001F93CF938C01FC016481758181E20E940D
:104530000997C82F8830F8F480E591E00E9489A49B
:104540008C2F0E94C221833131F08C2FCF911F918B
:104550000F910C94B29662E070E08C2F0E94EA9169
:10456000F80184819581EC2FF0E0EE0FFF1FE655F6
:10457000F74F91838083CF911F910F9108950F93EF
:104580001F93CF93DF931F921F92CDB7DEB7FC012D
:1045900024852830E0F48C0180E591E00E9489A414
:1045A00022E030E0AE014F5F5F4F60E170E0F80164
:1045B00084850E94C62189819A8198278927982716
:1045C0000F900F90DF91CF911F910F91089590E080
:1045D00080E0F6CF0F931F93CF93DF931F921F922C
:1045E000CDB7DEB7FC0124852830E0F48C0180E5EE
:1045F00091E00E9489A422E030E0AE014F5F5F4F5E
:1046000064E070E0F80184850E94C62189819A8166
:104610009827892798270F900F90DF91CF911F91AE
:104620000F91089590E080E0F6CFCF93DF93EC01F7
:104630008FE094E0998388831A821B821C821D82FA
:1046400080E591E00E9489A4BE016E5F7F4F44E047
:1046500050E08FE090E00E94FA91CE01DF91CF917F
:1046600008950E944693882331F08091BA088433DC
:1046700029F0873381F090E080E0089580E591E0B3
:104680000E9489A485E390E00E94A32185FD0DC0CE
:1046900082E090E0089580E591E00E9489A48EE296
:1046A00090E00E94A32180FFF3CF81E090E0089585
:1046B0001F920F920FB60F9211240BB60F922F93E9
:1046C0003F934F935F936F937F938F939F93AF939A
:1046D000BF93EF93FF938091B900887F803609F4F0
:1046E0004DC008F040C0883209F4A7C028F58031D9
:1046F00009F49BC0C8F4882309F4F1C0883009F498
:1047000094C0FF91EF91BF91AF919F918F917F9155
:104710006F915F914F913F912F910F900BBE0F9032
:104720000FBE0F901F901895883109F486C0803213
:1047300041F78093500714C0803409F497C040F4C7
:104740008033B9F38833E9F68093500785ECA8C02D
:10475000803509F481C0883509F490C0883489F621
:104760000E940B13CECF883909F486C038F58837FC
:1047700029F050F4883611F0803719F683E08093E1
:10478000510710924F0755C0883809F475C0803919
:1047900019F0803809F0B5CF80914F07803208F0CA
:1047A0006BC0E0914F0781E08E0F80934F0780919F
:1047B000BB00F0E0E15DF84F80833BC0803B39F007
:1047C000D0F4803A09F471C0883A09F09ACF84E0B5
:1047D0008093510710922E0710922D07F0E0E0E031
:1047E000199580912D0781110FC081E080932D07CD
:1047F00010920D0709C0803C09F4A8CF883C09F449
:10480000A5CF883B09F07DCFE0912E0781E08E0F88
:1048100080932E07F0E0E35FF84F80818093BB0028
:1048200090912E0780912D0725C080915607809387
:10483000BB0085EC8093BC0064CF909155078091BC
:104840005407981728F5E091550781E08E0F809363
:104850005507F0E08081EBCFE091550781E08E0FA6
:10486000809355078091BB00F0E0808390915507BD
:10487000809154079817E8F285E8DCCFE09155075E
:1048800081E08E0F809355078091BB00F0E080831C
:1048900080915307811164CF81E08093520784EAAD
:1048A0008093BC00109251072CCF85EC8093BC0004
:1048B0001092510780914F07803230F4E0914F07FA
:1048C000F0E0E15DF84F108260914F0770E08FE2F9
:1048D00097E0F0E0E0E0199510924F0712CF1092A8
:1048E00050073ECF009789F0FC0120852F702530BE
:1048F00061F40E94439B009741F0FC0120852F70DA
:10490000243019F481859285089590E080E008951F
:10491000CF92DF92EF92FF920F931F93182F6A01AD
:104920007B010E94ABA904C0969587957795679502
:104930001A95D2F76C217D218E219F218B019C013C
:1049400001501109210931090E3F1F4F2F4F3F4FD1
:1049500020F061E070E080E090E01F910F91FF9007
:10496000EF90DF90CF9008953F924F925F926F92B9
:104970007F928F929F92AF92BF92CF92DF92EF92EF
:10498000FF920F931F93CF93DF9300D000D0CDB74A
:10499000DEB77C01362E80910907882309F40DC10A
:1049A000D70114969C9180912902891708F405C1BA
:1049B0008091070790910807BAE06B1318C28E54D4
:1049C000994FFC011082D70118968D919C91892BEB
:1049D00009F4EFC08091AE069091AF06A091B006A9
:1049E000B091B106892B8A2B8B2B09F0CEC00E9487
:1049F000ABA92B013C01F70100851185D80119965F
:104A00006D917C916115710599F4F801858096800E
:104A1000A780B0848091C80A9091C90AA091CA0A5F
:104A2000B091CB0A88169906AA06BB0609F487C07E
:104A3000D8011B964D915C911C974115510509F4C5
:104A40007EC0F701248153968C91539790E0322FCA
:104A5000377002C0959587953A95E2F780FF6FC051
:104A6000C22ED12CC601887F9370892B39F45196C0
:104A70008D919C91887F9370C82AD92AD8018D91F5
:104A80009C91DC01ED91FC916115710509F4C4C0A4
:104A90000688F789E02D1995019709F050C06CE35D
:104AA000F801808191810E94E088A60170E060E0B9
:104AB0002AE0D8018D919C910E94F587F80122810E
:104AC000808191816EE27BE1222311F06CE27BE137
:104AD0000E94C889D8011D966D917C911E978D9179
:104AE0009C910E94718960E2F801808191810E940D
:104AF000E088D8011F966D917C9150978D919C9183
:104B00000E947189F80122818081918161E27BE1BB
:104B1000222311F06BE17BE10E94C88962EB76E011
:104B2000D8018D919C910E947189F80180819181B9
:104B3000DC01ED91FC91008CF18DE02D19950E9426
:104B4000ABA9AB01BC014419550966097709F70106
:104B500085819681453651056105710508F472C05D
:104B6000009721F06BE67BE10E94EC894FEF5FEF4D
:104B7000BA0180E00E9488246093AE067093AF066D
:104B80008093B0069093B10614C00E94ABA9009127
:104B9000AE061091AF062091B0063091B106601BB1
:104BA000710B820B930B603375478105910508F0FB
:104BB0001ECF1092080710920707D70115968D9106
:104BC0009C911697009771F014963C9120912A02BF
:104BD000231740F0DC01ED91FC910190F081E02D74
:104BE000632D199581E090E026960FB6F894DEBF0C
:104BF0000FBECDBFDF91CF911F910F91FF90EF902E
:104C0000DF90CF90BF90AF909F908F907F906F90EC
:104C10005F904F903F9008950488F589E02D2FE034
:104C200034E03A832983D80115968D909D90AD90FC
:104C3000BC9018978B829C82AD82BE82BE016F5F52
:104C40007F4F29CF4091AE065091AF066091B006DC
:104C50007091B106452B462B472B09F4AACF00973C
:104C600021F06CE57BE10E94EC891092AE06109277
:104C7000AF061092B0061092B106D70118960D91AA
:104C80001C91F801618572856115710591F445806B
:104C90005680678070848091C80A9091C90AA0915B
:104CA000CA0AB091CB0A481659066A067B0609F46F
:104CB00080CFD8011B964D915C911C9741155105F1
:104CC00009F477CFF701248153968C91539790E0A4
:104CD000322F377002C0959587953A95E2F780FF9D
:104CE00068CFC22ED12CC601887F9370892B39F4EE
:104CF00051968D919C91887F9370C82AD92AD801AA
:104D00008D919C91DC01ED91FC916115710509F487
:104D100058C00688F789E02D1995019709F049CF09
:104D20006CE3F801808191810E94E088A60170E027
:104D300060E02AE0D8018D919C910E94F587F801EE
:104D400022818081918167E47BE1222311F065E477
:104D50007BE10E94C889D8011D966D917C911E97B8
:104D60008D919C910E94718960E2F801808191810E
:104D70000E94E088D8011F966D917C9150978D918B
:104D80009C910E947189F8012281808191816AE35E
:104D90007BE1222311F064E37BE10E94C8896DE48A
:104DA0007BE1D8018D919C910E94C889F801808196
:104DB0009181DC01ED91FC91008CF18DE02D199534
:104DC000F8CE0488F589E02D2FE034E03A8329837A
:104DD000D80115964D905D906D907C9018974B8200
:104DE0005C826D827E82BE016F5F7F4F95CF84357E
:104DF00091050CF0E2CEBDE06B1709F4DECE9C010C
:104E00002F5F3F4F30930807209307078E54994F29
:104E1000FC016083D2CECF92DF92EF92FF920F938C
:104E20001F93CF93DF93EC01EC81FD81309709F460
:104E3000A4C08A819B81892B09F49FC0808188232B
:104E400009F49BC07A016B01E881F9810284F38542
:104E5000E02DCE0119950397D9F4EC81FD8180A551
:104E600091A5A2A5B3A5892B8A2B8B2B89F00E9433
:104E7000ABA9EC81FD8100A511A522A533A5601B7E
:104E8000710B820B930B663971058105910528F32F
:104E90008F81988521E0E21AF108DC01ED91FC9107
:104EA0000280F381E02DA701B60119958F819885C5
:104EB000DC01ED91FC910190F081E02DD60112967C
:104EC00060E09D012C193D092E153F0518F42D9128
:104ED000620FF7CF19950C811D814FEF5FEFBA017B
:104EE00080E00E948824F80160A771A782A793A799
:104EF00065EB78E186E09CE00E94C8894AE050E0DA
:104F00006E8186E09CE00E94458860EB78E186E057
:104F10009CE00E94C8898601C8018C199D098E15E4
:104F20009F05B8F4D8016C9140E150E06A3050F42C
:104F300068E474E086E09CE00E94718940E150E002
:104F4000F801608186E09CE00E9445880F5F1F4F5A
:104F5000E3CF86E09CE00E944188E881F9810484E7
:104F6000F585E02D63E0CE01DF91CF911F910F9188
:104F7000FF90EF90DF90CF901994DF91CF911F9128
:104F80000F91FF90EF90DF90CF9008958F929F92B6
:104F9000AF92BF92CF92DF92EF92FF920F931F9347
:104FA000CF93DF937C014A015901C0910A07D09148
:104FB0000B07062F660F110B209709F45CC088853C
:104FC0008F70863009F055C06AE474E0CE010E940B
:104FD000CB9A6C0182E08816910449F06FE474E08A
:104FE000E3E08E16910429F0D0E0C0E006C063E54E
:104FF00074E0CE010E94CB9AEC01C114D104D9F126
:10500000F60180858F708430B1F561857285A801C5
:10501000C7010E9465D8A80168E574E0C7010E9435
:1050200047D8209779F188858F70843059F5698544
:105030007A85A801C7010E9447D8A80168E574E0F5
:10504000C7010E9447D8A114B10429F0A801B501F5
:10505000C7010E9447D8C701DF91CF911F910F91DF
:10506000FF90EF90DF90CF90BF90AF909F908F9088
:105070000895D0E0C0E0A8016FEC7BE1C7010E9479
:1050800057CCC9CFF2E08F16910481F083E08816E7
:10509000910429F060915A0770915B07CACFA8016B
:1050A00069EC7BE1C7010E9439CCC7CFA80166EC4F
:1050B0007BE1F8CFCF92DF92EF92FF920F931F9395
:1050C000CF93DF93CDB7DEB7C154D1090FB6F894B3
:1050D000DEBF0FBECDBF6C01AB0130E020E060E46D
:1050E000CE0101967C010E94C627F70101900020A5
:1050F000E9F731978F010E191F09A801B701C60101
:105100000E9457D8892B11F010E000E0C801CF5B56
:10511000DF4F0FB6F894DEBF0FBECDBFDF91CF914A
:105120001F910F91FF90EF90DF90CF900895EF9235
:10513000FF920F931F93CF937C018C01C0E0C3308B
:10514000E1F0F801428150E070E060E02AE030E0F8
:1051500085E59BE00E94E78864EC7BE185E59BE0C8
:105160000E94C889CF5F0F5F1F4FC43041F7CF91B6
:105170001F910F91FF90EF900895F701458150E046
:1051800070E060E02AE030E085E59BE00E94E7887F
:1051900062EC7BE1E3CFCF93DF931F921F92CDB7F9
:1051A000DEB78091430D9091440D009711F48FE488
:1051B0009DE0BE016F5F7F4F681B790B072E000CCF
:1051C000880B990B0F900F90DF91CF9108954F921C
:1051D0005F926F927F929F92AF92BF92CF92DF9237
:1051E000EF92FF920F931F93CF93DF93CDB7DEB76C
:1051F00060970FB6F894DEBF0FBECDBFFC011986D5
:105200001A861B861C868A85807F8A87A081B18149
:10521000109709F4EEC08C91882309F4EAC000814C
:105220001181D8019C91992309F452C09D3209F44F
:10523000E4C090539A3028F00F5F1F4F1183008312
:10524000EECFC801912CDC016D01C81AD90A2D914D
:10525000022E000C330B205331092A303105A0F304
:105260007F016EE270E0C8010E942CD8FC01DC01D5
:10527000892B91F5CD2809F0C5C01D861E861F8695
:10528000188A88E0FE013996DE01119601900D9290
:105290008A95E1F729813A814B815C816D817E811C
:1052A0008F81988560960FB6F894DEBF0FBECDBF94
:1052B000DF91CF911F910F91FF90EF90DF90CF90F2
:1052C000BF90AF909F907F906F905F904F900895A8
:1052D000912CD12CC12CC4CF5D01AE1ABF0A1196FE
:1052E0008C911197082E000C990BC09711960A9774
:1052F00098F32181022E000C330B205331092A3000
:105300003105F0F52A30310514F029E030E037FF9F
:1053100002C030E020E0032E000C440B550BAAE045
:10532000B0E00E94A0D32B013C018281082E000C2A
:10533000990BC0978A30910588F48A30910514F052
:1053400089E090E097FF02C090E080E0092E000C19
:10535000AA0BBB0B480E591E6A1E7B1EA114B1047A
:1053600009F488CFF3E0AF16B10474F0C8010E94CD
:10537000B0CB2B013C018A85807F87608A8723C060
:1053800020E030E0A901CBCFB8E0CB16D10474F710
:10539000C8010E94D2CB9B01AC01A4E6B0E00E9400
:1053A000A0D3992041F07094609450944094411C93
:1053B000511C611C711C2A85207F26602A87460E9D
:1053C000571E681E791E6CE270E0F70180819181A2
:1053D0000E942CD8009741F4D7011D921C924D8653
:1053E0005E866F86788A4DCF0196F7019183808320
:1053F000F6CF412C512C3201F2CFC80101969924ED
:10540000939421CFC8010E94D2CB2A85207F2A60A5
:105410002A872B013C01D7CFCF92DF92EF92FF92E8
:105420000F931F93CF93DF93EC01A881B98110975D
:1054300081F18C91882369F108811981F8019081AB
:10544000992351F09D3241F090539A3028F00F5F2C
:105450001F4F19830883F0CFC8010E94D2CB6B0184
:105460007C016CE270E0C8010E942CD8009769F4BE
:1054700019821882C701B601DF91CF911F910F9158
:10548000FF90EF90DF90CF900895019699838883E5
:10549000F1CFC12CD12C7601EDCF08950895EF9274
:1054A000FF921F93CF93DF93192F7B01C82FD92F22
:1054B000D7FF03C0D195C195D10961E08C2F0E941F
:1054C000F8A882E0E816F10499F460E08C2F0E94BD
:1054D000CAA86EE778E186E09CE00E94C88986E071
:1054E0009CE0DF91CF911F91FF90EF900C94418849
:1054F000612FEF2851F46095661F6627661F8C2F79
:105500000E94CAA86AE778E1E6CF661F6627661F91
:105510008C2F0E94CAA865E778E1DDCF63E578E1CA
:1055200085E59BE00E94C88960E478E185E59BE021
:105530000E94C88962E378E185E59BE00E94C88902
:105540006AE278E185E59BE00E94C88985E59BE0F9
:105550000E9441886AE178E185E59BE00E94C88964
:105560006EE078E185E59BE00E94C88961E078E122
:1055700085E59BE00E94C8896CEE77E185E59BE0BC
:105580000E94C8896DED77E185E59BE00E94C8899E
:1055900065ED77E185E59BE00E94C8896AEC77E1DB
:1055A00085E59BE00E94C8896DEB77E185E59BE08E
:1055B0000E94C88963EB77E185E59BE00E94C8897A
:1055C0006BEA77E185E59BE00E94C8896FE977E1A6
:1055D00085E59BE00E94C88965E877E185E59BE069
:1055E0000E94C88966E677E185E59BE00E94C8894C
:1055F00061E577E185E59BE00E94C88969E377E191
:1056000085E59BE00E94C8896BE277E185E59BE038
:105610000E94C8896FE177E185E59BE00E94C88917
:1056200067E177E185E59BE00E94C8896CE077E15E
:1056300085E59BE00E94C8896FEF76E185E59BE0F8
:105640000E94C88967EF76E185E59BE00E94C889E2
:105650006CEE76E185E59BE00E94C8896DED76E110
:1056600085E59BE00E94C88964ED76E185E59BE0D5
:105670000E94C88966EC76E185E59BE00E94C889B6
:1056800068EB76E185E59BE00E94C8896CEA76E1EB
:1056900085E59BE00E94C88964EA76E185E59BE0A8
:1056A0000E94C88961E976E185E59BE00E94C8898E
:1056B00067E876E185E59BE00E94C88985E59BE087
:1056C0000C9441880F931F93CF93DF9300D000D0A9
:1056D000CDB7DEB70E948E2A66E070E185E59BE0DB
:1056E0000E94C889CE0101960E941523CE01019621
:1056F0000E9497280FE014E01A8309838091CE0A54
:105700009091CF0AA091D00AB091D10A8B839C834B
:10571000AD83BE83CE0101960E9497281A83098328
:105720001B821C821D821E8280E591E00E9489A45A
:1057300044E050E0BE016D5F7F4F81E090E00E9449
:10574000FA91CE0101960E9497281A8309831B8241
:105750001C821D821E8280E591E00E9489A444E0A3
:1057600050E0BE016D5F7F4F85E090E00E94FA91AE
:10577000CE0101960E9497286CE270E185E59BE0DE
:105780000E94C88988EC90E026960FB6F894DEBF98
:105790000FBECDBFDF91CF911F910F9108958091E2
:1057A00059078823B1F0E091A206F091A306309743
:1057B00031F08681978190935D0780935C076FEE4F
:1057C0007FE085E59BE00E94C88985E59BE00C941D
:1057D00041880895CF92DF92EF92FF920F931F932B
:1057E000CF93DF9300D000D0CDB7DEB7809109070B
:1057F00081119AC08091CD089091CE0802970CF447
:1058000093C08091AC069091AD06009709F48CC0CE
:105810006CE574E00E94CB9A8C01009709F484C077
:105820000E948A9FE82EF12CE114F10409F47CC057
:1058300070E060E0C8010E9472246C01EA94EF28D5
:1058400009F481C061E0C8010E94439BFC0101850D
:105850001285CE0101960E941523CE0101960E9469
:105860008CA460EE7FE085E59BE00E94C889B601CC
:1058700085E59BE00E9471896BEC74E085E59BE017
:105880000E947189B80185E59BE00E94399F6BEC0D
:1058900074E085E59BE00E9471896BEB78E085E51B
:1058A0009BE00E94718985E59BE00E94418862E04F
:1058B00072E084E29CE00E949117D0921A0CC09290
:1058C000190C10931C0C00931B0C8BEB98E0892B8C
:1058D000E9F58AE594E090931E0C80931D0C80916D
:1058E0005C0790915D07009741F070E060E00E94D6
:1058F000722490935B0780935A0780915A07909186
:105900005B07009731F19093200C80931F0C10924D
:10591000220C1092210C81E08093090767EC7FE054
:1059200085E59BE00E94C88926960FB6F894DEBFF5
:105930000FBECDBFDF91CF911F910F91FF90EF90E0
:10594000DF90CF90089502E012E083CF8BEB98E0D8
:10595000C2CF8CEC92E0892B19F48AE594E0D3CF86
:105960008CEC92E0D0CF0F931F93CF9362EC7FE04B
:1059700085E59BE00E94C88909E31BE0C0E0F801CF
:1059800081918F01803130F468E474E085E59BE01B
:105990000E947189C530C9F0F8013197408150E00B
:1059A00070E060E020E130E085E59BE00E94E78860
:1059B00060EC7FE085E59BE00E94C889CF5FC63040
:1059C000F1F6CF911F910F91089540913E0B50E059
:1059D00070E060E020E130E085E59BE00E94E78830
:1059E00085E59BE00E944188E9CFEF92FF920F93FB
:1059F0001F93CF93DF9300D000D01F92CDB7DEB7B7
:105A00007B01CE0107969F938F9301979F938F936E
:105A100001979F938F9301979F938F9301979F93E4
:105A20008F9301979F938F938E010F5F1F4F1F934B
:105A30000F9383E694E09F938F93DB0113968C91F1
:105A400013978F9312968C918F930E94ECD80FB678
:105A5000F894DEBF0FBECDBF0697ECF464E175E1AC
:105A60008FE59BE00E94C889D70112966D917C91C9
:105A70008FE59BE00E94718980E991E027960FB63F
:105A8000F894DEBF0FBECDBFDF91CF911F910F9174
:105A9000FF90EF9008958091310B9091320B892BFC
:105AA000A9F10E941B9C882389F182E70E94069C31
:105AB0008091310B9091320BDC01ED91FC910088CB
:105AC000F189E02D64E070E019958091310B90919F
:105AD000320BDC01ED91FC910280F381E02D46E078
:105AE00050E0B801199586E0F801A9E3BBE0019008
:105AF0000D928A95E1F78091310B9091320BDC0188
:105B0000ED91FC910488F589E02D19950E94B32C44
:105B100066E275E185E59BE00E94C88988EC90E02B
:105B2000ADCF0895EF92FF920F93CF93DF93CDB750
:105B3000DEB7A0970FB6F894DEBF0FBECDBF7C01D5
:105B400000E020E030E340E250E0BE016F5F7F4FB5
:105B50000E94801EBE016F5F7F4F86E09CE00E9426
:105B6000718961E37EE086E09CE00E94C889F701CC
:105B700061816F704AE050E086E09CE00E944588B9
:105B80006AE27EE086E09CE00E94C8894AE050E03C
:105B9000F701628186E09CE00E94458886E09CE0F7
:105BA0000E944188A0960FB6F894DEBF0FBECDBF0D
:105BB000DF91CF910F91FF90EF900895CF93DF93F6
:105BC00000D000D01F921F92CDB7DEB7FC016283D8
:105BD00098E0DE01119601900D929A95E1F72981E6
:105BE0003A814B815C816D817E818F819885289679
:105BF0000FB6F894DEBF0FBECDBFDF91CF910895F1
:105C0000CF93DF9300D000D01F921F92CDB7DEB7A5
:105C1000FC01608398E0DE01119601900D929A9547
:105C2000E1F729813A814B815C816D817E818F8191
:105C3000988528960FB6F894DEBF0FBECDBFDF91D2
:105C4000CF9108952F923F924F925F926F927F92E1
:105C50008F92AF92BF92CF92DF92EF92FF920F930B
:105C60001F93CF93DF93CDB7DEB7C457D1090FB6DB
:105C7000F894DEBF0FBECDBF3C01AE960FAFAE971E
:105C8000AF961FAFAF97E0962FAFE097E1963FAF8B
:105C9000E197E2964FAFE297E3965FAFE397E49622
:105CA0006FAFE497E5967FAFE59723961FAE1EAEE4
:105CB0002397FE01ED5BFF4F82E1DF011D928A9584
:105CC000E9F77296119211928EE0DF011D928A958A
:105CD000E9F767E774E086E09CE00E947189B5010E
:105CE00086E09CE00E94718960EB74E086E09CE0B5
:105CF0000E947189CE0183599F4F0E94922DD4FE3C
:105D00002CC0AE96EFADAE97E83108F067C1F0E079
:105D10008827E257F14D8F4F0C94D6D3F42FA62E3F
:105D2000EB2FEE2FEE2FEB2FA62EEE2FEE2FEE2FDA
:105D3000EE2FEE2FEE2FEE2FA62EA62EEE2FEE2F0D
:105D4000EE2FA62EA62EA62EA62EF42F67EC7BE015
:105D5000CE018B5A9F4F0E9429CC0E94E99A88233A
:105D600009F419C18091CC08811115C1A114B104A5
:105D700009F05FC030E020E043E050E060E4CE0195
:105D800001960E94C627D3011296ED91FC91608185
:105D900071814FE350E0CE0101960E9447D8D5FEB5
:105DA00026C1AE968FADAE97823009F420C1853002
:105DB00009F41DC1AF968FADAF978F709FE0980F1C
:105DC0009F70923018F0883009F011C101E020E096
:105DD00030E244E150E0BE016F5B7F4FCE0183595A
:105DE0009F4F0E94801E482DBE016F5B7F4FCE01EA
:105DF00001960E9479AA6DE97BE086E09CE00E9412
:105E0000C889BE016F5F7F4F86E09CE00E94718968
:105E10006AE97BE086E09CE00E94C889BE016F5B76
:105E20007F4F86E09CE00E94718986E09CE00E94A2
:105E30004188AF968FADAF978F701601270122244E
:105E40003324B0E14B225524882311F0D5FC06C041
:105E5000211431044104510409F409C130E020E067
:105E600043E050E060E4CE0101960E94C627D301D2
:105E70001296ED91FC91608171814FE350E0CE016B
:105E800001960E9447D8A114B10469F068E574E056
:105E9000CE0101960E9421D84FE350E0B501CE011A
:105EA00001960E9447D868E574E0CE0101960E94F1
:105EB00021D84FE350E06FE57BE021143104410429
:105EC000510459F4E0968FADE0974FE350E06EE651
:105ED0007BE0873011F065E57BE0CE0101960E9402
:105EE00039CCAF968FADAF978F708450823008F069
:105EF000A5C067E1CE0183599F4F0E94002EA69650
:105F00002FAFA697A7963FAFA797A8964FAFA89792
:105F1000A9965FAFA997AA966FAFAA97AB967FAFE6
:105F2000AB97AC968FAFAC97AD969FAFAD9700E0B7
:105F300020E030E344E150E0BE016F5B7F4FCE01D3
:105F400083599F4F0E94801E65E47BE086E09CE0C1
:105F50000E94C889BE016F5F7F4F86E09CE00E946F
:105F6000718962E47BE086E09CE00E94C889BE0102
:105F70006F5B7F4F86E09CE00E94718986E09CE029
:105F80000E9441880E94E99A882329F08091CC08D8
:105F9000882309F45DC0B701A601C3010E948319DB
:105FA00090E080E0CC58DF4F0FB6F894DEBF0FBE14
:105FB000CDBFDF91CF911F910F91FF90EF90DF90B8
:105FC000CF90BF90AF908F907F906F905F904F90E9
:105FD0003F902F90089561ED7BE0BACE63EA7BE0BD
:105FE00086E09CE00E94C889E894D4F8B6CED4FE3E
:105FF00020CF66968FAD6697882309F41ACF482D77
:10600000BE016B5A7F4FCE0101960E9479AA64E9C6
:106010007BE086E09CE00E94C889BE016F5F7F4FF5
:1060200086E09CE00E94718961E97BE086E09CE06B
:106030000E94C889BE016B5A7F4FF3CE20E030E347
:1060400023282428252811F420E030E200E072CF34
:10605000482DBE016F5B7F4FCE0101960E9479AA49
:1060600040E050E260E070E0C3010E945A19D4FEA3
:1060700097C0A114B10409F028C1AE96EFADAE9758
:10608000E150E63120F5F0E08827E65BFF4C8F4FCA
:106090000C94D6D35D3167306730673067305D313F
:1060A000673067306730673067306730673062313C
:1060B0005A31673067306730603051315431573171
:1060C0006BE77CE0CE018B5A9F4F0E9429CC30E0D9
:1060D00020E043E050E060E4CE0101960E94C62734
:1060E000D3011296ED91FC91608171814FE350E0F4
:1060F000CE0101960E9447D8A114B10469F068E569
:1061000074E0CE0101960E9421D84FE350E0B50122
:10611000CE0101960E9447D868E574E0CE01019651
:106120000E9421D84FE350E060E57BE0CE0101966C
:106130000E9439CC6CE37BE086E09CE00E94C88939
:10614000BE016F5F7F4F86E09CE00E94718969E32A
:106150007BE086E09CE00E94C889BE016B5A7F4FBD
:1061600086E09CE00E94718986E09CE00E94418864
:106170000E94E99A882309F40ECF8091CC088111FE
:106180000ACF482DBE016B5A7F4FCE0101960E9467
:1061900079AA40E050E160E070E0C3010E945A1922
:1061A000D6FE7CC040E051E060E070E0C3010E9498
:1061B000AC19672B682B692B09F495C06BE27CE066
:1061C000CE018B5A9F4F0E9429CC30E020E043E063
:1061D00050E060E4CE0101960E94C627D3011296DA
:1061E000ED91FC91608171814FE350E0CE01019609
:1061F0000E9447D8A114B10469F068E574E0CE01AB
:1062000001960E9421D84FE350E0B501CE010196DE
:106210000E9447D868E574E0CE0101960E9421D81B
:106220004FE350E068E77BE0CE0101960E9439CC55
:1062300063E37BE086E09CE00E94C889BE016F5F5B
:106240007F4F86E09CE00E94718960E37BE086E0FE
:106250009CE00E94C889BE016B5A7F4F86E09CE09B
:106260000E94718986E09CE00E9441880E94E99A20
:10627000882309F490CE8091CC0881118CCE482DD2
:10628000BE016B5A7F4FCE0101960E9479AA40E071
:1062900050E460E070E0C3010E945A1981E090E090
:1062A00081CE65E87CE00ECF6FE87CE00BCF69E93A
:1062B0007CE008CF63E57CE005CFF3018285853083
:1062C00009F005CF69E47CE0FDCE00E020E030E39A
:1062D00040E150E0BE016B5A7F4FCE0183599F4F82
:1062E0000E94801EF4CE40E056E060E070E0C30102
:1062F0000E94AC19611576408105910519F46FE390
:106300007CE05ECF61E27CE05BCFDC011196EC913A
:106310001197EF70E150EB3008F039C0F0E08827BA
:10632000EB56FE4C8F4F0C94D6D3B831B831C731F1
:10633000A031A031A931C031C031C031A031A0316C
:1063400014966D917D918D919C9117970E941CD20E
:10635000089514966D917D918D919C91179724E6E7
:1063600030E040E050E00E9481D3CA01B901EECF95
:1063700014966C9170E090E080E00E941AD208952B
:1063800014966D917D918D919C911797089560E081
:1063900070E0CB010895DC011196EC911197EF703C
:1063A000E150EB3008F037C0F0E08827E552FE4CB2
:1063B0008F4F0C94D6D3ED31ED310B32E631E6310F
:1063C000FC31F331F331F331E631E63114966D915E
:1063D0007D918D919C911797089514966C9170E022
:1063E00090E080E0089514966D917D918D919C913F
:1063F00017970E94D3D4089514966D917D918D9135
:106400009C91179724E630E040E050E00E9481D351
:10641000CA01B901089560E070E0CB010895CF9200
:10642000DF92EF92FF920F931F93CF93DF93CDB73D
:10643000DEB762970FB6F894DEBF0FBECDBF6C011A
:106440000B871C872D873E874F87588B698B7A8BEC
:106450006EE57AE1C7010E9420CCEEE0F0E0892BE6
:10646000F1F068E57AE1C7010E9420CCE0E1F0E0BC
:10647000892BA9F062E57AE1C7010E9420CCEFE008
:10648000F0E0892B61F01D856EE47AE1C7010E947E
:1064900020CCE12FF0E0892B11F4EDE0F0E09B85BA
:1064A000992341F0309731F4EF2809F45CC08FEF65
:1064B0009FEFCAC0E131F10508F037C08827EC59D9
:1064C000FD4C8F4F0C94D6D35732B3327532953280
:1064D00095329532953265331C349532953295322A
:1064E0009532953226345F343434CE010B960E94B7
:1064F000CB3120EF260F2931D0F6D6011496ED913D
:10650000FC91159723A39B01AC0133274427552702
:106510001296ED91FC910280F381E02D60817181F2
:1065200004E814E0C6010E944A21D6011496ED91B8
:10653000FC911597118A1496ED91FC91159781E0C5
:1065400081871496ED91FC9115978DE482871496BE
:10655000ED91FC9115978FE5838714966D917C9151
:1065600045E250E04CC0F601048115814FEF5FEF2A
:10657000BA0180E00E948824D80198966D937D939B
:106580008D939C939B97D601ED91FC910484F585A6
:10659000E02D64E0C6011995EB85E150E63128F65F
:1065A000F0E0D60114962D913C9115978827E4527E
:1065B000FD4C8F4F0C94D6D3F23203339532953283
:1065C0000333F232953295329532953295329532C7
:1065D000953233334B33953295329532953247337A
:1065E00043334933F90185A1858F1496ED91FC91D0
:1065F000858D8160858F4DE050E06CE172E0C601D1
:106600000E940B271FC0F90185A1858F1496ED917B
:10661000FC91858D8E7F858F4DE050E06FE072E0BC
:10662000C6010E940B27D6011296ED91FC910280C3
:10663000F381E02D49E854E06EE874E080819181B7
:106640000E9497AA81E090E062960FB6F894DEBFB0
:106650000FBECDBFDF91CF911F910F91FF90EF90B3
:10666000DF90CF900895F901178AD6011496ED9125
:10667000FC91159785A1858F1496ED91FC91858DE0
:106680008160858F52CF81E0F901878BEECF82E068
:10669000FBCF84E0F9CF83E0F901878B1496ED916D
:1066A000FC91159785A1858F1496ED91FC91159716
:1066B000858D8160858F1496ED91FC91818D83305D
:1066C00009F033CF82E0818F30CF1982F601048147
:1066D00015819031C1F190F4923009F440C09E30A0
:1066E000B9F0CE010B960E94CB3161157105810581
:1066F000910509F058C0F80117A243C0913141F14A
:10670000923179F782E0F801818F68E07AE106C082
:1067100083E0D80159968C9360EE79E1CE01019621
:106720000E9429CCD6011296ED91FC910280F38152
:10673000E02D42E954E0BE016F5F7F4F808191817F
:106740000E9497AAF2CEF801118E64EF79E1E6CFAC
:1067500081E0D80159968C936EEF79E1DFCFD801B3
:1067600097961C92048115814FEF5FEFBA0180E08C
:106770000E948824D80198966D937D938D939C9365
:106780009B97D6011496ED91FC91159785A1858F65
:106790001496ED91FC91858D8E7F858F4DE050E0B4
:1067A0006FE072E02CCFD80197961C92615071096E
:1067B00081099109660F771F881F991F2EEF30E01E
:1067C00040E050E00E9481D3DA01C9010196A11D89
:1067D000B11D813071F0A8F2823029F1833009F0C7
:1067E000A1CFD6011496ED91FC91118E64EF79E161
:1067F00008C0D6011496ED91FC9182E0818F68E08B
:106800007AE1CE0101960E9429CCD6011496ED9131
:10681000FC91159785A1858F1496ED91FC91858D3E
:106820008160858F7FCFD6011496ED91FC9181E038
:10683000818F6EEF79E1E5CFCE010B960E94CB31CF
:10684000D6011496ED91FC91678B6FCED60114960C
:10685000ED91FC91913029F0923009F066CE148EC2
:1068600064CE80E5848F61CEF6010481158191307C
:1068700049F09230B1F0CE010B960E94CB31F80175
:10688000638F53CE83E0D8015B968C930280F381B3
:10689000E02D0280F381E02D47E954E06EE974E0D9
:1068A0004DCFF801138ED6011296ED91FC91028026
:1068B000F381E02D47E954E06EE874E03FCFD60164
:1068C0001496ED91FC91913031F0923009F02DCE7B
:1068D000858D877FD6CE858D8860D3CE8F929F920F
:1068E000AF92BF92CF92DF92EF920F931F93CF930D
:1068F000DF9300D000D01F921F92CDB7DEB709837F
:106900001A832B833C834D835E836F837887DC01FE
:1069100012962D913C9121153105A1F490E080E073
:1069200028960FB6F894DEBF0FBECDBFDF91CF9192
:106930001F910F91EF90DF90CF90BF90AF909F90FD
:106940008F9008958C01C9010E948A9FC82ED12C76
:10695000B6E0CB16D10464F40E947D9FBC01F8011F
:10696000828193810E945F9FFFEFCF1ADF0AF0CFF1
:1069700065E0D80112968D919C910E94439B6C0119
:10698000892B61F28981803148F6CE0101960E94FF
:10699000CB31161617061806190644F4F601808541
:1069A000982F9D7039F18F70873021F1D60118969C
:1069B0008C9118978F7018968C9366E977E086E033
:1069C0009CE00E94C889D8011296ED91FC916081EB
:1069D000718186E09CE00E9471896CE877E086E036
:1069E0009CE00E94C88986E09CE00E94418881E08A
:1069F00090E096CF0E94ABA94B015C01CE010196BD
:106A00000E94CB31860E971EA81EB91EF601818604
:106A10009286A386B48682E0E11087E09981929500
:106A2000907F892BD60118968C936FE777E086E0EC
:106A30009CE00E94C889D8011296ED91FC9160817A
:106A4000718186E09CE00E94718969E777E086E0C9
:106A50009CE00E94C889CE0101960E94CB31AB0117
:106A6000BC012AE030E086E09CE00E94E78865E710
:106A700077E0B5CFAF92BF92CF92EF92FF920F9394
:106A80001F93CF93DF93CDB7DEB7C856D1090FB6AA
:106A9000F894DEBF0FBECDBFA2960FAFA297A3960C
:106AA0001FAFA397A4962FAFA497A5963FAFA59726
:106AB000A6964FAFA697A7965FAFA797A8966FAF7A
:106AC000A897A9967FAFA997970148E0FE01EF59D3
:106AD000FF4FDE01A75ABF4F01900D924A95E1F793
:106AE000A296EFADA297E150ED3008F0F9C0EC2C82
:106AF0005C01F0E08827E058FA4C8F4F0C94D6D315
:106B0000F935033663366E3659368D35F0357036C5
:106B100070360C361E36453631362130310531F4AB
:106B2000C5010E944619009709F449C067E0CE01EB
:106B3000875A9F4F0E94002E61E677E086E09CE036
:106B40000E94C8894AE050E06A966FAD6A9786E075
:106B50009CE00E94458866E577E086E09CE00E9424
:106B6000C889CE01875A9F4F0E94CB31AB01BC012F
:106B70002AE030E086E09CE00E94E78886E09CE026
:106B80000E9441886A960FAD6A976B961FAD6B970E
:106B90006C962FAD6C976D963FAD6D976E964FAD21
:106BA0006E976F965FAD6F97A0966FADA097A19609
:106BB0007FADA197C5010E946E3481E090E0C85975
:106BC000DF4F0FB6F894DEBF0FBECDBFDF91CF9180
:106BD0001F910F91FF90EF90CF90BF90AF900895CD
:106BE000232B29F4C5010E944619009741F366E062
:106BF0009ECF2130310529F4C5010E944619009726
:106C0000F1F262E094CF232B29F4C5010E944619CA
:106C10000097A9F261E08BCF40E051E060E070E0C6
:106C2000C5010E94AC19672B682B692B29F4C5019B
:106C30000E944619009719F26BE079CF40E051E0CD
:106C400060E070E0C5010E94AC19672B682B692BCE
:106C500031F0C5010E944619009709F4B0CF6AE0EF
:106C600066CF40E056E060E070E0C5010E94AC19DC
:106C7000611576408105910531F4C5010E944619E0
:106C8000009709F49CCF6CE052CF40E056E060E002
:106C900070E0C5010E94AC1961157640810591052F
:106CA00031F0C5010E944619009709F488CF6DE0C4
:106CB0003ECF232B31F4C5010E944619009709F4F9
:106CC0007ECF63E034CF2130310531F4C5010E941D
:106CD0004619009709F473CF65E029CF64E027CF08
:106CE00090E080E06CCFCF93DF93EC0161157105EC
:106CF00039F48F8181708F8381E0DF91CF91089586
:106D00008981982F9F7029F180E09430B0F79B0122
:106D1000770F440B550B2959310941095109A4E654
:106D2000B0E00E94A0D32BE531E040E050E00E94AB
:106D300081D337FF02C030E020E02536310514F062
:106D400024E630E02F5F220F8F818170282B2F8364
:106D5000D3CF807F82608983DACF2F923F924F9288
:106D60005F926F927F928F929F92AF92BF92CF92DB
:106D7000DF92EF92FF920F931F93CF93DF93CDB7E4
:106D8000DEB766970FB6F894DEBF0FBECDBF6C01BD
:106D900009871A872B873C874D875E876F87788B9B
:106DA00082E1E816F10480F5F701E85EFC4F90817E
:106DB000998BCE0109960E94C71497FD04C0BC01AF
:106DC000C6010E9473368B85D60112968C9312975A
:106DD00089858C931196EC911197EF70EC3008F047
:106DE0006CC0F0E08827E850F94C8F4F0C94D6D354
:106DF0005A3821372137A038063728396D38A93855
:106E0000A938A9386D386D38198AD3CF10E09A8522
:106E10009F709D3008F019C4E92FF0E08827EC5EE0
:106E2000F84C8F4F0C94D6D35D375F397F395F397B
:106E30002A392A395F395F39253B253B5F395F396C
:106E400033389A859F709D3008F01DC1E92FF0E01E
:106E50008827E25DF84C8F4F0C94D6D35D37073806
:106E6000FB3753373E373B37DE370B384338433831
:106E7000C837C83733388889F60187838F85D601AC
:106E800016968C9316978E8515968C9315978D85EF
:106E900014968C93149711968C911197807F892B5F
:106EA00011968C930AC08F859889F6018683878115
:106EB00090FB80F987838E858583F989FF2309F408
:106EC00064C0D60111968C918F702F2F30E08217FD
:106ED000130609F45AC06BE87DE086E09CE00E944E
:106EE000C889F60161816F704AE050E086E09CE05D
:106EF0000E94458868E87DE086E09CE00E94C889A1
:106F00004AE050E0698986E09CE00E94458866E896
:106F10007DE086E09CE00E94C889D6010C91198230
:106F20001A821B821C821D821E821F8218868989FA
:106F30008F709A81907F892B8A830983EE24EA944B
:106F4000FE2C11961C91119712962C911297139664
:106F50003C91139714964C91149715965C91159744
:106F600016966C91169717967C91CE0101960E9409
:106F7000AD36F60120833183428353836483758366
:106F800086839783C6010E94922D88E0F60170C126
:106F90008D859E85AF85B8898F3F9105A105B10587
:106FA00029F024F08FEF90E0A0E0B0E0B7FF03C03D
:106FB00080E090E0DC01F60184837FCF6D857E85E3
:106FC0008F85988924E630E040E050E00E9481D32C
:106FD0002F3F31054105510529F024F02FEF30E016
:106FE00040E050E057FF03C020E030E0A901D601A7
:106FF00014962C9362CF8F859889F60186838781BA
:1070000090FB80F987838E8585838D85D5CF8D858F
:1070100014968C9352CF8D849E84AF84B88820E0E0
:1070200030E0A901C501B4010E9415D287FD17C047
:1070300020E030E04FE753E4C501B4010E9409D5D8
:10704000181634F4812C912C4FE7A42E43E4B42E6F
:10705000C501B4010E94DAD4F60164832ECF812CDD
:10706000912C5401F5CFD60111968C911197807F08
:107070008C6011968C9311978D859E8515969C93A7
:107080008E9314971ACF68E17EE086E09CE00E9420
:10709000C8896A856F704AE050E086E09CE00E94F3
:1070A000458865E17EE086E09CE00E94C889F601A3
:1070B0006181C2C09A859F7011968C911197807FD3
:1070C000892B11968C938D859E85AF85B889F601A5
:1070D00084839583A683B783F0CE9A859F7093307F
:1070E00089F09C3009F4BFCF4D855E856F85788926
:1070F000F60144835583668377838181807F892B62
:107100008183DBCEC6010E94529BD60114968C93DC
:1071100014978F85988916968C93169717968C914D
:10712000179790FB80F917968C9317978E85159675
:107130008C93159711968C911197807F8260B0CEB9
:10714000CE0109960E94529BD60114968C931497F7
:10715000F1CF9A859F709D3008F057C0E92FF0E07D
:107160008827EA54F74C8F4F0C94D6D35D37D0382C
:10717000FD388238FD38FD38C338EF38EF38EF3846
:10718000DE38EA3833388D859E85AF85B889F601BB
:1071900084839583A683B7838181807F8660B0CF07
:1071A0006D8570E090E080E00E941AD2D6011496BE
:1071B0006D937D938D939C9317977FCE6D857E8580
:1071C0008F8598890E941CD2F6016483758386831B
:1071D000978373CE6D857E858F859889E5CFF6017F
:1071E0008181807F982B91838D859E85AF85B8891D
:1071F00084839583A683B78360CE11968C91119773
:10720000807F982B11969C935ECF63E07EE086E0B2
:107210009CE00E94C8896A856F704AE050E086E071
:107220009CE00E94458860E07EE086E09CE00E9451
:10723000C889D60111966C916F704AE050E086E0E3
:107240009CE00E94458886E09CE00E94418835CE03
:1072500011E0DDCD4D855E856F857889F60144832B
:107260005583668377838181807F982B918388E023
:10727000DE01119601900D928A95E1F729813A81FC
:107280004B815C816D817E818F81988566960FB67A
:10729000F894DEBF0FBECDBFDF91CF911F910F914C
:1072A000FF90EF90DF90CF90BF90AF909F908F9026
:1072B0007F906F905F904F903F902F900895963001
:1072C00009F4C1C048F46D85913071F06FEF70E042
:1072D000933051F060E008C0973009F4C0C09A5074
:1072E0006D857E859230B0F784E68F8788898E7FA2
:1072F000888B1E868A85807F82608A876D871123AE
:1073000009F48DC02E8530E0AFEFB0E00E94B3D31A
:1073100024E630E040E050E00E9481D349015A0168
:10732000FFEF8F169104A104B10429F024F0812C01
:10733000912C54018A948D858A8B082F10E028881F
:107340002694A22DA150BB0B1D01BFEF2B163B06AF
:1073500009F0A5C0E0E88E1691040CF087C08FE715
:1073600090E088199909809FD001819FB00D909F6E
:10737000B00D11242FEF30E00E94EDD321E83EE75D
:1073800040E050E00E9481D3D60117962C93ABE9E0
:10739000B0E0A50194010E94A0D32FE7422E512C0A
:1073A000612C712CA30192010E9481D32C593F4F73
:1073B0004F4F5F4F7901AEEFB1E0A50194010E94FC
:1073C000A0D3A30192010E9481D3D8010E94A0D32F
:1073D0002FEF30E040E050E00E9481D389012F3F41
:1073E000310519F014F00FEF10E063EF7DE086E057
:1073F0009CE00E94C889B70186E09CE00E94399F0A
:1074000065EE7DE086E09CE00E94C889B80186E0D8
:107410009CE00E94399F86E09CE00E94418863EBDB
:107420007DE086E09CE00E94C88986E09CE00E94A6
:1074300041886CEA7DE086E09CE00E94C889C60134
:107440000E94922D3ACD6D857E858F85988924E6A0
:1074500030E040E050E00E9481D3B90145CF6D8516
:107460007E858F8598890E94D3D43ECFA501940153
:107470002058310941095109ABE9B0E00E94A0D37D
:107480002FE730E040E050E00E9481D32C593F4F7D
:107490004F4F5F4F7901D60117961C92A6CF9101ED
:1074A000AAEBBFEF0E94E5D324E630E040E050E0D5
:1074B0000E9481D329013A01B4E64B0E511C611C94
:1074C000711C26E430E0D1010E94EDD324E630E0C7
:1074D00040E050E00E9481D3DA01C9014E96A11D1F
:1074E000B11D8B8B9C8BAD8BBE8B90E88916910464
:1074F0000CF090C08FE790E088199909809FD00127
:10750000819FB00D909FB00D11242B893C894D892E
:107510005E890E94ABD39B01AC01AFEFB0E00E944B
:10752000A0D324E63AE640E050E00E9481D3D601A1
:1075300017962C93A5019401240D351D461D571D4A
:10754000AEEFB1E00E94A0D323EE30E040E050E087
:107550000E9481D379018A011901AFEFB0E0A50142
:1075600094010E94A0D32FE730E040E050E00E9459
:1075700081D35901EA89AE2FB0E0A80197010E949A
:10758000A0D32FEF30E040E050E00E9481D389018A
:107590002F3F310519F014F00FEF10E06FED7DE093
:1075A00086E09CE00E94C8892AE030E0B301A20195
:1075B00086E09CE00E94E78869ED7DE086E09CE043
:1075C0000E94C8892AE030E04B895C896D897E89F8
:1075D00086E09CE00E94E78861ED7DE086E09CE02B
:1075E0000E94C889B50186E09CE00E94399F69EC41
:1075F0007DE086E09CE00E94C889B80186E09CE0BE
:107600000E94399F60EC7DE086E09CE00E94C88982
:10761000B101FDCEA501940120583109410951095C
:10762000ABE9B0E00E94A0D32FE730E040E050E0AB
:107630000E9481D32C593F4F4F4F5F4F5901D601C4
:1076400017961C92312C212CA9CF6AE97DE086E0A7
:107650009CE00E94C8896A856F704AE050E086E02D
:107660009CE00E94458867E97DE01DCDFC01918189
:10767000892F8F7021F0823029F080E00895907F6B
:10768000926091839B0177FF02C030E020E02E36AC
:1076900081E0380714F02DE631E02683878130FB46
:1076A00080F9878381E008950F931F93CF93DF9331
:1076B000EC01088119816FE270E0C8010E9474D862
:1076C000009749F0FC011192CF01DF91CF911F91FA
:1076D0000F910C942A1BC8010E942A1B009711F0DD
:1076E00019821882DF91CF911F910F910895DC01CB
:1076F0001296ED91FC91309729F090859F7081E072
:10770000953009F080E00895CF92DF92FF920F93B9
:107710001F93CF93DF938C01EB016A01CB010E9491
:10772000773BF82E882309F483C0D6FE0EC0D8011B
:107730008C918B3009F450C008F041C040E051E01A
:1077400060E070E08A3009F450C0D4FE09C0F8014E
:10775000608186EF860F843018F0CE010E94D01928
:10776000D5FE66C0D80114964D915D916D917C91C6
:10777000179711968C918F70873030F08930C8F14F
:107780008A50823008F45DC0CE010E94E814EE8178
:10779000FF81309709F44CC080858F709EEF980F61
:1077A000923010F0811144C0D80111968C91982F1D
:1077B0009295907F80858F70892B808739C08C301F
:1077C00081F040E056E060E070E08D3009F0BDCF20
:1077D000CE010E948319B9CF40E051E060E070E033
:1077E000F7CF40E056E060E070E0CE010E945A1909
:1077F000ACCFEE81FF813097D9F080858F709EEFFE
:10780000980F923010F0811113C04187528763871F
:107810007487EE81FF818085807F83608087EE8121
:10782000FF818085982F907F8F708067903629F236
:107830008F2DDF91CF911F910F91FF90DF90CF900F
:107840000895CE010E94E814F3CF8F929F92AF92D9
:10785000BF92CF92DF92FF920F931F93CF93DF934C
:10786000EC018A819B810E948A9F082F10E00430DE
:10787000110554F40E947D9FBC018A819B810E9466
:107880005F9F0F5F1F4FF3CFEA81FB810681178156
:107890000115110531F0D80112968D919C919D83AF
:1078A0008C83EC81FD81309721F0828193819F83CD
:1078B0008E83EE81FF81309749F00280F381E02DC5
:1078C000309721F08281938199878887011511056E
:1078D00041F0F80180858F70843059F128F48230AE
:1078E00071F0FF24FA940CC0853001F18630C9F79D
:1078F00061EA74E0C8010E94CB9A8C01E7CFF18461
:10790000FA86CE010E94773B811138C010E000E07A
:107910001C870B87DF91CF911F910F91FF90DF9014
:10792000CF90BF90AF909F908F9008950681178160
:10793000CDCFC184D284C114D10499F2F6018081E3
:10794000882379F297EB892E9CE0992EB12CA12CFB
:10795000FA2CC4010E9430CCAC01B401C6010E94D3
:1079600049CC892BB9F1FFEFAF1ABF0A89E0880E25
:10797000911CA7E1AA16B10459F7B3CFCE010E941A
:10798000419F8C010097B1F0FC0182819381892B8A
:1079900039F08F2D0E9451A08C01892B09F4B6CFAC
:1079A000D801ED91FC910684F785E02DBE01C80158
:1079B0001995AECF8F2D0E9451A08C01892B09F40F
:1079C000A5CFEA85F0E0EE0FFF1FEB5BF34F1183CD
:1079D0000083E6CFC6010E944E8F8A2D90E0B0E072
:1079E000A0E0F80181879287A387B4878085807F94
:1079F0008260808785CFAF92BF92CF92DF92EF9265
:107A0000FF920F931F93CF93DF93CDB7DEB76597A8
:107A10000FB6F894DEBF0FBECDBF8C017B015A01BB
:107A2000FC0151834083148613861586168E158EAD
:107A3000672B09F479C0452B09F476C06FE270E03A
:107A4000C7010E942CD86C01892B09F465C0F7018D
:107A5000DE01119690E080E0BD012191222341F0EA
:107A60002F3231F08431910519F02D930196F5CF25
:107A7000860F971FFC011082C5010E94CB9AF80166
:107A800093838283FFEFCF1ADF0AD601F8013D9678
:107A900030E020E0CF01BD014D91442349F04F3249
:107AA00039F02F30310521F041932F5F3F4FF3CF55
:107AB000F801E20FF31F1586FB0140814F3219F5E3
:107AC0002F5F3F4FC601820F931F0E942A1BF801B0
:107AD000968F858FC8010E94773B882319F0C801D3
:107AE0000E94253C65960FB6F894DEBF0FBECDBF51
:107AF000DF91CF911F910F91FF90EF90DF90CF908A
:107B0000BF90AF9008950E942A1BF801968F858F31
:107B1000892B01F31586DECFB701C5010E94CB9AF0
:107B2000F80193838283D6CFF80113821282D2CFD9
:107B3000CF92DF92EF92FF920F931F93CF93DF9339
:107B4000EC016A017B0188859985892BA9F48A81DA
:107B50009B810E948A9F082F10E00530110564F474
:107B60000E947D9F99878887BC018A819B810E94A2
:107B70005F9F0F5F1F4FF1CFE885F985309781F048
:107B80008085982F9F7051F4807F82608087E88580
:107B9000F985C186D286E386F48602C09230B9F3B5
:107BA000DF91CF911F910F91FF90EF90DF90CF90D9
:107BB0000895FC0180859185009799F0FC0120854E
:107BC0002F70223029F4618572858385948508950C
:107BD000253039F460E00E94439B009711F0FC01CE
:107BE000F2CF60E070E0CB01089563E0FC01828198
:107BF00093810E94439B009719F0FC0181850895B1
:107C00008FEF0895FF920F931F93CF93DF93CDB71C
:107C1000DEB764970FB6F894DEBF0FBECDBF8C0100
:107C2000F62EDC0116966C91FF2011F081E068279A
:107C3000F80184810E94CAA8F80187819085A185F6
:107C4000B285883E9340A105B10508F45FC06BEC96
:107C50007AE186E09CE00E94C88966EC7AE186E0E1
:107C60009CE00E94C889D80114966D917C9186E0B1
:107C70009CE00E94399F61EC7AE186E09CE00E94E2
:107C8000C8896F2D70E086E09CE00E94399F86E0F5
:107C90009CE00E9441888FE290E09C878B87FE01E8
:107CA0003D9688E0DF011D928A95E9F76AEB7AE15B
:107CB000CE010B960E9415CCF801828193810E941F
:107CC000F53DFF2079F162EB7AE1853151F06BEA05
:107CD0007AE1863131F06FE97AE18F3011F467EAA9
:107CE0007AE1CE0101960E9429CCD8011296ED913D
:107CF000FC910280F381E02DAE01455F5F4FBE0134
:107D00006F5F7F4F808191810E9497AA64960FB622
:107D1000F894DEBF0FBECDBFDF91CF911F910F91C1
:107D2000FF9008956BE97AE18230D9F266E97AE151
:107D3000D8CFAF92BF92CF92EF92FF920F931F9343
:107D4000CF93DF9300D000D01F921F92CDB7DEB744
:107D50005C0109831A832B833C834D835E836F838D
:107D6000788760E17BE186E09CE00E94C889CE01D3
:107D700001960E94922DE114F10439F069E07BE153
:107D8000C7010E9420CC009749F1F50102811381BF
:107D90000115110509F18981811161C08B81813043
:107DA00009F465C068F1823049F1082F10E066EEF1
:107DB0007AE186E09CE00E94C88966ED7AE186E07F
:107DC0009CE00E94C889B80186E09CE00E94399F2F
:107DD00086E09CE00E94418890E080E028960FB603
:107DE000F894DEBF0FBECDBFDF91CF911F910F91F1
:107DF000FF90EF90CF90BF90AF900895CC20D1F03E
:107E0000CE0101960E94529B892B09F44FC0C801F4
:107E10000E94D93D672B682B692BF1F44FEF5FEF80
:107E2000BA0180E00E948824AB01BC01C8010E9415
:107E3000983D12C0C8010E94F53D8E3019F048F4FB
:107E4000813051F4CE0101960E94529B892B21F082
:107E5000DECF83518430B0F381E090E0BFCF80313A
:107E600000F58E30A0F6813091F28230F9F06EEF9D
:107E70007AE186E09CE00E94C88961EF7AE186E0C1
:107E80009CE00E94C8894AE050E0698186E09CE05D
:107E90000E94458886E09CE00E94418801E010E055
:107EA00086CF8351843008F4B2CFE1CF40E050E078
:107EB000BA01C8010E94983D60E0C5010E94023EDF
:107EC000CBCF0F931F93CF93DF93DC0112962D91AD
:107ED0003C91232B81F1EC0164E079E186E09CE0A8
:107EE0000E94C8894AE050E06E8186E09CE00E94D2
:107EF000458886E09CE00E9441888C819D81892B89
:107F000061F40A811B818CE290E00E94E7C9BC0108
:107F1000C8010E94A0209D838C83EC81FD81309755
:107F200069F462EF78E18FE59BE00E94C8898FE5F4
:107F30009BE00E94418890E080E05FC085E2DF0125
:107F40001D928A95E9F7EC81FD8182E28283EC81C2
:107F5000FD8116A2EC81FD8115A2EC81FD8117A2A5
:107F60000C811D814FEF5FEFBA0180E00E948824F1
:107F7000F80160A771A782A793A78E81811116C00F
:107F800062E00E94F8A869EB78E185E59BE00E9439
:107F9000C88985E59BE00E94418889E69BE00E94B4
:107FA000958010922A0281E080935807EF81F8852E
:107FB000A089B18982E08C93A485B5851C92A685A1
:107FC000B7858FEC8C93108EA489B58986E08C934D
:107FD000A289B3898C9188698C930288F389E02DFA
:107FE00080818F7D8083E881F9810484F585E02D8F
:107FF00062E0CE01199581E090E0DF91CF911F9171
:108000000F910895CF92DF92EF92FF920F931F93FB
:10801000CF93DF936115710509F454C06A017B01A8
:10802000EC01CB010E94773B082F882351F1D70147
:1080300016968D919C910097C9F1FC011085212F16
:108040002F703EEF320F323010F0211124C0129504
:108050001F70D4FE04C0C7010E94F53D8883112320
:1080600039F18981807F182B1983D7011696ED91FC
:10807000FC9181859285A385B4858C839D83AE8395
:10808000BF83802FDF91CF911F910F91FF90EF90D1
:10809000DF90CF900895253049F460E00E94439B23
:1080A000009721F0DC0118961C91D1CF10E0D1CFC0
:1080B000D7011696ED91FC9180858F70823021F06A
:1080C000833079F000E0DDCF41855285638574858A
:1080D0008981807F8A6089834C835D836E837F83FF
:1080E000D0CF41855285638574858981807F876083
:1080F00089834C835D836E837F83C3CF6F927F922E
:108100008F92AF92BF92CF92DF92EF92FF920F9336
:108110001F93CF93DF9300D000D01F921F92CDB753
:10812000DEB73C016A017B01590140FF03C0E894BE
:10813000C0F8D3F8D3FC0DC00E94CB286639710576
:108140008105910530F08091CD089091CE0805977A
:1081500029F5B701A6014427507766277727C30181
:108160000E9483196FE17BE086E09CE00E94C88951
:108170008FEF9FEF28960FB6F894DEBF0FBECDBFEE
:10818000DF91CF911F910F91FF90EF90DF90CF90F3
:10819000BF90AF908F907F906F90089519821A8250
:1081A0001B821C821D821E821F8218868A81807F0C
:1081B0008A8340E050E3B301CE0101960E94024061
:1081C00040E050E760E070E0C3010E94AC19C62AAD
:1081D000D72AE82AF92A8824839409811A812B81D5
:1081E0003C814D815E816F817885C3010E94222E82
:1081F000C1CF0F931F93CF93DF9300D000D01F9276
:108200001F92CDB7DEB719821A821B821C821D8293
:108210001E821F8218862A81207F2A83FC01028108
:108220001381C8010E94F53D813041F020F0823079
:1082300011F0853081F490E080E002C081E090E0B0
:1082400028960FB6F894DEBF0FBECDBFDF91CF9159
:108250001F910F91089540E050E2B801CE010196C0
:108260000E940240CE0101960E94529BE9CF0F93DB
:108270001F93CF93DF93DC011B960D911C91011589
:10828000110519F1EC010E94419F0097F1F0D8010E
:10829000ED91FC91DC0112968D919C91C817D90744
:1082A00059F40684F785E02D70E060E0C801DF91A5
:1082B000CF911F910F9119940280F381E02DC80195
:1082C000DF91CF911F910F911994DF91CF911F9161
:1082D0000F9108958F929F92AF92BF92CF92DF92AB
:1082E000EF92FF920F931F93CF93DF93CDB7DEB73B
:1082F000CF55D1090FB6F894DEBF0FBECDBF8C01AC
:108300006B016115710519F04115510579F56EEB99
:108310007FE086E09CE00E94C88965EB7FE086E014
:108320009CE00E94C889B80186E09CE00E947189A7
:1083300063EB7FE086E09CE00E94C88986E09CE0D9
:108340000E944188C15ADF4F0FB6F894DEBF0FBEBE
:10835000CDBFDF91CF911F910F91FF90EF90DF90F4
:10836000CF90BF90AF909F908F900895460F571F6A
:10837000DA011C920E94CB284B016DEA7FE086E077
:108380009CE00E94C889B40186E09CE00E94399F6D
:108390006AEA7FE086E09CE00E94C889B80186E036
:1083A0009CE00E94718967EA7FE086E09CE00E9481
:1083B000C889BAE38B16B1E09B064CF46AE97FE00A
:1083C0008FE59BE00E94C8898FE59BE0B9CF68E903
:1083D0007FE086E09CE00E94C889B60186E09CE0D0
:1083E0000E94718966E97FE086E09CE00E94C8896E
:1083F00086E09CE00E9441881A821982FE01339631
:108400008EE3DF011D928A95E9F78091CD08909166
:10841000CE08059791F563E070E0C8010E945A28E4
:108420007C01892BD1F5E091D80AF091D90A80819D
:1084300080FF88CF61E070E0C8010E945A28892B34
:1084400009F480CF64E270E0C8010E9474D8892BDF
:1084500009F078CF68E77FE086E09CE00E94C88959
:10846000B80186E09CE00E94718986E09CE00E9451
:108470004188C8010E9436A765CF61E070E0C8015D
:108480000E945A287C01892B09F465C04FE350E013
:10849000B801CE0101960E9465D8A12CBB24B394EB
:1084A000E00EF11E6FE67FE0C7010E9420CC892B11
:1084B00009F45EC064E270E0C8010E9474D8892BA0
:1084C00009F040CFB11003C0AA2009F43BCF40917E
:1084D000660750916707B701CE018F5B9F4F0E94DF
:1084E000FB3CCE018F5B9F4F0E94773B182F882368
:1084F00059F0B601CE018F5B9F4F0E94C0A111E0E1
:10850000181619060CF010E0CE018F5B9F4F0E94E9
:108510003741112309F416CF8981882309F412CF3A
:108520008091CD089091CE08059709F40BCF61E5B5
:108530007FE086E09CE00E94C889BE016F5F7F4FAC
:1085400086E09CE00E94718986E09CE00E94418860
:10855000CE0101968FCF62E070E0C8010E945A28D8
:108560007C01892B09F4EECEAA24A394B12C98CFD8
:10857000F60101900020E9F73197EC19FD093297D7
:1085800008F498CFC8010E9436A7B11003C0AA20F2
:1085900009F4D8CEC6010E948E8ED4CECF93DF933D
:1085A000EC01598348837B836A831C861B861D8666
:1085B0001E8E1D8E0E94773B882329F0CE01DF910D
:1085C000CF910C94253CDF91CF9108952F923F924B
:1085D0004F925F926F927F928F929F92AF92BF92D3
:1085E000CF92DF92EF92FF920F931F93CF93DF937F
:1085F000CDB7DEB7A4970FB6F894DEBF0FBECDBFE0
:10860000FC016115710509F4D0C0DB0118969C913D
:108610009F70953009F0C9C0EBA20AA319013A0175
:10862000F9A3E8A3FB0146805780809162078F5F22
:1086300080936207FE2DF160FCA34114510409F4FC
:10864000AFC0D20118968C918F70843049F018F029
:10865000873008F491C0D20112964D905C90EDCF16
:10866000F20161857285A8A1B9A18D919C910E94AA
:10867000CB9A4C01009779F3FC0180858F7085308F
:1086800051F74091660750916707B401CE010196FA
:108690000E94CE426114710419F1CE0101960E942C
:1086A000773B8823E9F0AAA0CCA07101D3010C91FB
:1086B00011961C91119712962C91129713963C913A
:1086C000139714964C91149715965C9115971696DE
:1086D0006C91169717967C91CE0101960E941646D2
:1086E0008B858730A9F561E0C4010E94439BEBA014
:1086F0000AA19101A301BC0188A199A10E94E642AF
:1087000061147104A1F5882391F180916207815071
:1087100080936207CE0101960E94374181E0A496C2
:108720000FB6F894DEBF0FBECDBFDF91CF911F9182
:108730000F91FF90EF90DF90CF90BF90AF909F9000
:108740008F907F906F905F904F903F902F90089503
:108750006114710461F4CE0101960E94773B882375
:1087600031F0CE0101960E94D743892B71F6CE01DC
:1087700001960E9437416FCF912C812CB12CA12CF6
:10878000D12CC12CF301E080F1800281138124817E
:108790003581468157816FEFC2010E9460585BCFDF
:1087A0008091620781508093620780E0B8CFCF92BA
:1087B000DF92EF92FF920F931F93CF93DF9300D03E
:1087C00000D01F921F92CDB7DEB76C0119821A82BA
:1087D0001B821C821D821E821F8218868A81807FD6
:1087E0008A8361ED7AE086E09CE00E94C889D60128
:1087F0001296ED91FC916081718186E09CE00E946F
:1088000071896FEC7AE086E09CE00E94C889C6011D
:108810000E94773B81111CC066EC7AE086E09CE008
:108820000E94C88986E09CE00E9441880FEF1FEFFC
:10883000C80128960FB6F894DEBF0FBECDBFDF91FA
:10884000CF911F910F91FF90EF90DF90CF900895FF
:10885000C6010E94F53DF82EF601838594850097A8
:1088600091F0DC01ED91FC910288F389E02D1995DE
:108870008C0197FD08C081E00115110509F480E025
:108880000E94051AD5CFF6018285873009F431C0E0
:10889000EFEFEF0DE63108F02CC0F0E08827EC5A3E
:1088A000FB4B8F4F0C94D6D36A447344794479447C
:1088B00073446A44794479447944794479447944E5
:1088C00079446A4479447944794479446A446A44ED
:1088D0006A446A4467EA7AE086E09CE00E94C889BC
:1088E00001E010E0A5CF80E00E94051A10E000E052
:1088F0009FCF40E050E2B601CE0101960E940240B7
:10890000D6011A968C911A97873071F160F48330F2
:1089100009F456C0843061F067EB7AE086E09CE0B1
:108920000E94C889E3CF883009F44AC08930A1F792
:10893000CE0101960E94529B8C016CEA7AE086E09F
:108940009CE00E94C889B80186E09CE00E94399FA3
:1089500086E09CE00E94418891E080E0012B09F4D0
:1089600090E0092F182F64CF1496ED91FC9180852B
:108970008F7010E000E0853001F764EC7AE086E06B
:108980009CE00E94C889F60164817581E12C00E0B9
:1089900030E020E050E040E0C6010E94E642F82EC0
:1089A000082F10E061EC7AE086E09CE00E94C88924
:1089B0008F2D0E94051A86E09CE00E94418838CFE6
:1089C000CE0101960E94CB318B01B7CF4F925F92BF
:1089D0006F927F928F929F92AF92BF92CF92DF92CF
:1089E000FF920F931F93CF93DF9300D000D01F927D
:1089F0001F92CDB7DEB76130710509F481C0FC016B
:108A0000628173816115710509F47AC08C01198244
:108A10001A821B821C821D821E821F8218868A81F6
:108A2000807F8A8340E050E2CE0101960E9402409E
:108A3000CE0101960E94529B6C01F80182819381C4
:108A40000E94D93D2B013C01F801278130854185E9
:108A50005285D6010E94ABD32FEF30E040E050E0CA
:108A60000E945FD349015A010E94ABA9FF24F394ED
:108A700081149104A104B10461F064197509860997
:108A80009709FF24F394681579058A059B0508F476
:108A9000F12C411451046104710491F1F8018780B3
:108AA0009084A184B2840E94ABA9F801811491043E
:108AB000A104B10451F06419750986099709681574
:108AC00079058A059B0508F449C0A280B3804FEF61
:108AD0005FEFBA0180E00E948824AB01BC01C501B0
:108AE0000E94983DCD2861F0F80184810E946513B1
:108AF000F8019681891304C061E0C8010E94023E1A
:108B000090E080E028960FB6F894DEBF0FBECDBF90
:108B1000DF91CF911F910F91FF90DF90CF90BF9089
:108B2000AF909F908F907F906F905F904F9008953F
:108B3000FF20D9F060E0C8010E94023EF801828166
:108B400093810E94D743892BD9F640E050E0BA01C7
:108B5000F801828193810E94983DD2CF84810E9446
:108B60006513F80196818913E3CFCD2849F2F80106
:108B700084810E946513F80196818913C1CFF11099
:108B8000BFCFBACFCF93DF93EC016EE67AE186E0F8
:108B90009CE00E94C88969E67AE186E09CE00E9438
:108BA000C8896C817D8186E09CE00E94399F63E6E4
:108BB0007AE186E09CE00E94C88986E09CE00E9401
:108BC000418861E08C810E94F8A86E818C810E94AE
:108BD000CAA88A819B81009729F040E050E0BA0141
:108BE0000E94983DE881F9810484F585E02D62E0DA
:108BF000CE0119958A819B81009799F00E94D743F5
:108C00001816190674F40A80DB81C02D4FEF5FEF50
:108C1000BA0180E00E948824AB01BC01CE010E9411
:108C2000983D81E090E0DF91CF9108952F923F929F
:108C30004F925F926F927F928F929F92AF92BF926C
:108C4000CF92DF92EF92FF920F931F93CF93DF9318
:108C5000CDB7DEB7C95DD1090FB6F894DEBF0FBE40
:108C6000CDBF1C01C754DF4F0883C95BD040C65439
:108C7000DF4F1883CA5BD040C554DF4F2883CB5BDE
:108C8000D040C454DF4F3883CC5BD040C354DF4F57
:108C90004883CD5BD040C254DF4F5883CE5BD04079
:108CA000C154DF4F6883CF5BD040C054DF4F78831F
:108CB000C05CD040CF53DF4FF982E882C15CD04026
:108CC000CD52DF4FC882C35DD040C053DF4FA88272
:108CD000C05DD0400E94CB286B01CC52DF4F79831E
:108CE0006883C45DD040683C71059CF46EE87AE00E
:108CF0008FE59BE00E94C889B6018FE59BE00E944A
:108D0000399F8FE59BE00E9441882FEF3FEF0C9445
:108D10005B510E94ABA9CA52DF4F688379838A8373
:108D20009B83C65DD040C554DF4F8881CB5BD0406C
:108D3000A82FB0E0C553DF4FB983A883CB5CD040E8
:108D4000E091CD08F091CE08CF52DF4FF983E88350
:108D5000C15DD040CF53DF4FE881F981C15CD04085
:108D6000309721F0808181110C94FF55D1011D961F
:108D70008C91882341F0C1010D96CF53DF4F998329
:108D80008883C15CD040C553DF4FE881F981CB5C5B
:108D9000D040EF2B11F00C945B56CF53DF4FE8819E
:108DA000F981C15CD040309711F00C940856D10184
:108DB0005D960D90BC91A02DC553DF4FB983A8835C
:108DC000CB5CD040AB2B11F40C945B56C554DF4FF9
:108DD0008881CB5BD04081110C945B56C553DF4F2B
:108DE0006881CB5CD040CE0187549F4F0E94DE2D1E
:108DF000CF55DF4F2883C15AD040CE55DF4F38833F
:108E0000C25AD040CD55DF4F4883C35AD040CC55CD
:108E1000DF4F5883C45AD040CB55DF4F6883C55AC3
:108E2000D040CA55DF4F7883C65AD040C955DF4F6E
:108E30008883C75AD040C855DF4F9883C85AD0405E
:108E40000C945B56D10112968D919C91892B09F45B
:108E50005CCFC553DF4FE881F981CB5CD0403197BF
:108E6000A1F4C654DF4F8881CA5BD0408F70F1E017
:108E7000C153DF4FF883CF5CD040811128C0C1536C
:108E8000DF4F1882CF5CD04022C0C553DF4F08812E
:108E90001981CB5CD040012B09F044C0C754DF4F8F
:108EA0008881C95BD040882309F44EC08850823045
:108EB00008F44AC0C153DF4F1882CF5CD04081E034
:108EC00090E0C553DF4F99838883CB5CD040C75473
:108ED000DF4F1881C95BD040112309F45DC040E029
:108EE00052E060E070E0C1010E94AC19672B682B72
:108EF000692B09F451C01C3009F44EC06BE47AE0D0
:108F00008FE59BE00E94C8898FE59BE00E94418825
:108F1000AAEFBFEFC953DF4FB983A883C75CD04026
:108F20000C94B456C553DF4F28813981CB5CD040B7
:108F30002430310509F4A3CF2930310509F49FCF3E
:108F40002330310509F469C0C654DF4F8881CA5BFC
:108F5000D0408F7009F461C040E054E060E070E000
:108F6000C1010E94AC19672B682B692B09F455C00D
:108F700066E37AE08FE59BE00E94C8898FE59BE07D
:108F80000E944188EAEFFFEFC953DF4FF983E8837E
:108F9000C75CD0400C94B456C553DF4F088119818B
:108FA000CB5CD04004301105E9F5C053DF4FE880B9
:108FB000C05DD040C754DF4F0881C95BD040C65464
:108FC000DF4F1881CA5BD040C554DF4F2881CB5B8F
:108FD000D040C454DF4F3881CC5BD040C354DF4F06
:108FE0004881CD5BD040C254DF4F5881CE5BD0402A
:108FF000C154DF4F6881CF5BD040C054DF4F7881D0
:10900000C05CD040C1010E946E34C953DF4F9983C8
:109010008883C75CD0400C94B456C153DF4F18828C
:10902000CF5CD040CD52DF4F1881C35DD0401330AC
:1090300091F4D1011A968C91873069F468E17AE055
:1090400086E09CE00E94C88986E09CE00E944188FE
:10905000E9EFFFEF99CF88E0FE01E754FF4FDE0113
:10906000AF54BF4F01900D928A95E1F7E114F104DE
:1090700009F451C067EC7BE0C7010E9420CC892B2A
:1090800009F450C061ED7BE0C7010E9420CC892B20
:1090900009F451C06FEE7BE0C7010E9420CC892B00
:1090A00009F452C069EF7BE0C7010E9420CC892BF4
:1090B00009F453C065E87CE0C7010E9420CC892BED
:1090C00009F454C06FE87CE0C7010E9420CC892BD2
:1090D00009F46CC069E47CE0C7010E9420CC892BB4
:1090E00009F467C063E57CE0C7010E9420CC892BAE
:1090F00009F462C069E97CE0C7010E9420CC892B99
:1091000009F45DC06BE77CE0C7010E9420CC03E15D
:1091100010E0892B69F1C353DF4F19821882CD5CAF
:10912000D0402CC021E030E0C353DF4F3983288387
:10913000CD5CD04023C082E090E0C353DF4F9983E1
:109140008883CD5CD0401AC0A5E0B0E0C353DF4FA8
:10915000B983A883CD5CD04011C0E6E0F0E0C353F2
:10916000DF4FF983E883CD5CD04008C004E110E014
:10917000C353DF4F19830883CD5CD040C754DF4F02
:109180001881C95BD040143009F4F3C2D8F411231C
:1091900009F444C0412C512C32010FEF1FEFC95389
:1091A000DF4F19830883C75CD0407DC325E130E0E1
:1091B000BBCF8EE090E0C1CFAFE0B0E0C7CFE6E13B
:1091C000F0E0CDCF88EF810F823020F788E0FE01FC
:1091D000E754FF4FDE01119601900D928A95E1F759
:1091E000C654DF4FE881CA5BD040EF7009F493C3E7
:1091F000E150EB3008F08FC3F0E08827ED5FF64BCD
:109200008F4F0C94D6D3794C794C8B4C6A4C6A4C6A
:10921000E44CD34CD34CD34C6A4C6A4C19821A821E
:109220001B821C821D821E821F8218868A81807F7B
:109230008A83C654DF4F8881CA5BD0408F7009F49F
:109240008CC2C553DF4F08811981CB5CD0400A30F6
:10925000110509F435C25CF40115110579F10230EC
:10926000110509F4C3C0412C512C320120C2C55351
:10927000DF4F28813981CB5CD0402B30310509F498
:10928000B8C12C30310579F7B101CE0101960E94A9
:10929000BC9FCE0187549F4F0E94C714BC01CE01D2
:1092A00001960E94733688E0FE013196DE01A754D4
:1092B000BF4F01900D928A95E1F7F4C1EF2859F064
:1092C00063E07AE086E09CE00E94C88986E09CE04A
:1092D0000E944188C8CFC1010E94D74318161906C1
:1092E00014F00C94E955CE0187549F4F0E94CB3166
:1092F000672B682B692B09F072C162E0CE0187549D
:109300009F4F0E94002EC756DF4F2883C959D04077
:10931000C656DF4F3883CA59D040C556DF4F488301
:10932000CB59D040C456DF4F5883CC59D040C35698
:10933000DF4F6883CD59D040C256DF4F7883CE5976
:10934000D040C156DF4F8883CF59D040C056DF4F41
:109350009883C05AD0404424439430E1532E612C6A
:10936000712C31E0CD53DF4F3883C35CD040AA2449
:10937000A39446C061E0CE0187549F4F0E94002E07
:10938000CF56DF4F2883C159D040CE56DF4F3883A8
:10939000C259D040CD56DF4F4883C359D040CC5638
:1093A000DF4F5883C459D040CB56DF4F6883C5592F
:1093B000D040CA56DF4F7883C659D040C956DF4FD8
:1093C0008883C759D040C856DF4F9883C859D040CA
:1093D0004424439420E1522E612C712C81E0CD5322
:1093E000DF4F8883C35CD040A12C0AC0412C512C94
:1093F0003201CD53DF4F1882C35CD040AA24AA9417
:10940000B101CE0101960E94BC9F8A819CE0980F19
:109410009F70923058F4C654DF4F9881CA5BD04099
:109420009F70923019F4807F82608A83D1011A96EE
:109430009C91973069F4C654DF4F8881CA5BD04055
:109440008F708250843020F48A81807F82608A838A
:10945000F101A385B485892F90E0109741F0ED913B
:10946000FC911197008CF18DE02DCD0119957C01B7
:10947000C754DF4F0881C95BD040C654DF4F188105
:10948000CA5BD040C554DF4F2881CB5BD040C45469
:10949000DF4F3881CC5BD040C354DF4F4881CD5B78
:1094A000D040C254DF4F5881CE5BD040C154DF4F13
:1094B0006881CF5BD040C054DF4F7881C05CD04022
:1094C000CE0101960E94AD36C757DF4F2883C95899
:1094D000D040C657DF4F3883CA58D040C557DF4FFA
:1094E0004883CB58D040C457DF4F5883CC58D04026
:1094F000C357DF4F6883CD58D040C257DF4F7883C2
:10950000CE58D040C157DF4F8883CF58D040C05786
:10951000DF4F9883C059D040CE0101960E94922D12
:10952000CD53DF4FF881C35CD040FF2359F1C654BF
:10953000DF4F8881CA5BD0408F709FE0980F9F708B
:10954000923020F08A5F8F708230E0F48A818F70D1
:1095500081508230B8F42D8130E0AFEFB0E00E944E
:10956000B3D324E630E040E050E00E9481D32F3FA7
:1095700031054105510529F024F02FEF30E040E09E
:1095800050E02D8388E0FE013196DE01A754BF4FE5
:1095900001900D928A95E1F708E2502AB12C2FEF45
:1095A0003FEFC953DF4F39832883C75CD040D101D7
:1095B0001A968C911A97873009F01CC6CC52DF4F4F
:1095C000E881F981C45DD040EE35F1400CF0B9C4BA
:1095D00063EB79E08FE59BE00E94C88992CB412C38
:1095E000512C320191E0CD53DF4F9883C35CD040C2
:1095F000BECEB101CE0101960E94BC9FC254DF4F86
:109600009881CE5BD0408A81282F2F7041F0223084
:1096100049F0412C512C3201BB24B39449C0807FC6
:1096200082608A83892F90E08536910514F084E664
:1096300090E08E8388E0FE013196DE01A754BF4F93
:1096400001900D928A95E1F762E0CE0187549F4F19
:109650000E94DE2DCF57DF4F2883C158D040CE5710
:10966000DF4F3883C258D040CD57DF4F4883C358AF
:10967000D040CC57DF4F5883C458D040CB57DF4F32
:109680006883C558D040CA57DF4F7883C658D0404A
:10969000C957DF4F8883C758D040C857DF4F9883DA
:1096A000C858D040412C98E2592E612C712CB12C15
:1096B000CD53DF4F1882C35CD040AA24AA946FCF49
:1096C000B101CE0101960E94BC9FC154DF4F688159
:1096D000CF5BD040C054DF4F7881C05CD040717008
:1096E000CE0101960E94363BCD53DF4F8883C35C89
:1096F000D040412C512C3201BB24B3948823E9F291
:1097000088E0FE013196DE01A754BF4F01900D9213
:109710008A95E1F762E0CE0187549F4F0E94DE2DCB
:10972000EA962FAFEA97EB963FAFEB97EC964FAFE9
:10973000EC97ED965FAFED97EE966FAFEE97EF96E5
:109740007FAFEF97C158DF4F8883CF57D040C058C5
:10975000DF4F9883C058D040A5CF412C512C320107
:109760008FEF9FEFC953DF4F99838883C75CD04049
:109770009AC0C553DF4FA881B981CB5CD0401997FF
:1097800009F471C0C1010E94D74318161906B4F537
:1097900062E0CE0187549F4F0E94002EE2962FAFC9
:1097A000E297E3963FAFE397E4964FAFE497E596F1
:1097B0005FAFE597E6966FAFE697E7967FAFE797DF
:1097C000E8968FAFE897E9969FAFE99744244394D2
:1097D00080E1582E612C712CEFEFFFEFC953DF4F62
:1097E000F983E883C75CD040B12CF1E0CD53DF4F63
:1097F000F883C35CD040AA24A394D9CE61E0CE0103
:1098000087549F4F0E94002EAA962FAFAA97AB961F
:109810003FAFAB97AC964FAFAC97AD965FAFAD9700
:10982000AE966FAFAE97AF967FAFAF97E0968FAF24
:10983000E097E1969FAFE1974424439400E1502ED6
:10984000612C712C0FEF1FEFC953DF4F1983088371
:10985000C75CD040B12C11E0CD53DF4F1883C35CFF
:10986000D040A12CA4CE40E051E060E070E0C10106
:109870000E94AC19672B682B692BE1F040E051E0A6
:1098800060E070E0C1010E945A194424439410E43E
:10989000512E612C712C21E030E0C953DF4F398308
:1098A0002883C75CD040B12CCD53DF4F1882C35CF6
:1098B000D04066C240E051E060E070E0C1010E942B
:1098C000831944244394B0E45B2E612C712C81E015
:1098D00090E048CFC354DF4F288139814A815B81B2
:1098E000CD5BD040A4E6B0E00E94A0D36B017C0128
:1098F0000DC0C354DF4FC880CD5BD04094E6C99EF5
:10990000600111240D2C000CEE08FF08C114D104D5
:10991000E104F10429F4A5E0CA2ED12CE12CF12CAC
:10992000193041F4F094E094D094C094C11CD11C3F
:10993000E11CF11CB101CE0187549F4F0E94BC9FD6
:1099400060E0CE0187549F4F0E94002EA2962FAF59
:10995000A297A3963FAFA397A4964FAFA497A596BF
:109960005FAFA597A6966FAFA697A7967FAFA7976D
:10997000A8968FAFA897A9969FAFA997C553DF4F19
:10998000A881B981CB5CD040AA30B10509F4FBC1F4
:1099900024F5109709F4BEC0129709F47AC0412C3F
:1099A000512C32014EC220E030E048EC52E4C35466
:1099B000DF4F688179818A819B81CD5BD0400E9495
:1099C0007BD20E94D3D492CFC354DF4FC880D980BA
:1099D000EA80FB80CD5BD04099CFC553DF4FE88153
:1099E000F981CB5CD040EB30F10509F44BC23C97D8
:1099F000B1F6C654DF4F8881CA5BD0408F70823089
:109A000009F092C2C701B60124E630E040E050E020
:109A10000E9481D3C054DF4F8881C05CD0408695BE
:109A200090E0280F391F1216130614F021E030E0E1
:109A30002536310514F024E630E0220FC054DF4F04
:109A40008881C05CD0408170282BC054DF4F2883B0
:109A5000C05CD04062E0CE0187549F4F0E94DE2D53
:109A60002A962FAF2A972B963FAF2B972C964FAF66
:109A70002C972D965FAF2D972E966FAF2E972F9622
:109A80007FAF2F9760968FAF609761969FAF61977A
:109A9000D3C1CD53DF4F1882C35CD040D1011B9698
:109AA0008D919C911C97009709F03BC01A968C9160
:109AB00090E0E0E58E2E912CA12CB12C8530910503
:109AC00049F0812C912C5401449721F0812C912C48
:109AD00054018A943E01B9EB6B0E711CD3011196AF
:109AE000EC911197EF70E150EB3008F034C1F0E0E9
:109AF00023018827E158F24B8F4F0C94D6D3994D10
:109B0000994DAB4EAB4EAB4E7C4E3E4E3E4E3E4E16
:109B1000CD4DCD4DF1E0CD53DF4FF883C35CD04048
:109B2000BDCFDC01ED91FC91008CF18DE02D1995FC
:109B3000C0CFF3011481C701B60124E630E040E054
:109B400050E00E9481D3DA01C901810F911DA11D4E
:109B5000B11DB7FF03C080E090E0DC018F3F9105AD
:109B6000A105B10529F024F08FEF90E0A0E0B0E06E
:109B7000C354DF4F8883CD5BD04066EA74E086E053
:109B80009CE00E947189C2010E94922D412C78E2D2
:109B9000572E612C712CB12CEBC014960D911D9198
:109BA0002D913C911797C953DF4F088319832A835E
:109BB0003B83C75CD040B4E6CB16D104E104F1048A
:109BC00084F5A4E6B0E0A90198010E94A0D3C60ED6
:109BD000D71EE81EF91E81149104A104B104B9F046
:109BE000A50194010E94A0D3362F272FB701A6010B
:109BF00077FF03C040E050E0BA01C32ED22E7C01B3
:109C00004C155D056E057F0514F46A017B01F301B7
:109C1000C482D582E682F7828181807F86608183DB
:109C2000ACCFC701B60124E630E040E050E00E942E
:109C300081D3C953DF4F88819981AA81BB81C75CD9
:109C4000D040280F391F4A1F5B1F81149104A104C3
:109C5000B10461F057FF03C020E030E0A901821693
:109C60009306A406B50614F4A5019401D201149636
:109C70002D933D934D935C9317977FCFF3016481B0
:109C80007581868197810E94D3D4C953DF4F688341
:109C900079838A839B83C75CD040C701B60124E6E1
:109CA00030E040E050E00E9481D3C953DF4F68812B
:109CB00079818A819B81C75CD040620F731F841FAA
:109CC000951F81149104A104B10461F097FF03C0B2
:109CD00060E070E0CB0186169706A806B90614F47A
:109CE000C501B4010E941CD2D30114966D937D93DB
:109CF0008D939C93179741CFF30184819581A68121
:109D0000B781C80ED91EEA1EFB1E81149104A1045E
:109D1000B104C9F0A4E6B0E0A50194010E94A0D36B
:109D2000362F272FB701A60177FF03C040E050E090
:109D3000BA01C32ED22E7C014C155D056E057F0540
:109D400014F46A017B01D3011496CD92DD92ED9259
:109D5000FC92179712CF88E0FE013196D301019053
:109D60000D928A95E1F7412C512C3201BB24B3941A
:109D7000EFEFFFEFC953DF4FF983E883C75CD040B3
:109D8000AA24AA9414CCC654DF4F8881CA5BD04061
:109D90008F70823009F057C0C701B60124E630E069
:109DA00040E050E00E9481D3C154DF4F8881CF5BF7
:109DB000D040C054DF4F6881C05CD040962F917076
:109DC000280F391F2E36B1E03B072CF437FF05C0B2
:109DD0002DE631E002C030E020E0C154DF4F28839F
:109DE000CF5BD040C054DF4F8881C05CD04030FB97
:109DF00080F9C054DF4F8883C05CD04062E0CE0160
:109E000087549F4F0E94DE2D6A962FAF6A976B96FC
:109E10003FAF6B976C964FAF6C976D965FAF6D973A
:109E20006E966FAF6E976F967FAF6F97A0968FAF5E
:109E3000A097A1969FAFA197412C68E2562E612C66
:109E4000712CB12C19C088E0FE013196DE01A754B7
:109E5000BF4F01900D928A95E1F767EF79E08FE5AA
:109E60009BE00E94C8898FE59BE00E944188412CBD
:109E7000512C3201BB24B394CD53DF4F1882C35C05
:109E8000D04076CFC654DF4F8881CA5BD0408F70F8
:109E90008230E9F5C701B60124E630E040E050E049
:109EA0000E9481D3C254DF4F8881CE5BD04090E0C6
:109EB000280F391F37FF02C030E020E0253631057A
:109EC00014F024E630E0C254DF4F2883CE5BD0404C
:109ED00062E0CE0187549F4F0E94DE2D62962FAF25
:109EE000629763963FAF639764964FAF64976596AA
:109EF0005FAF659766966FAF669767967FAF679718
:109F000068968FAF689769969FAF699795CF88E0FD
:109F1000FE013196DE01A754BF4F01900D928A9544
:109F2000E1F76BEE79E09BCF88E0FE013196DE0130
:109F3000A754BF4F01900D928A95E1F76FED79E03C
:109F40008ECFCD52DF4F3881C35DD04030FD77C01A
:109F50001496ED91FC9180858F70853009F06FC06B
:109F6000CF52DF4FE881F981C15DD040359709F4C8
:109F700066C0C553DF4F08811981CB5CD0400130EA
:109F8000110509F011C7C754DF4F8881C95BD04064
:109F90008A50823008F0ADC76BE979E086E09CE03A
:109FA0000E94C889D1011296ED91FC916081718166
:109FB00086E09CE00E94718986E09CE00E944188D6
:109FC000C754DF4F8881C95BD0408A3071F08B3035
:109FD000C1F030E020E040E050E460E070E0C1011A
:109FE0000E947E4001E010E0B9C640E051E060E030
:109FF00070E0C1010E945A196AE0C1010E94D019A3
:10A00000E8CFC053DF4FB881C05DD040B1110EC062
:10A0100062E879E08FE59BE00E94C8898FE59BE0CC
:10A020000E944188EBEFFFEF0C94C44740E051E001
:10A0300060E070E0C1010E9483196BE0DECF10E0A8
:10A04000C353DF4F28813981CD5CD040232B09F4E5
:10A0500041C7CF53DF4F19821882C15CD0403AC745
:10A06000863009F454C7873009F041C7C1010E9406
:10A07000F53D082F863009F062C066E579E086E09C
:10A080009CE00E94C88966E070E086E09CE00E9447
:10A09000399F86E09CE00E94418862E0CE018754AF
:10A0A0009F4F0E94002E29AF3AAF4BAF5CAF6DAF10
:10A0B0007EAF8FAF21969FAF21973DC0C1010E9417
:10A0C000F53D853021F083E090E00C9405486DE685
:10A0D00079E086E09CE00E94C88965E070E086E057
:10A0E0009CE00E94399F86E09CE00E944188B1017B
:10A0F000CE0187549F4F0E94BC9F61E0CE018754E0
:10A100009F4F0E94002E22962FAF229723963FAF9B
:10A11000239724964FAF249725965FAF25972696D1
:10A120006FAF269727967FAF279728968FAF2897F0
:10A1300029969FAF2997689440F854F8D8C668E3E9
:10A1400079E086E09CE00E94C889602F70E086E09C
:10A150009CE00E94399F86E09CE00E944188A3E039
:10A16000B0E00C948A47AA2009F4E7C66EE179E0D2
:10A1700086E09CE00E94C889E3E0F0E00C94C447CC
:10A1800069E079E086E09CE00E94C88903E010E085
:10A19000E5C52FEFA2120DC0C1010E94D7431816CA
:10A1A00019064CF06CEE78E086E09CE00E94C889CD
:10A1B0008ACFAA20B9F362E0CE0187549F4F0E9454
:10A1C000002E29A73AA74BA75CA76DA77EA78FA74C
:10A1D00098AB689440F854F835E0932EC7C640E039
:10A1E00050E2B101CE0187549F4F0E94024081117D
:10A1F000DCC6DDC6BFEFAB1265C0C1010E94D7430C
:10A20000AA24A394181619060CF45FC0A12C6EEDB5
:10A2100078E086E09CE00E94C889EA2C0A2C000CB9
:10A22000FF08B70186E09CE00E94399F67ED78E067
:10A2300086E09CE00E94C889CD53DF4FF881C35C63
:10A24000D0406F2F70E086E09CE00E94399F86E04E
:10A250009CE00E944188CF53DF4F88809980C15C89
:10A26000D04081149104F1F1C1010E94F53DC82E46
:10A27000D12CC114D10409F46701C353DF4F088105
:10A280001981CD5CD0400115110509F453C0C016E9
:10A29000D10611F16BEB78E086E09CE00E94C88962
:10A2A000B60186E09CE00E94399F86E09CE00E9417
:10A2B00041882DEF3FEFC953DF4F39832883C75CB7
:10A2C000D04052C5AA2009F4A2CFE1E0CD53DF4F20
:10A2D000E883C35CD0409BCFCF53DF4F19821882F5
:10A2E000C15CD040C754DF4F9880C95BD040B6E115
:10A2F000B91508F4E5C1E92DF0E08827ED57FE4ACD
:10A300008F4F0C94D6D3DD51165307531952DD519C
:10A31000E852AA526152DD51DD515C535C537B53CC
:10A320007B5338533853605360536053385338531A
:10A3300038533853D1011B968D919C91009709F4A5
:10A34000D1CFDC01ED91FC910088F189E02DC05363
:10A35000DF4FA880C05DD040CD53DF4FC880C35CC5
:10A36000D0407401C754DF4F0881C95BD040C65448
:10A37000DF4F1881CA5BD040C554DF4F2881CB5BCB
:10A38000D040C454DF4F3881CC5BD040C354DF4F42
:10A390004881CD5BD040C254DF4F5881CE5BD04066
:10A3A000C154DF4F6881CF5BD040C054DF4F78810C
:10A3B000C05CD04019950C940548912CC153DF4FD7
:10A3C0002881CF5CD040222309F404C6C053DF4F5C
:10A3D000C880C05DD040CF54DF4F0881C15BD04002
:10A3E000CE54DF4F1881C25BD040CD54DF4F28815F
:10A3F000C35BD040CC54DF4F3881C45BD040CB54DA
:10A40000DF4F4881C55BD040CA54DF4F5881C65BDF
:10A41000D040C954DF4F6881C75BD040C854DF4F7C
:10A420007881C85BD040C1010E943A35E89455F864
:10A43000D1C5C1010E94F53D853009F044CE66EAE0
:10A4400078E086E09CE00E94C88965E070E086E0E4
:10A450009CE00E94399F86E09CE00E944188B10107
:10A46000CE0187549F4F0E94BC9FF10182858530A9
:10A47000C9F46EE0CE0187549F4F0E94002E29A39D
:10A480003AA34BA35CA36DA37EA38FA398A7689464
:10A4900040F854F8912CF1E0CD53DF4FF883C35CC2
:10A4A000D0408CCF61E0CE0187549F4F0E94002E98
:10A4B000298F3A8F4B8F5C8F6D8F7E8F8F8F98A3F4
:10A4C000E6CFC1010E94F53D182F863081F56FE877
:10A4D00078E086E09CE00E94C88966E070E086E053
:10A4E0009CE00E94399F86E09CE00E94418862E0E7
:10A4F000CE0187549F4F0E94002E298B3A8B4B8BA5
:10A500005C8B6D8B7E8B8F8B988F40E050E068E08A
:10A5100070E0C1010E945A19689440F854F8912CD7
:10A5200001E0CD53DF4F0883C35CD04047CF61E7E4
:10A5300078E086E09CE00E94C889612F70E086E0A8
:10A540009CE00E94399F86E09CE00E94418823E0C5
:10A5500030E0B1CE40E051E060E070E0C1010E9427
:10A56000AC19672B682B692B61F5A11027C0B101CD
:10A57000CE0187549F4F0E94BC9F61E0CE0187545B
:10A580009F4F0E94002E29873A874B875C876D87F3
:10A590007E878F87988B40E050E068E070E0C101D3
:10A5A0000E948319689440F854F826E0922E31E016
:10A5B000CD53DF4F3883C35CD04000CF67E578E0F0
:10A5C000F3CD62E478E086E09CE00E94C889C7CDC4
:10A5D000AA20D1F062E0CE0187549F4F0E94002E46
:10A5E00029833A834B835C836D837E838F83988733
:10A5F000689440F854F895E0992EB1E0CD53DF4FC0
:10A60000B883C35CD040DACE65E278E0B1CDC55402
:10A61000DF4F8881CB5BD040823008F073C0C1012E
:10A620000E94F53D853009F032CF4DCDC554DF4F46
:10A630008881CB5BD040823008F02CCFAA20C1F0BB
:10A640006CE078E086E09CE00E94C88961E0C1018E
:10A650000E94D019CF53DF4F28813981C15CD0408F
:10A6600040E058E160E070E0C1010E947E408ECD84
:10A67000C554DF4F8881CB5BD040823008F04FCF8C
:10A68000992009F447C0C654DF4F8881CA5BD04087
:10A690008F7031F4B101CE0187549F4F0E94BC9F4F
:10A6A000689440F810E3512A912C21E0CD53DF4FFC
:10A6B0002883C35CD04082CE689456F8912C77CF23
:10A6C000C654DF4F8881CA5BD0408F7051F46894C4
:10A6D00054F8912C81E0CD53DF4F8883C35CD04088
:10A6E0006DCE90E3592A912CA1E0CD53DF4FA88382
:10A6F000C35CD04063CE912C412C80E4582E612C59
:10A70000712C7BCF912CE1E0CD53DF4FE883C35C0C
:10A71000D04054CE11E0CD53DF4F1883C35CD040FE
:10A720004DCEF10183859485892B09F4CBC041146A
:10A7300051046104710439F0A201B101CE018754C2
:10A740009F4F0E94843BD1011B968D919C91CF53CA
:10A75000DF4FE880F980C15CD040DC01ED91FC91D5
:10A760000088F189E02DC053DF4FA880C05DD04044
:10A77000CD53DF4FC880C35CD040C754DF4F088142
:10A78000C95BD040C654DF4F1881CA5BD040C55466
:10A79000DF4F2881CB5BD040C454DF4F3881CC5B86
:10A7A000D040C354DF4F4881CD5BD040C254DF4F0F
:10A7B0005881CE5BD040C154DF4F6881CF5BD04021
:10A7C000C054DF4F7881C05CD0401995C953DF4F2A
:10A7D00099838883C75CD040F10183859485DC012F
:10A7E000ED91FC91008CF18DE02D1995059711F4F8
:10A7F000689440F856FCC5C1992021F0692DC1012B
:10A800000E94D019CF52DF4FA881B981C15DD040DD
:10A81000159709F425C430E020E0B301A201C1017D
:10A820000E947E40C153DF4FB881CF5CD040BB2334
:10A8300009F416C4CF53DF4F88819981C15CD040A1
:10A84000892B09F40DC46FEA77E086E09CE00E9452
:10A85000C88986E09CE00E944188CF53DF4FA880E2
:10A86000B980C15CD040812C73016201CF54DF4FAD
:10A870000881C15BD040CE54DF4F1881C25BD0400D
:10A88000CD54DF4F2881C35BD040CC54DF4F38819B
:10A89000C45BD040CB54DF4F4881C55BD040CA5425
:10A8A000DF4F5881C65BD040C954DF4F6881C75B1A
:10A8B000D040C854DF4F7881C85BD040C1010E94AE
:10A8C000222ECEC38285853009F484C0863009F0FB
:10A8D00093CFC754DF4FD880C95BD040DD2009F447
:10A8E00079C0C1010E949A9F7C0141145104610406
:10A8F000710439F0A201B101CE0187549F4F0E942B
:10A90000843BE114F10409F477CF10E000E0F7FE96
:10A9100005C0F194E194F10801E010E0C70101974E
:10A920008635910508F068CFCE2C61E08E2D0E940F
:10A93000F8A8EFEFED0DE63108F049C0F0E0882708
:10A94000EB55FB4A8F4F0C94D6D3BB54BD54E75400
:10A95000E754BD54BB54BD54E754E754E754E7549F
:10A96000E754E754BB54BB54E754E754E754BB5493
:10A97000E754BB54BB54F1E00F27602F8C2D0E948D
:10A98000CAA867EE77E086E09CE00E94C889B7011C
:10A9900086E09CE00E94399F65EE77E086E09CE0CF
:10A9A0000E94C889B80186E09CE00E94399F86E039
:10A9B0009CE00E944188689440F854F801E010E05F
:10A9C000C953DF4F19830883C75CD04015CF0FEF01
:10A9D0001FEFD7CF411451046104710439F0A20173
:10A9E000B101CE0187549F4F0E94843BC553DF4F76
:10A9F00028813981CB5CD0402230310509F4BDC0BB
:10AA00002330310581F02130310509F0F5CE68940D
:10AA100040F854F821E030E0C953DF4F39832883F0
:10AA2000C75CD040E9CEC1010E94D93D6B017C01D9
:10AA3000892B61F565ED77E085E59BE00E94C8898B
:10AA4000D1011296ED91FC916081718185E59BE0C9
:10AA50000E94718962EB74E085E59BE00E94718938
:10AA60002AE030E0B701A60185E59BE00E94E78877
:10AA700085E59BE00E944188D1011296ED91FC9101
:10AA80006081718188EB94E00E94FDAACE01875419
:10AA90009F4F0E94853120E030E048EC52E40E9454
:10AAA0007BD20E94D3D4C953DF4F688379838A83D2
:10AAB0009B83C75CD040C953DF4FC880D980C75C37
:10AAC000D0404FEF5FEF60E070E088E00E948824A4
:10AAD000CD53DF4F688379838A839B83C35CD040E7
:10AAE000CD53DF4FE880F980C35CD0406EEC77E057
:10AAF00086E09CE00E94C889D1011296ED91FC91FC
:10AB00006081718186E09CE00E9471896AEC77E047
:10AB100086E09CE00E94C889C953DF4F6881798133
:10AB2000C75CD04086E09CE00E94399F65EC77E0EE
:10AB300086E09CE00E94C889CD53DF4F488159814F
:10AB40006A817B81C35CD040662777272AE086E054
:10AB50009CE00E94F58786E09CE00E944188B70156
:10AB6000A601C1010E94983DE1E0F0E0C953DF4F2A
:10AB7000F983E883C75CD0403FCE689440F855F82D
:10AB80001DCF81E090E0C953DF4F99838883C75C74
:10AB9000D04032CECF52DF4FE881F981C15DD04045
:10ABA000359709F45DC240E050E4B101CE0187540D
:10ABB0009F4F0E94843B30E020E040E050E460E0A2
:10ABC00070E0C1010E947E404BC2ACEFBFEF0C941D
:10ABD0008A47CE0187549F4F0E94CB312B013C0105
:10ABE000411451046104710411F00C94BA49B1E0AC
:10ABF000CD53DF4FB883C35CD0400C94F449C553A8
:10AC0000DF4F08811981CB5CD040012B09F053C084
:10AC10008081882311F40C94D746CE018F539F4F27
:10AC20000E94543BC553DF4F99838883CB5CD0404F
:10AC3000C554DF4F8881CB5BD040811132C0C553F2
:10AC4000DF4F6881CB5CD040CE0187549F4F0E947C
:10AC5000DE2DC755DF4F2883C95AD040C655DF4F78
:10AC60003883CA5AD040C555DF4F4883CB5AD040AD
:10AC7000C455DF4F5883CC5AD040C355DF4F68834B
:10AC8000CD5AD040C255DF4F7883CE5AD040C155FF
:10AC9000DF4F8883CF5AD040C055DF4F9883C05BC9
:10ACA000D040C553DF4FE881F981CB5CD040EF2B1A
:10ACB00011F40C94D74663E87AE086E09CE00E94A9
:10ACC000C889B60186E09CE00E94399F6CE77AE073
:10ACD00086E09CE00E94C889D1011296ED91FC911A
:10ACE0006081718186E09CE00E94718966E77AE06C
:10ACF00086E09CE00E94C889CF53DF4F688179814C
:10AD0000C15CD04086E09CE00E94718964E77AE0F3
:10AD100086E09CE00E94C889CE0187549F4F0E9424
:10AD2000922DCF53DF4FE880F980C15CD040E11411
:10AD3000F10411F40C942247F7018081843211F060
:10AD40000C94224760E67AE086E09CE00E94C88985
:10AD500086E09CE00E9441880CEF1FEFC953DF4F53
:10AD600019830883C75CD040C953DF4F888199811C
:10AD7000C75CD040C752DF4F0FB6F894DEBF0FBE9E
:10AD8000CDBFDF91CF911F910F91FF90EF90DF909A
:10AD9000CF90BF90AF909F908F907F906F905F907B
:10ADA0004F903F902F9008951FEFA11225C0C10131
:10ADB0000E94D743AA24A394181619060CF0A12CBC
:10ADC000C553DF4F28813981CB5CD040213031051C
:10ADD00099F4C754DF4F8881C95BD040863061F455
:10ADE00040E051E060E070E0C1010E94AC19672BC7
:10ADF000682B692B09F081C0CF53DF4F288139813F
:10AE0000C15CD040D10114966D917C91CD52DF4F41
:10AE1000E880C35DD040C053DF4F0881C05DD040A3
:10AE2000AE0147545F4FC1010E94E642C153DF4F5C
:10AE3000B881CF5CD04010E0BB23C1F1C053DF4FDD
:10AE4000C880C05DD040EE24EA94FE2CCF54DF4F82
:10AE50000881C15BD040CE54DF4F1881C25BD04027
:10AE6000CD54DF4F2881C35BD040CC54DF4F3881B5
:10AE7000C45BD040CB54DF4F4881C55BD040CA543F
:10AE8000DF4F5881C65BD040C954DF4F6881C75B34
:10AE9000D040C854DF4F7881C85BD040C1010E94C8
:10AEA0003A35C153DF4F1881CF5CD040CF53DF4FCD
:10AEB00088819981C15CD040892B09F4C1C8C353F2
:10AEC000DF4FE881F981CD5CD040EF2B09F0C1C89C
:10AED000689440F8C754DF4F8881C95BD040853003
:10AEE00009F457C908F0BCC8833009F4E7C8912CAD
:10AEF0003DC02FEFA2126DCF5ACFC353DF4F8881D1
:10AF00009981CD5CD04010E0892B09F0A2C840E0C7
:10AF100051E060E070E0C1010E94AC19672B682B22
:10AF2000692B09F02DC9BFEFAB121DC9C1010E94E9
:10AF3000D743181619060CF419C9B101CE0187546C
:10AF40009F4F0E94BC9F61E0CE0187549F4F0E949B
:10AF5000002E29AB3AAB4BAB5CAB6DAB7EAB8FAB92
:10AF600098AF689440F854F846E0942ED301C2019B
:10AF7000689440F8C554DF4F2881CB5BD040223025
:10AF800060F4C754DF4F2881C95BD040222329F0E9
:10AF90002C013D01689440F854F8C654DF4F888175
:10AFA000CA5BD0408F7009F41AC9689455F8112310
:10AFB00011F0E89455F8A201B101CE0187549F4FDA
:10AFC0000E94843BA1E0B0E0C953DF4FB983A8835E
:10AFD000C75CD040B110F9CDD1011B968D919C91E9
:10AFE000009709F49ECBDC01ED91FC910488F58972
:10AFF000E02DC754DF4F0881C95BD040C654DF4FF6
:10B000001881CA5BD040C554DF4F2881CB5BD0404C
:10B01000C454DF4F3881CC5BD040C354DF4F4881EC
:10B02000CD5BD040C254DF4F5881CE5BD040C1547D
:10B03000DF4F6881CF5BD040C054DF4F7881C05C68
:10B04000D040199581116DCB6CEE77E08FE59BE0D8
:10B050000E94C8898FE59BE00E94418856FC9ACDEA
:10B0600064EA77E086E09CE00E94C889C953DF4F1C
:10B0700068817981C75CD04086E09CE00E94399F5E
:10B080006DE977E086E09CE00E94C8890E94ABA948
:10B09000AB01BC01CA52DF4F088119812A813B8173
:10B0A000C65DD040401B510B620B730B2AE086E05B
:10B0B0009CE00E94F58786E09CE00E94418854CE87
:10B0C0002F923F924F925F926F927F928F929F92B8
:10B0D000AF92BF92CF92DF92EF92FF920F931F93A6
:10B0E000CF93DF93CDB7DEB7CB57D1090FB6F89426
:10B0F000DEBF0FBECDBFE296EFAEE297E396FFAEA6
:10B10000E397E4960FAFE497E5961FAFE597E696D1
:10B110002FAFE697E7963FAFE797E8964FAFE897F0
:10B12000E9965FAFE997009709F453C024012B2CEF
:10B13000EC96AFAEEC97EB96DFAEEB97EA96CFAE20
:10B14000EA97362E8C0180912A02893020F4809172
:10B1500029028930A0F180E091E00E94E7C97C01DA
:10B16000892B69F11C821B821E821D828FEF9FEF4B
:10B1700098878F8389E992E09A8389831A86198652
:10B18000FC86EB8680E091E0988B8F871E861D867B
:10B19000B801CE0101960E9476A067EC74E086E0CB
:10B1A0009CE00E947189B70186E09CE00E94718951
:10B1B00086E09CE00E944188C7010E9483CAF80192
:10B1C00080858F70843009F45FC128F4882309F4E6
:10B1D00064C180E02FC0853009F446C08630C9F7CD
:10B1E0006AE174E0C8010E94CB9A3C01009709F41F
:10B1F00076C0912C812CB12CA12CD12CC12CE296A3
:10B20000EFACE297E396FFACE397E4960FADE497DB
:10B21000E5961FADE597E6962FADE697E7963FAD2D
:10B22000E797E8964FADE897E9965FADE997632D0C
:10B230000E946058C558DF4F0FB6F894DEBF0FBEAE
:10B24000CDBFDF91CF911F910F91FF90EF90DF90D5
:10B25000CF90BF90AF909F908F907F906F905F90B6
:10B260004F903F902F900895809162078F5F809359
:10B270006207668077806114710459F14201EC968F
:10B28000AFACEC97B22CEA96CFACEA97EB96DFAC7A
:10B29000EB97E296EFACE297E396FFACE397E49688
:10B2A0000FADE497E5961FADE597E6962FADE697CF
:10B2B000E7963FADE797E8964FADE897E9965FAD23
:10B2C000E997632DC3010E946058F3016280738087
:10B2D000D2CF809162078150809362077ACF6DEC64
:10B2E00074E0C8010E94CB9A2C0162ED74E0C801A1
:10B2F0000E94CB9A7C0167ED74E0C8010E94CB9A52
:10B30000332039F0F1E03F1609F49FC0D12CC12C55
:10B310000CC06BED74E0C8010E94CB9A3C0160EE5A
:10B3200074E0C8010E94CB9A6C016114710409F4A5
:10B330003801C114D10409F468014114510431F4F5
:10B34000EA964FACEA97EB965FACEB97E114F10409
:10B3500021F4EC96EFACEC97F22C6114710409F433
:10B36000A5C0F30180858F70843009F09FC061848F
:10B370007284C114D10409F49CC0F60180858F70D9
:10B38000843009F096C0C184D28410E000E04114FA
:10B39000510409F4F3C06114710409F4B1C06CE103
:10B3A0007CE186E09CE00E94C889F201618572859B
:10B3B00086E09CE00E94718967E17CE186E09CE088
:10B3C0000E94C889B30186E09CE00E94718986E0F2
:10B3D0009CE00E944188CE018F589F4F0E94922D81
:10B3E000E114F10409F0D3C0F20180858F7084303C
:10B3F00009F083C1409166075091670761857285A6
:10B40000CE0101960E94FB3CCE0101960E94773B43
:10B410008823B1F00E94CB286B01683C71050CF0C9
:10B4200083C066ED7BE18FE59BE00E94C889B60191
:10B430008FE59BE00E94399F8FE59BE00E94418849
:10B44000CE0101960E94374158C165EE74E0C801F3
:10B450000E94CB9A3C016AEE74E0C8010E94CB9A2C
:10B460006C016114710409F04AC16BED74E0C8010C
:10B470000E94CB9A3C01C114D10409F450CF892B0E
:10B4800009F05BCF380159CFD12CC12C712C612C24
:10B49000F12CE12C512C412C48CFD12CC12C712CFA
:10B4A000612CF12CE12C512C412C47CF712C612CBB
:10B4B00060CF00E020E030E340E150E0BE016F5992
:10B4C0007F4FCE018F589F4F0E94801E6C01E496E3
:10B4D0000FADE49710E00115110509F058CFE29681
:10B4E0008FADE297811109C0E3968FADE3978F701E
:10B4F00009F44DCF02E010E04ACF01E010E047CF61
:10B500006DE07CE186E09CE00E94C889F2016185E3
:10B51000728586E09CE00E94718968E07CE186E0AB
:10B520009CE00E94C88957CF6114710431F0B301C7
:10B53000CE0101960E94C0A183CFA12CC12CF12C79
:10B54000E12CE2960FADE297E3961FADE397E49608
:10B550002FADE497E5963FADE597E6964FADE697BC
:10B56000E7965FADE797E8966FADE897E9967FAD10
:10B57000E997CE0101960E94164662CFE114F104CC
:10B5800009F4BBC0C114D10409F4B7C004C0C1148C
:10B59000D10409F429CFF70180858F70843009F038
:10B5A000A8C08185928525961FAE1EAE259748EED0
:10B5B00053E060E070E029964CAF5DAF6EAF7FAFB7
:10B5C00029972FEA32E023963FAF2EAF23972F968D
:10B5D0009FAF8EAF2F9761961FAE1EAE6197639699
:10B5E0001FAE1EAE639765961FAE1EAE659767963B
:10B5F0001FAE1EAE679769961FAF0EAF69976A962A
:10B600001FAE6A9740E450E0BE016F5F7F4FCE01EE
:10B610008F5B9F4F0E94609C21E030E02C0F3D1F0C
:10B62000820F931FFC01108260E07CE186E09CE0C9
:10B630000E94C889F7016185728586E09CE00E94BE
:10B6400071896FEE74E086E09CE00E947189BE0112
:10B650006F5F7F4F86E09CE00E9471896BEF7BE11A
:10B6600086E09CE00E94C889B60186E09CE00E94CA
:10B67000718986E09CE00E9441880E94E99A8823B3
:10B68000C1F18091CC08811134C06FE270E0CE012D
:10B6900001960E942CD8892B51F4F701218532851F
:10B6A00043E050E060E4CE0101960E94C62764EFBB
:10B6B0007BE186E09CE00E94C889BE016F5F7F4FFE
:10B6C00086E09CE00E9471896FEE7BE186E09CE061
:10B6D0000E94C889B60186E09CE00E94718986E0DC
:10B6E0009CE00E94418841E0B601CE0101960E9493
:10B6F00079AA4114510409F077CE81E09BCD892BC2
:10B7000009F01BCE0CCE8F929F92AF92BF92CF9238
:10B71000DF92EF92FF920F931F93CF93DF9300D0AE
:10B7200000D01F921F92CDB7DEB7E982FA820B8359
:10B730001C832D833E834F835887DC011296ED9145
:10B74000FC91309791F1048115810115110569F182
:10B75000F80180858F70853041F57B01C8010E941A
:10B760008A9F823010F161E0C8010E94439B0097DC
:10B77000E1F0DC0118962C912F702630B1F4B7015E
:10B780000E94CB9A009789F0912C812CB12CA12C8E
:10B79000D12CC12CE980FA800B811C812D813E8146
:10B7A0004F8158856FEF0E94605828960FB6F89425
:10B7B000DEBF0FBECDBFDF91CF911F910F91FF90E4
:10B7C000EF90DF90CF90BF90AF909F908F900895B3
:10B7D0002F923F924F925F927F928F929F92AF9261
:10B7E000BF92CF92DF92EF92FF920F931F93CF936E
:10B7F000DF93CDB7DEB7C75AD1090FB6F894DEBFD5
:10B800000FBECDBFDC0114962D913C911597232BD3
:10B8100009F4CDC55B016C01ED91FC910284F385C7
:10B82000E02D19958230910509F417C1C4F597FFF1
:10B83000BEC5F60187819085DC01ED91FC91008405
:10B84000F185E02D199585970CF4F3C045E250E0A1
:10B85000BE016F5F7F4FF601878190850E94C3878D
:10B86000D60117968D919C91DC01ED91FC9100849D
:10B87000F185E02D1995892B09F436C162E070E05D
:10B8800080E090E00E9479A9F60187819085DC0133
:10B89000ED91FC910284F385E02D1995E1CF843080
:10B8A000910509F473C0BCF1059719F6AA94AB2869
:10B8B00009F0FFC06DE379E186E09CE00E94EC892D
:10B8C0004DE050E062E072E0C6010E940B27D60115
:10B8D0001496AD90BC904FEF5FEFBA0180E00E94EC
:10B8E0008824F50160A771A782A793A7D601ED91DF
:10B8F000FC910484F585E02D62E0C6011995D6011E
:10B900001496ED91FC9115978FEF80831496ED912D
:10B91000FC9181838ECFD6011496ED91FC9180A588
:10B9200091A5A2A5B3A5892B8A2B8B2B09F481CFD6
:10B930000E94ABA9D6011496ED91FC91159700A534
:10B9400011A522A533A5601B710B820B930B6639E1
:10B9500071058105910508F46CCFED91FC9104848B
:10B96000F585E02D62E0C6011995F6010481158187
:10B970004FEF5FEFBA0180E00E948824D8019896CB
:10B980006D937D938D939C939B9753CFD601149683
:10B99000ED91FC9180A591A5A2A5B3A5892B8A2B39
:10B9A0008B2BD9F10E94ABA9D6011496ED91FC9195
:10B9B00000A511A522A533A5601B710B820B930B6B
:10B9C000683873418105910540F1D601ED91FC91F4
:10B9D0000484F585E02D65E0C6011995F601048122
:10B9E00015814FEF5FEFBA0180E00E948824D801F3
:10B9F00098966D937D938D939C939B97D601149607
:10BA0000ED91FC9117A269E479E186E09CE00E9447
:10BA1000C88986E09CE00E944188F6018781908574
:10BA2000DC01ED91FC910084F185E02D1995892BC5
:10BA300019F481E090E03FC062E070E080E090E0C7
:10BA40000E9479A9F60187819085DC01ED91FC9136
:10BA50000284F385E02D1995E0CFD6011496ED917F
:10BA6000FC9180A591A5A2A5B3A5892B8A2B8B2B30
:10BA7000E1F00E94ABA9D6011496ED91FC9100A5CE
:10BA800011A522A533A5601B710B820B930B68389F
:10BA900073418105910548F0D601ED91FC91048434
:10BAA000F585E02D65E0C6011995AA94AB2809F447
:10BAB000C0CE90E080E0C955DF4F0FB6F894DEBFEE
:10BAC0000FBECDBFDF91CF911F910F91FF90EF90EF
:10BAD000DF90CF90BF90AF909F908F907F905F90BE
:10BAE0004F903F902F90089569E379E186E09CE0C4
:10BAF0000E94C8894AE050E0F601668186E09CE039
:10BB00000E94458864E379E186E09CE00E94C88950
:10BB1000CE0101965C014E0195E2890E911CD50182
:10BB20006D915D0140E150E06A3058F468E474E0E2
:10BB300086E09CE00E94718940E150E0F501319778
:10BB4000608186E09CE00E9445888A149B0439F756
:10BB50006EE286E09CE00E94E08886E09CE00E9425
:10BB60004188FE01339680E0AE16BF0619F0919130
:10BB7000890FFACF9DA198130FC46DE279E186E099
:10BB80009CE00E94C88986E09CE00E9441888DA1CB
:10BB9000D6011496ED91FC91159797A1891709F498
:10BBA00048CF87A314960D90BC91A02D85E2FE018D
:10BBB000319601900D928A95E1F7D6011496ED9198
:10BBC000FC91C056DF4F188219821A821B82C05A1C
:10BBD000D040CC55DF4F188219821A821B82C45A7A
:10BBE000D040CF55DF4F8881C15AD040807FCF559C
:10BBF000DF4F8883C15AD04083A190E01C01B0E19F
:10BC00002B0E311C499708F014CF7584878986A3C1
:10BC1000118D538CD60114962D913C91858DD901AF
:10BC200095968C93848C912C878DD6011296ED91EC
:10BC3000FC910280F381E02D42EF54E06EE974E064
:10BC400080FD02C06EE874E0808191810E9497AA15
:10BC5000B0E88B16910409F086C0D6011296ED91DA
:10BC6000FC910280F381E02D49EF54E06EE974E02D
:10BC7000808191810E9497AA6FEF74E086E09CE03A
:10BC80000E947189D6011496ED91FC914AE050E032
:10BC900065A186E09CE00E94458886E09CE00E94C9
:10BCA0004188D6011496ED91FC91159785A11296C5
:10BCB000ED91FC910280F381E02D4AE055E06EE9C0
:10BCC00074E083FD02C06EE874E0808191810E947F
:10BCD00097AAD6011296ED91FC9113970280F381F9
:10BCE000E02D808191811496ED91FC9125A141E197
:10BCF00055E06EE974E021FD02C06EE874E00E9438
:10BD000097AA1EA2113009F4F4C1E0F1123009F42F
:10BD100025C2133009F457C26DE179E1CE01869650
:10BD20000E9429CC60E0CE0180569F4F0E94002ED9
:10BD3000E9962FAFE997EA963FAFEA97EB964FAFB8
:10BD4000EB97EC965FAFEC97ED966FAFED97EE96B5
:10BD50007FAFEE97EF968FAFEF97C158DF4F988385
:10BD6000CF57D04043C0892809F086CFD60112961C
:10BD7000ED91FC910280F381E02D49EF54E06EE8F3
:10BD800074E076CF64EF79E1CE0186960E9429CCEB
:10BD900060E1CE0180569F4F0E94002EC856DF4FB3
:10BDA0002883C859D040C756DF4F3883C959D0407F
:10BDB000C656DF4F4883CA59D040C556DF4F588317
:10BDC000CB59D040C456DF4F6883CC59D040C356BE
:10BDD000DF4F7883CD59D040C256DF4F8883CE598C
:10BDE000D040C156DF4F9883CF59D040D60112962C
:10BDF000ED91FC910280F381E02D42E954E0BE0117
:10BE00006A5D7F4F808191810E9497AAC056DF4F63
:10BE1000E880C05AD040CF55DF4FF880C15AD0409B
:10BE2000CE55DF4F0881C25AD040CD55DF4F188123
:10BE3000C35AD040CC55DF4F2881C45AD040CB558F
:10BE4000DF4F3881C55AD040CA55DF4F4881C65AA6
:10BE5000D040C955DF4F5881C75AD04063E974E0DC
:10BE6000C6010E94835BD6011296ED91FC9102807F
:10BE7000F381E02D47E954E06EE874E0552011F0BD
:10BE80006EE974E0808191810E9497AA032C000CD6
:10BE900044085508D6011296ED91FC910280F38179
:10BEA000E02D6081718104E814E0A2019101C601D6
:10BEB0000E944A21872C912CB12CA12CBFEF7B161C
:10BEC00081F0D6011296ED91FC910280F381E02D74
:10BED000608171810DE115E0A5019401C6010E9408
:10BEE0004A2118AA19AA1AAA1BAA89A9807F8A60BE
:10BEF00089AB88A939A92AA99BA9E82EE1968FAF19
:10BF0000E197E2963FAFE297E3962FAFE397E4968F
:10BF10009FAFE497222DE8962CAE3DAE4EAE5FAEBD
:10BF2000E897F32EE3960FADE397192FE6963FAD12
:10BF3000E697E7964FADE797E8965FADE89765E837
:10BF400074E0C6010E94835B18AA19AA1AAA1BAA48
:10BF500089A9807F8A6089AB88A999A9AAA9BBA968
:10BF600088AF99AFAAAFBBAF8CAE9DAEAEAEBFAE41
:10BF700063E0CE01C8960E94DE2DA9962FAFA99747
:10BF8000AA963FAFAA97AB964FAFAB97AC965FAF71
:10BF9000AC97AD966FAFAD97AE967FAFAE97AF96BD
:10BFA0008FAFAF97E0969FAFE09779018A019B0131
:10BFB000AC016EE175E0C6010E94835B1EA2D60152
:10BFC0001496ED91FC9186A1811132C160EE79E168
:10BFD000CE0186960E9429CC6EE0CE0180569F4FFE
:10BFE0000E94002EA1962FAFA197A2963FAFA297D5
:10BFF000A3964FAFA397A4965FAFA497A5966FAFF4
:10C00000A597A6967FAFA697A7968FAFA797A89656
:10C010009FAFA897D6011496ED91FC91159726A194
:10C0200030E050E040E01296ED91FC910280F38107
:10C03000E02D6081718103E215E0C6010E944A2172
:10C04000D6011496ED91FC9185A180FD14C068E69F
:10C0500079E1CE0186960E9429CC62E0CE0180561D
:10C060009F4F0E94002E28AB39AB4AAB5BAB6CAB49
:10C070007DAB8EAB9FABD6011296ED91FC91028009
:10C08000F381E02D49E854E0BE016A5D7F4F808175
:10C0900091810E9497AAC056DF4FE880C05AD040D5
:10C0A000CF55DF4FF880C15AD040CE55DF4F0881C1
:10C0B000C25AD040CD55DF4F1881C35AD040CC551D
:10C0C000DF4F2881C45AD040CB55DF4F3881C55A45
:10C0D000D040CA55DF4F4881C65AD040C955DF4FBE
:10C0E0005881C75AD0406AE874E0C6010E94835B59
:10C0F000A0CC6EEF79E1CE0186960E9429CC61E159
:10C10000CE0180569F4F0E94002EC057DF4F2883DC
:10C11000C059D040CF56DF4F3883C159D040CE569A
:10C12000DF4F4883C259D040CD56DF4F5883C359A3
:10C13000D040CC56DF4F6883C459D040CB56DF4F38
:10C140007883C559D040CA56DF4F8883C659D0403E
:10C15000C956DF4F9883C759D04048CE68E07AE18E
:10C16000CE0186960E9429CC62E1CE0180569F4F77
:10C170000E94002EC857DF4F2883C858D040C757A9
:10C18000DF4F3883C958D040C657DF4F4883CA585D
:10C19000D040C557DF4F5883CB58D040C457DF4FEE
:10C1A0006883CC58D040C357DF4F7883CD58D040F8
:10C1B000C257DF4F8883CE58D040C157DF4F988396
:10C1C000CF58D04013CE60EE79E1CE0186960E9422
:10C1D00029CC6EE0CE0180569F4F0E94002EC058A1
:10C1E000DF4F2883C058D040CF57DF4F3883C15826
:10C1F000D040CE57DF4F4883C258D040CD57DF4F95
:10C200005883C358D040CC57DF4F6883C458D040C0
:10C21000CB57DF4F7883C558D040CA57DF4F88834C
:10C22000C658D040C957DF4F9883C758D040DECD9D
:10C23000813029F566E27AE1CE0186960E9429CC0A
:10C2400065E1CE0180569F4F0E94002E69962FAF68
:10C2500069976A963FAF6A976B964FAF6B976C96EC
:10C260005FAF6C976D966FAF6D976E967FAF6E9761
:10C270006F968FAF6F97A0969FAFA097CBCE82306F
:10C2800029F56CE17AE1CE0186960E9429CC64E121
:10C29000CE0180569F4F0E94002E61962FAF61976E
:10C2A00062963FAF629763964FAF639764965FAFB6
:10C2B000649765966FAF659766967FAF669767964A
:10C2C0008FAF679768969FAF6897A4CE833029F5A4
:10C2D0006AEE79E1CE0186960E9429CC6FE0CE010C
:10C2E00080569F4F0E94002E29962FAF29972A969D
:10C2F0003FAF2A972B964FAF2B972C965FAF2C977B
:10C300002D966FAF2D972E967FAF2E972F968FAFCE
:10C310002F9760969FAF60977DCE843029F560E3BC
:10C320007AE1CE0186960E9429CC66E1CE01805644
:10C330009F4F0E94002E21962FAF219722963FAF4C
:10C34000229723964FAF239724965FAF2497259685
:10C350006FAF259726967FAF269727968FAF2797A3
:10C3600028969FAF289756CE8D3609F053CE6DE1B3
:10C3700079E1CE0186960E9429CC60E0CE018056FC
:10C380009F4F0E94002E28AF39AF4AAF5BAF6CAF12
:10C390007DAF8EAF9FAF3ECE61E279E186E09CE05B
:10C3A0000E94C88986E09CE00E94418842CB8FEFC2
:10C3B0009FEF81CB2F923F924F925F926F927F922D
:10C3C0008F929F92AF92BF92CF92DF92EF92FF92A5
:10C3D0000F931F93CF93DF93CDB7DEB767970FB659
:10C3E000F894DEBF0FBECDBF1C017C8B6B8B40E091
:10C3F00050E860E070E00E94AC19672B682B692B55
:10C4000009F45DC019821A821B821C821D821E8261
:10C410001F8218868A81807F8A8340E050E3B101C1
:10C42000CE0101960E940240D1011B968D919C91F4
:10C43000892B09F444C040E050E860E070E0C1019D
:10C440000E945A1969EE7AE086E09CE00E94C88951
:10C45000F10183859485DC01ED91FC910088F189DF
:10C46000E02DA12CCC24C394F12CE12C09811A815C
:10C470002B813C814D815E816F81788519958F3F3D
:10C480009807E9F0D1011296ED91FC9160817181DC
:10C49000892B09F0C5C086E09CE00E94718967EE97
:10C4A0007AE086E09CE00E94C8896FED7AE086E041
:10C4B0009CE00E94C88986E09CE00E94418865E07B
:10C4C000F101828193810E94439B9A8B898B009713
:10C4D00009F4DAC0DC011896BC91BD8B9B2E9294B6
:10C4E0003FE09322FC0141845284638474840E945F
:10C4F000ABA9992009F4C8C0461A570A680A790AF4
:10C5000019861A861B861C8699861A85107F1A60E2
:10C510001A874D865E866F86788A8B899C890497F8
:10C5200069F588248394B12CA12CC12CD12C20E155
:10C53000E22EF12C092D2B853C854D855E856F857E
:10C540007889C1010E94222EC301B20128EE33E096
:10C5500040E050E00E9481D3BA01A9012AE030E016
:10C5600086E09CE00E94E78860E17BE086E09CE05A
:10C570000E94C88986E09CE00E94418877FE84C0C2
:10C5800092E049165104610490E879060CF47CC0ED
:10C590000E94CB282B017F8B6E8B88248394B12C37
:10C5A000A12CC12CD12C90E1E92EF12C09851A8502
:10C5B0002B853C854D855E856F857889C1010E94FC
:10C5C000222EAE89BF89A83CB105BCF567EF7AE0A1
:10C5D0008FE59BE00E94C889B2018FE59BE00E9435
:10C5E000399F8FE59BE00E9441888FEF9FEF679610
:10C5F0000FB6F894DEBF0FBECDBFDF91CF911F9174
:10C600000F91FF90EF90DF90CF90BF90AF909F90F1
:10C610008F907F906F905F904F903F902F900895F4
:10C6200086E09CE00E9471896DED7AE086E09CE0F6
:10C630000E94C88969ED7AE03ACFE989FA89808554
:10C640008F70808719821A821B821C821D821E8233
:10C650001F8218868A81807F8A8399828D898F7054
:10C66000AA24A394873009F0A12C82E0C82EF12CD3
:10C67000E12C09811A812B813C814D815E816F8182
:10C680007885C1010E9416468B899C89019701F526
:10C6900040E050E360E070E0C1010E94AC19AB01E2
:10C6A000BC01411551056105710591F08091CD08DE
:10C6B0009091CE08069761F430E020E0C1010E941D
:10C6C0007E4040E050E360E070E0C1010E945A19F2
:10C6D000D1011B968D919C91009719F490E080E018
:10C6E00086CFDC01ED91FC910284F385E02D199554
:10C6F000892BA1F3F10183859485DC01ED91FC91F7
:10C700000480F581E02D6B897C89199570CF6F923B
:10C710007F928F929F92AF92BF92CF92DF92EF92D1
:10C72000FF920F931F93CF93DF93CDB7DEB7C8541B
:10C73000D1090FB6F894DEBF0FBECDBF3C014B014F
:10C74000FC01008111816DEC74E0C8010E94CB9A5C
:10C750005C0162ED74E0C8010E94CB9A6C0167ED48
:10C7600074E0C8010E94CB9AA114B10431F4C11441
:10C77000D10419F4892B09F4D0C069E275E0C8012D
:10C780000E94CB9A7C016EE275E0C8010E94CB9AB0
:10C790008C016BE477E086E09CE00E94C8894AE067
:10C7A00050E0F301638186E09CE00E94458869E4E3
:10C7B00077E086E09CE00E94C889B40186E09CE0B6
:10C7C0000E94399F86E09CE00E944188C114D104F8
:10C7D00009F455C0F60180858F70843009F04FC090
:10C7E0006185728540E450E0CE0101960E9465D8D3
:10C7F0000E94E99A882309F442C08091CC088111F3
:10C800003EC06FE270E0CE0101960E942CD8892BC9
:10C8100051F4F6012185328543E050E060E4CE0119
:10C8200001960E94C6278114910409F4B5C0E11451
:10C83000F10409F088C041E06EE974E0CE01019690
:10C840000E9479AA63E477E086E09CE00E94C889B0
:10C85000BE016F5F7F4F86E09CE00E94718960E4BB
:10C8600077E086E09CE00E94C8896EE974E086E08B
:10C870009CE00E94718986E09CE00E944188A1149E
:10C88000B10409F44AC0F50180858F70843009F045
:10C8900044C0409166075091670761857285CE015B
:10C8A00001960E94FB3CCE0101960E94773B8823B3
:10C8B00081F1892809F4B7C0F701EF2809F0CCC04D
:10C8C00025961CAE1DAE1EAE1FAE259729961CAE3A
:10C8D0001DAE1EAE1FAE299723961FAD2397107F66
:10C8E000A12CC12CF12CE12C01E024962FAD249732
:10C8F00025963FAD259740E027965FAD2797289670
:10C900006FAD289729967FAD2997CE0101960E9499
:10C910001646CE0101960E943741C85BDF4F0FB625
:10C92000F894DEBF0FBECDBFDF91CF911F910F9165
:10C93000FF90EF90DF90CF90BF90AF909F908F903F
:10C940007F906F900895F70180858F70843009F093
:10C9500096CF61857285FB018081882309F48FCF92
:10C9600041E0CE0101960E9479AA6AE377E086E071
:10C970009CE00E94C889BE016F5F7F4F86E09CE00B
:10C980000E94718967E377E086E09CE00E94C88995
:10C99000F701618572856BCF01151105E9F441E05E
:10C9A0006EE874E0CE0101960E9479AA61E377E017
:10C9B00086E09CE00E94C889BE016F5F7F4F86E0E1
:10C9C0009CE00E9471896EE277E086E09CE00E9424
:10C9D000C8896EE874E04BCFF80180858F70843091
:10C9E00009F04DCF61857285FB018081882309F4B0
:10C9F00046CF41E0CE0101960E9479AA68E277E035
:10CA000086E09CE00E94C889BE016F5F7F4F86E090
:10CA10009CE00E94718965E277E086E09CE00E94DC
:10CA2000C889F801B6CFF801012BB1F425961CAEE8
:10CA30001DAE1EAE1FAE259729961CAE1DAE1EAEB6
:10CA40001FAE299723961FAD2397107FA12CC12CD1
:10CA5000F12CE12C02E049CF80858F70843009F001
:10CA600058CF61857285FB018081882309F451CFFD
:10CA7000CE0101960E94C0A14CCFEF92FF920F937E
:10CA80001F93CF93DF93EC018B011E821D821A82CC
:10CA90001B821C82E880F980E114F10459F1809135
:10CAA000AC069091AD06892B29F1672B09F487011B
:10CAB000F80180858F708630E9F463E375E0C80182
:10CAC0000E94CB9A009719F0FC0181858A836CE55E
:10CAD00076E0C8010E94CB9AFC01892B61F1808528
:10CAE0008F70823071F0853079F0F9E0EF0EF11C33
:10CAF000FE82ED82DF91CF911F910F91FF90EF9019
:10CB0000089581858B83F1CF0680F781E02D3097E2
:10CB100061F380858F70823041F781858B83068039
:10CB2000F781E02D309709F380858F708230E9F628
:10CB300081858C83DACFF801808191810E94B4CB0A
:10CB4000E1CF0F931F93CF93DF93CDB7DEB76F97EE
:10CB50000FB6F894DEBF0FBECDBF2091AC0630916A
:10CB6000AD06232B09F409C120916207022E000CA7
:10CB7000330B82179307B4F461E97EE08FE59BE005
:10CB80000E94C8898FE59BE00E94418880E06F96F3
:10CB90000FB6F894DEBF0FBECDBFDF91CF911F91CE
:10CBA0000F9108956BE77EE086E09CE00E94C889C3
:10CBB00086E09CE00E9441888091A1068F5F80936F
:10CBC000A10666E37EE085E59BE00E94C88985E5D5
:10CBD0009BE00E944188E0916407F09165073097DF
:10CBE00009F1809162078F5F809362070681178148
:10CBF0000115110591F0D80118968C918F7086302F
:10CC000041F41A83098370E060E0CE0101960E942E
:10CC10003D65F80102811381EBCF8091620781505D
:10CC200080936207E0916607F09167073097A1F162
:10CC30000681178101151105C9F1D80118968C914B
:10CC40008F70853029F5C8010E948A9F882301F1E1
:10CC50004091660750916707F80160817181CE01AC
:10CC600001960E94FB3CCE0101960E94773B8823EF
:10CC700059F08C859D85009739F0DC01ED91FC9190
:10CC80000084F185E02D1995CE0101960E9437416F
:10CC9000F80102811381CECF6BE67EE086E09CE056
:10CCA0000E94C88986E09CE00E944188109261073A
:10CCB0001092600763E67EE086E09CE00E94C889EF
:10CCC00086E09CE00E94418864E670E080E090E0AD
:10CCD0000E9479A91092090710925F076BE47EE029
:10CCE00086E09CE00E94C8890E94CB28AB01BC0171
:10CCF0002AE086E09CE00E94F5878091AC06909146
:10CD0000AD06009711F00E94CFA41092AD061092CC
:10CD1000AC06109265071092640710926707109294
:10CD2000660710920B0710920A071092A306109242
:10CD3000A20610925D0710925C0710925B0710929A
:10CD40005A071092590766E47EE086E09CE00E9454
:10CD5000C8890E94CB28AB01BC012AE086E09CE098
:10CD60000E94F58786E09CE00E94418810925E0751
:10CD70008091A10681508093A10681E008CF2F9277
:10CD80003F924F925F927F928F929F92AF92BF920B
:10CD9000CF92DF92EF92FF920F931F93CF93DF9387
:10CDA000CDB7DEB7A9970FB6F894DEBF0FBECDBFE3
:10CDB0006C01F62E1A014901DC018D919C911197AD
:10CDC000892B09F4D2C01596ED91FC91309709F4A6
:10CDD000CCC080818071BFEF6B13C9C0C9F481E002
:10CDE000A9960FB6F894DEBF0FBECDBFDF91CF91ED
:10CDF0001F910F91FF90EF90DF90CF90BF90AF9079
:10CE00009F908F907F905F904F903F902F900895CC
:10CE10004330510521F3F180F2942FE0F2226BE1CF
:10CE200077E086E09CE00E94C8894AE050E0D601A5
:10CE300013966C9186E09CE00E94458869E177E05A
:10CE400086E09CE00E94C889D6011596ED91FC9180
:10CE500061816F704AE050E086E09CE00E94458866
:10CE600066E177E086E09CE00E94C8894AE050E0F5
:10CE70006F2D86E09CE00E94458886E09CE00E9441
:10CE80004188D6011596ED91FC9181818F70F8163D
:10CE900009F468C0008103FB002700F9198E1A8E7F
:10CEA0001B8E1C8E1D8E1E8E1F8E18A28A8D807F5B
:10CEB0008A8FD6011596ED91FC9181818F708F1527
:10CEC000A9F1B3E02B16310489F164E177E086E043
:10CED0009CE00E94C8894AE050E0F601638186E048
:10CEE0009CE00E94458862E177E086E09CE00E9439
:10CEF000C889D6011596ED91FC9161816F704AE069
:10CF000050E086E09CE00E9445886FE077E086E094
:10CF10009CE00E94C8894AE050E06F2D86E09CE0CA
:10CF20000E94458886E09CE00E944188BFE0BF15D2
:10CF300008F455C1EF2DF0E08827EE55F8498F4FE2
:10CF40000C94D6D3BB67FB674768B268BD68476877
:10CF500020684768C068CC683468CF68DA68EF68D2
:10CF6000EF68DD6880818F7E808380E039CF882301
:10CF700009F494CFFACFF601A580B680D5011196B9
:10CF80008C918F70853009F42AC168F48230D9F011
:10CF90006EE275E0C4010E94CB9A2C01712CEE2048
:10CFA00009F491C0A7C08730D1F08A3089F76CE3CB
:10CFB00075E0C4010E94CB9A2C01F501708072FAD1
:10CFC000772470F8ECCF66E375E0C4010E94CB9A39
:10CFD0002C01F501708070FA772470F8E0CF65E3DA
:10CFE00075E0C4010E94CB9A2C01D5017C9071FAA6
:10CFF000772470F8D4CF69E275E0C4010E94CB9A1F
:10D000002C01D6011596ED91FC91808180FB77244F
:10D0100070F8982F9E7F80FF916090834114510497
:10D0200009F0BDCF61E0CE0149960E94002E298B08
:10D030003A8B4B8B5C8B6D8B7E8B8F8B988FAFCFAE
:10D0400063E475E0C4010E94CB9A2C01D6011596C9
:10D05000ED91FC91808181FB772470F8982F9D7F62
:10D0600081FF926090839BCF69E475E0C4010E94C8
:10D07000CB9A2C01D6011596ED91FC91808182FB13
:10D08000772470F8982F9B7F82FF9460EBCF6EE23D
:10D0900075E0C4010E94CB9A2C01892B69F462E0EF
:10D0A000CE0149960E94002E29873A874B875C87DC
:10D0B0006D877E878F87988BEE2009F48EC0BFE046
:10D0C000712CFB1217C0E3E02E16310409F48AC05C
:10D0D000602F70E0C6010E948763D6011596ED911E
:10D0E000FC9180818F7E8083BFE0FB1203C0EE2025
:10D0F00009F475CE6DEC74E0C4010E94CB9A8C01EA
:10D1000062ED74E0C4010E94CB9A5C0167ED74E0AB
:10D11000C4010E94CB9A99A788A7A114B10481F4F5
:10D120000115110569F460E0CE0149960E94002EB8
:10D1300029833A834B835C836D837E838F839887B7
:10D14000D6011596ED91FC914114510409F05BC094
:10D15000898D811158C0BFE0FB126AC080818F7E2B
:10D1600080833DCE6FE475E0C4010E94CB9A2C0110
:10D17000D6011596ED91FC912DCF64E575E0F4CFC5
:10D180006AE575E0C4010E94CB9A2C01D601159680
:10D19000ED91FC9170802BCF60E675E0F3CF67E6F0
:10D1A00075E0C4010E94CB9A2C01D6011596ED9131
:10D1B000FC9104CF6DE675E0F4CF712C512C412C1D
:10D1C000EE2009F480CF69E275E0011102C06EE241
:10D1D00075E0C4010E94CB9A2C01712C74CF512CA4
:10D1E000412C6ACFD6011596ED91FC91808180612A
:10D1F00000FB83F9808381818F709F2D9295907FB2
:10D20000892B818371CF83E028163104C9F4818191
:10D210008F708F1509F4E3CD9FE0F91609F4DFCD87
:10D22000F29490EFF9228F2981838081806198CFD9
:10D230009F2D9F70F92E8181807FF82AF1828ECFF9
:10D24000AFE0FA1639F0BF2DBF70FB2E8181807FD1
:10D25000F82AF18280818F7E808364E775E0C201C5
:10D260000E94CB9A4C01009709F452C0FC018085C2
:10D270008F70843029F0853031F0823009F048C059
:10D28000B401C60143C070E060E0C4010E94722492
:10D290006C010097E9F1BC018091640790916507EA
:10D2A0000E94CB9A9AA389A370E060E0CE01819698
:10D2B0000E943D656DE775E086E09CE00E94718903
:10D2C000B60186E09CE00E94718962E875E086E024
:10D2D0009CE00E94718961E070E08EA19FA1892B82
:10D2E00011F470E060E086E09CE00E94399F86E0E7
:10D2F0009CE00E9441888EA19FA1892B49F061E0AA
:10D30000C4010E94439BBC01CE0181960E94881AF1
:10D3100088A499A46801E98CFA8C0B8D1C8D2D8D45
:10D320003E8D4F8D58A1672DC2010E94605857CD88
:10D330002F923F924F925F926F927F928F929F9225
:10D34000AF92BF92CF92DF92EF92FF920F931F9313
:10D35000CF93DF93CDB7DEB7CB56D1090FB6F89494
:10D36000DEBF0FBECDBFDC0115962D913C91232B66
:10D3700009F4EEC59B01225031092230310508F035
:10D380007BC05B013C01FC018281803409F472C3E3
:10D3900008F069C0843008F06FC0873009F46CC0B1
:10D3A0008091A0068F5F8093A006D301CD90DC9082
:10D3B000C114D10491F06AE174E0C6010E94CB9AD5
:10D3C000FC01892B51F090859F709550923028F484
:10D3D00081859285009709F06C01E12C00E09601AF
:10D3E000A5016FEFC3010E94BF66F301828181FB3B
:10D3F000002700F913819AEC910F903118F08730D3
:10D4000009F04AC067E875E0D3018D919C910E94B4
:10D41000CB9A4C01009709F43FC0FC0180858F70C6
:10D420008530D1F58091730C181329C08091740C4C
:10D43000803429F58091750C9091760C1C01990F20
:10D440004408550860E0C4010E94439BFC018185AB
:10D450009285A385B485281639064A065B060CF02A
:10D4600069C010E042C0823409F404C328F090E897
:10D47000980F943008F491CF90E080E06BC5109342
:10D48000730C80E48093740C812F0E9434A99093D4
:10D49000760C8093750CD2CF212F30E0F901E85E35
:10D4A000FD4D8491F901EE53FE4D1491F901E459BB
:10D4B000FE4DF490FF2009F43AC081110E9463A848
:10D4C000EF2DF0E0EE0FFF1FE552F94FA591B4915B
:10D4D000EC911E2331E020E009F430E0832F922FFD
:10D4E00011E00817190609F0BCCFF3E0AF16B1043C
:10D4F00009F4A6C0D3011596ED91FC91E181EF707E
:10D50000E150EC3008F09CC0F0E08827E557F54981
:10D510008F4F0C94D6D3AB6A386CDF6A096B386CCA
:10D52000556B386C886BA86BC16BFF6B1F6C90E000
:10D5300080E0D6CF61E0C4010E94439B11E0FC0172
:10D5400081859285A385B48582159305A405B505CB
:10D550000CF0CBCF86CF0E94ABA9DC01CB01AA2770
:10D56000BB27F30125813681F90122813381821B9A
:10D57000930BA109B109AA27BB27883E9340A105B7
:10D58000B10508F45DC06FE475E0D3018D919C9105
:10D590000E94CB9AEE24E394012F892B41F464E599
:10D5A00075E0C6010E94CB9A892B09F4ACC09601A4
:10D5B00042E050E063E0C3010E94BF6641C00E94A8
:10D5C000ABA9DC01CB01AA27BB27F301258136815A
:10D5D000F90122813381821B930BA109B109AA278A
:10D5E000BB278C329140A105B10550F1EE24E394A4
:10D5F000012F960142E050E064E0C3010E94BF6643
:10D600000E94ABA9D3011596ED91FC9173836283BF
:10D6100017C00E94ABA9DC01CB01AA27BB27F301ED
:10D6200025813681F90122813381821B930BA10967
:10D63000B109AA27BB2786399105A105B105B0F626
:10D64000D3011596ED91FC91808183FB882780F9A9
:10D65000181709F42DC1D3011596ED91FC91808125
:10D66000982F907E09F06CC10E94ABA9F301A581AF
:10D67000B68113967C936E9312971196EC91119745
:10D68000EF70112309F4A2C1E23009F46AC108F075
:10D690005DC1EE2309F494C1EC90E3FAEE24E0F8C6
:10D6A00001E09601A5016FE07DC10E94ABA9DC01FC
:10D6B000CB01AA27BB27F30125813681F9012281FD
:10D6C0003381821B930BA109B109AA27BB27883E8E
:10D6D0009340A105B10508F4B3CF6AE575E0C60132
:10D6E0000E94CB9AEE24E394012F892B39F460E653
:10D6F00075E0C6010E94CB9A892B29F0960142E081
:10D7000050E068E058CF960142E050E06DE053CF22
:10D710000E94ABA9DC01CB01AA27BB27F30125811D
:10D720003681F90122813381821B930BA109B10952
:10D73000AA27BB278C329140A105B10508F480CF00
:10D74000EE24E394012F960142E050E069E055CFCA
:10D750000E94ABA9DC01CB01AA27BB27F3012581DD
:10D760003681F90122813381821B930BA109B10912
:10D77000AA27BB2786399105A105B10508F460CF1A
:10D78000DFCF0E94ABA9DC01CB01AA27BB27F301A5
:10D7900025813681F90122813381821B930BA109F6
:10D7A000B109AA27BB27883E9340A105B10508F41B
:10D7B00047CF67E675E0C6010E94CB9A892B39F402
:10D7C0006DE675E0C6010E94CB9A892B41F0EE24EC
:10D7D000E394012F960142E050E06BE0ECCE69E467
:10D7E00075E0C6010E94CB9AEE24E394012F9601C6
:10D7F00042E050E066E0892B09F088CFDCCE0E9441
:10D80000ABA9DC01CB01AA27BB27F3012581368117
:10D81000F90122813381821B930BA109B109AA2747
:10D82000BB278C329140A105B10508F409CFEE2445
:10D83000E394012F960142E050E06CE0DECE0E94BE
:10D84000ABA9DC01CB01AA27BB27F30125813681D7
:10D85000F90122813381821B930BA109B109AA2707
:10D86000BB2786399105A105B10508F4E9CEDFCFC4
:10D870000E94ABA9DC01CB01AA27BB27F3012581BC
:10D880003681F90122813381821B930BA109B109F1
:10D89000AA27BB2788359240A105B10508F4D0CE50
:10D8A000EE24E394012F960142E050E060E083CE45
:10D8B0000E94ABA9F30185809680DC01CB01AA27E9
:10D8C000BB27F40122813381821B930BA109B1098B
:10D8D000AA27BB2780339547A105B105F8F0C114ED
:10D8E000D104E1F0D60118968C918F708630B1F496
:10D8F0006BE875E0C6010E94CB9AFC01892B71F0A0
:10D9000080858F70823009F03FC361857285838581
:10D910009485672B682B692B09F09DCEF4018081DB
:10D920008F71806480838091A00681508093A006CF
:10D93000A3CD61857285838594850E94D3D4E9CF78
:10D94000982F907E90528F71892BECCFE53049F063
:10D95000E73009F0A1CEE12C01E09601A5016AE0D3
:10D9600021C063E475E0C6010E94CB9A892BA9F41B
:10D970006AE575E0C6010E94CB9A892B71F460E6D6
:10D9800075E0C6010E94CB9A892B39F465E375E0F6
:10D99000C6010E94CB9A892B99F0E12C01E09601F7
:10D9A000A50166E0C3010E94BF66882309F4BBCFCE
:10D9B000D3011596ED91FC91808110FB83F9B2CFD4
:10D9C000E12C01E09601A50161E0ECCFE150ED30E2
:10D9D00008F048C0F0E08827EF50F3498F4F0C94CF
:10D9E000D6D3FE6C326D046D046D326D0A6D326DEE
:10D9F0002C6D2C6D2C6D2C6D2C6D046DE12C00E0CC
:10DA00009601A50162E0CECFE12C00E09601A501D0
:10DA100065E0C8CF63E475E0C6010E94CB9A892B0C
:10DA2000A9F46AE575E0C6010E94CB9A892B71F4CE
:10DA300060E675E0C6010E94CB9A892B39F465E354
:10DA400075E0C6010E94CB9A892B31F0E12C00E0F1
:10DA50009601A50167E0A6CFE12C00E09601A501A3
:10DA600060E0A0CFEC90E3FAEE24E0F881E0E82655
:10DA700000E017CEB3E0AB16B10409F4FDCC67E8C3
:10DA800075E0F301808191810E94CB9A8C01D301D2
:10DA900013968C919091730C8913DFC09091740C44
:10DAA000903409F0DAC08091750C9091760C2C01BD
:10DAB0000115110509F400C1F80120852F702530EA
:10DAC00009F0FAC0C8010E948A9FA2968FAFA29760
:10DAD000843008F4CEC063E0C8010E94439BDC019F
:10DAE00019968D919C914AE0E42EE89E1001E99EE2
:10DAF000300C112462E0C8010E94439BFC01818527
:10DB00009285E89E6001E99ED00C1124AC96DFAEB0
:10DB1000CEAEAC974601DD0CAA08BB0861E0C80197
:10DB20000E94439B7C0160E0C8010E94439BDC0192
:10DB300019962D913D914D915C911C97A6962CAF15
:10DB40003DAF4EAF5FAFA6979201052C000C440B82
:10DB5000550BA6968CAD9DADAEADBFADA697281B5F
:10DB6000390B4A0B5B0BB101032C000C880B990B92
:10DB7000681979098A099B090E944FD3D701199620
:10DB80002D913D914D915C911C97A696CCACDDAC4E
:10DB9000EEACFFACA6972C193D094E095F09A6967D
:10DBA0002CAF3DAF4EAF5FAFA6970E9481D3820EE0
:10DBB000931EA41EB51EA2962FADA297253009F480
:10DBC0006AC081E090E0A101032C000C660B770B8A
:10DBD000481559056A057B050CF466C0B501A4011A
:10DBE000AC96CEACDFACAC974601DD0CAA08BB0806
:10DBF000481559056A057B050CF45BC04A015B01B9
:10DC0000A2962FADA297223009F069C06201550C8F
:10DC1000EE08FF0860E0C8010E94439BFC0181857B
:10DC20009285A385B485C816D906EA06FB060CF4CE
:10DC3000B8C161E0C8010E94439BFC0181859285C7
:10DC4000A385B4858C159D05AE05BF050CF014CCDD
:10DC5000C12CD12C7601C394A7C18093730C90E49E
:10DC60009093740C0E9434A99093760C8093750C59
:10DC70001ECF8AE0849D4001859D900C1124092CC3
:10DC8000000CAA08BB08AC961FAE1EAEAC97212CA8
:10DC900038E2332E96CF64E0C8010E94439BDC013A
:10DCA00019968D919C918FCF44244A9423E0522E53
:10DCB00097CF512C412CA4CF2AE0289F4001299FC7
:10DCC000900C1124092C000CAA08BB08AC961FAEBE
:10DCD0001EAEAC97212C98E2392E81E090E0D30162
:10DCE0001596ED91FC9162817381A201461B570B41
:10DCF00057FF03C05195419551098417950774F05A
:10DD00008081982F929596959770963050F49F5FEA
:10DD10009295990F907E8F71892B02C080818F71AF
:10DD200080838081803AB8F0AC96EEADFFADAC97C1
:10DD30006F01FF0FEE08FF088C149D04AE04BF04B2
:10DD400051F0C101330CAA0BBB0B88169906AA0629
:10DD5000BB0609F091CB6415750509F48DCB6D9662
:10DD60001CAE1DAE1EAE1FAE6D976B968FAD6B9742
:10DD7000807F86606B968FAF6B976D968CAD9DADF7
:10DD8000AEADBFAD6D9765968CAF9DAFAEAFBFAF7B
:10DD90006597AAE0B0E0A50194010E94A0D369961E
:10DDA0006CAF7DAF8EAF9FAF699767ED76E086E091
:10DDB0009CE00E94C8894AE050E0D30113966C9120
:10DDC00086E09CE00E94458865ED76E086E09CE078
:10DDD0000E94C889CE018F5A9F4F0E94922D6AE1FE
:10DDE00074E0F301808191810E94CB9A912C812C67
:10DDF000B12CA12CD12CC12C6296EFAC629763960A
:10DE0000FFAC639764960FAD649765961FAD6597F9
:10DE100066962FAD669767963FAD679768964FAD4C
:10DE2000689769965FAD69976FEF0E946058D3015C
:10DE30000D911C916DEC74E0C8010E94CB9A7C019D
:10DE400062ED74E0C8010E94CB9A8C010097E9F161
:10DE5000FC0180858F708430C1F56185728540E456
:10DE600050E0CE0101960E9465D86FE270E0CE01CD
:10DE700001960E942CD8892B59F4D80119962D911E
:10DE80003C9143E050E060E4CE0101960E94C62739
:10DE900000E020E030E240E150E0BE016F5B7F4FE8
:10DEA000CE018F5A9F4F0E94801E0E94E99A8823BC
:10DEB00061F08091CC08811108C041E0BE016F5B28
:10DEC0007F4FCE0101960E9479AAE114F104C9F1B5
:10DED000F70180858F708430A1F5409166075091DD
:10DEE000670761857285CE0101960E94FB3CCE01D9
:10DEF00001960E94773B882301F1A12CC12CF12CC3
:10DF0000E12C62960FAD629763961FAD639764969E
:10DF10002FAD649765963FAD659766964FAD669752
:10DF200067965FAD679768966FAD689769967FADA6
:10DF30006997CE0101960E941646CE0101960E9475
:10DF40003741D3011596ED91FC915382428294CAD8
:10DF50008FEF9FEFC559DF4F0FB6F894DEBF0FBEAE
:10DF6000CDBFDF91CF911F910F91FF90EF90DF9088
:10DF7000CF90BF90AF909F908F907F906F905F9069
:10DF80004F903F902F900895833009F4D2CC813088
:10DF900009F0C4CC6185062E000C770B880B990B19
:10DFA000B8CCC12CD12C7601D3011596ED91FC9102
:10DFB00082819381092E000CAA0BBB0BC816D906CF
:10DFC000EA06FB0609F458CAB601C3010E9487633A
:10DFD000D3011596ED91FC91D382C2824DCABF92B6
:10DFE000CF92DF92EF92FF920F931F93CF93DF9325
:10DFF000CDB7DEB72E970FB6F894DEBF0FBECDBFFC
:10E000002091640730916507232B09F4A6C0209165
:10E0100063072111A2C07C01809163078F5F809309
:10E020006307809162078F5F809362070E94ABA9AC
:10E030000091A8061091A9062091AA063091AB067E
:10E04000601B710B820B930B6B3071058105910581
:10E0500008F479C083E0E816F104A9F00E94ABA9A6
:10E060000091A4061091A5062091A6063091A7065E
:10E07000601B710B820B930BBB24B3946436710548
:10E080008105910508F4B12CE0916407F0916507D2
:10E090000681178101151105C1F1F80180858F7086
:10E0A000863079F51987088770E060E0CE01089620
:10E0B0000E943D65B701CE0108960E9498696AE109
:10E0C00074E0C8010E94CB9AFC01892BD1F09085A5
:10E0D0009F7095509230A8F4C680D780C114D104A7
:10E0E00081F0DA82C982B801CE0101960E943D65B5
:10E0F000B701CE0101960E949869F601C280D380D3
:10E10000EDCFF80102811381C5CFF3E0EF16F104E2
:10E1100051F00E94ABA96093A8067093A906809362
:10E12000AA069093AB06BB2051F00E94ABA9609366
:10E13000A4067093A5068093A6069093A706109256
:10E14000730C1092740C8091620781508093620767
:10E15000809163078150809363072E960FB6F894E1
:10E16000DEBF0FBECDBFDF91CF911F910F91FF900A
:10E17000EF90DF90CF90BF9008958091CC088F5F93
:10E180008093CC08A89583E090E00E94EF6F809187
:10E190005807811102C00E94038F8091CC088150E2
:10E1A0008093CC080895CF92DF92EF92FF92CF93A5
:10E1B000DF93EC018C85883068F40E94B2960E944F
:10E1C000ABA96B017C018C850E94CE96811109C0A0
:10E1D00088E08C87DF91CF91FF90EF90DF90CF9018
:10E1E00008950E94BD7061E070E080E090E00E94C0
:10E1F00079A90E94ABA9AB01BC014C195D096E095C
:10E200007F098D859E85B0E0A0E0481759076A0711
:10E210007B07C8F28C850E94C096DACF8F929F92BE
:10E22000BF92CF92DF92EF92FF920F931F93CF9303
:10E23000DF93CDB7DEB7AD970FB6F894DEBF0FBE54
:10E24000CDBF8091AC069091AD06892B09F4BFC279
:10E25000809162078111BBC2809162078F5F8093BA
:10E26000620769E073E185E59BE00E94C88985E566
:10E270009BE00E9441880091AC061091AD0662E9D6
:10E2800075E0C8010E94CB9A909367078093660758
:10E2900068E975E0C8010E94CB9A90930B078093C0
:10E2A0000A076AEB75E0C8010E94CB9A9093650754
:10E2B000809364076FE975E0C8010E94CB9A909340
:10E2C000A3068093A206009749F1DC011696ED9112
:10E2D000FC91309719F120852F702530F9F465EF06
:10E2E00072E185E59BE00E94C8898091A206909129
:10E2F000A3060E948A9F809359074AE050E0682F46
:10E3000085E59BE00E94458885E59BE00E94418869
:10E31000E091A206F091A3068681978190935D0714
:10E3200080935C070E94EA2B1092610710926007AD
:10E33000E0916607F0916707309709F4F8C0E6802E
:10E34000F78000916607109167070115110509F420
:10E35000E7C0E114F10409F4E3C0F70180858F7090
:10E36000853099F7C7010E948A9F823070F3A80117
:10E37000B701CE0101960E94CE42CE0101960E94C5
:10E38000773B882309F466C08C859D85009759F5F5
:10E39000CE0101960E949A9F8C01912C812C97FFAF
:10E3A00006C011950195110988248394912CCE0102
:10E3B00001960E94F53DC82ED12C8B85853009F43D
:10E3C00052C0863009F046C0B02E61E0802F0E9416
:10E3D000F8A861E0892809F481C0CA94CD2809F021
:10E3E00081C060E07FC0DC01ED91FC910284F38587
:10E3F000E02D1995892B49F08C859D85DC01ED91E7
:10E40000FC910084F185E02D19958C859D85DC01BA
:10E41000ED91FC910680F781E02D1995892BD1F0C3
:10E42000CE0101960E94F53D882341F040E050E185
:10E4300060E070E0CE0101960E9483198F8198857B
:10E44000892B41F040E050E260E070E0CE0101969F
:10E450000E948319D7011296ED90FC90CE0101968F
:10E460000E9437416ECFCD2829F462E0CE0101969B
:10E470000E94D01940E050E160E070E0CE010196CA
:10E480000E9483198F819885892B41F040E050E2EA
:10E4900060E070E0CE0101960E94831961E0802F58
:10E4A0000E94F8A860E0802F0E94CAA86DEE72E179
:10E4B00086E09CE00E94C889B80186E09CE00E944A
:10E4C000399F68EE72E186E09CE00E94C88966EEA2
:10E4D00072E186E09CE00E94C889BCCFCA94CD2836
:10E4E00009F07FCFC62ED12C8B2D0E94CAA861EED9
:10E4F00072E186E09CE00E94C889B80186E09CE059
:10E500000E94399F6FED72E186E09CE00E94C8890D
:10E51000B60186E09CE00E94399F6DED72E1D9CF93
:10E52000F80186819781909361078093600786E068
:10E530009CE00E94418869EC72E185E59BE00E94C5
:10E54000C88985E59BE00E944188E0916407F091CD
:10E550006507309709F4ACC0809162078F5F8093A4
:10E560006207068117810115110509F49CC0D801C5
:10E5700018968C918F70863009F08AC018A70FA367
:10E5800070E060E0CE0187960E943D658CA59DA558
:10E59000892B09F47DC08091AC069091AD06892B42
:10E5A00009F476C0EFA0F8A4E114F104B9F1F70181
:10E5B00080858F70863091F5F9A2E8A270E060E066
:10E5C000CE0180960E943D65EDA1FEA110821182D0
:10E5D000128213826AE174E0C7010E94CB9AFC01A7
:10E5E000892BE1F090859F7095509230B8F4C680E9
:10E5F000D780C114D10491F0DA82C982B701CE016B
:10E6000001960E943D65EE81FF8110821182128287
:10E610001382D6011296CD90DC90EBCF64EC72E1C0
:10E6200086E09CE00E94C8894AE050E06AA586E046
:10E630009CE00E94458862EC72E186E09CE00E94CA
:10E64000C8894AE050E069A586E09CE00E944588C0
:10E6500086E09CE00E944188ECA5FDA51082118215
:10E660001282138289A5843020F4823040F060E069
:10E6700007C0803489F08234A1F0803249F462E02E
:10E680008AA50E94F8A8ECA5FDA58181807F8183E1
:10E69000F8010281138167CF62E08AA50E94F8A881
:10E6A000F7CF60E0FACF80916207815080936207D4
:10E6B00065EB72E185E59BE00E94C8896DEA72E135
:10E6C00085E59BE00E94C88981E020916607309132
:10E6D0006707232B09F480E00E94EF1964EA72E1D6
:10E6E00085E59BE00E94C88981E020916407309114
:10E6F0006507232B09F480E00E94EF196DE972E1B0
:10E7000085E59BE00E94C88981E020915C073091FB
:10E710005D07232B09F480E00E94EF1964E972E1A0
:10E7200085E59BE00E94C889809109070E94EF1946
:10E7300085E59BE00E9441886FE872E185E59BE0FA
:10E740000E94C8890E94CB28AB01BC012AE085E564
:10E750009BE00E94F58785E59BE00E94418881E06F
:10E7600080935F0782E29BE00E94F617882351F0B6
:10E7700082E29BE00E94D37084E090E09093CE0808
:10E780008093CD088091CD089091CE08079731F401
:10E7900084E090E09093CE088093CD08809162074A
:10E7A00081508093620780915F07AD960FB6F89411
:10E7B000DEBF0FBECDBFDF91CF911F910F91FF90B4
:10E7C000EF90DF90CF90BF909F908F90089580E062
:10E7D000ECCFCF92DF92EF92FF921F93CF93DF9314
:10E7E000EC017B016A018C85883048F40E94CE964A
:10E7F000882319F08C850E94B29688E08C87F701F7
:10E8000082819381A481B5810097A105B10551F45E
:10E8100090E080E0DF91CF911F91FF90EF90DF902B
:10E82000CF9008958F3F9F4FAF4FBF4F89F370E058
:10E8300060E081E20E940997182F8C87883040F7AA
:10E8400080E591E00E9489A4A7014E5F5F4F24E01C
:10E8500030E06CE070E0812F0E947521B601812FBD
:10E860000E94DD9664E070E0812F0E94EA910E9490
:10E87000ABA96B017C018C850E94CE96873121F17A
:10E880008C3111F1882321F20E94ABA9AB01BC01AC
:10E890004C195D096E097F098D859E85B0E0A0E069
:10E8A00084179507A607B70748F00E94BD7061E07E
:10E8B00070E080E090E00E9479A9DDCF8C850E9415
:10E8C000C09688E08C87A4CF81E090E0A3CFAF9280
:10E8D000BF92DF92EF92FF920F931F93CF93DF933C
:10E8E00000D000D0CDB7DEB78C017B01D42EFB0168
:10E8F00084819581892BF9F0A080B1806FE370E06D
:10E90000C5010E942CD80097B1F09C012A193B093F
:10E9100037FD11C050E040E0B701CE0101960E94E2
:10E920002787BE016F5F7F4FC7010E947585CE01AB
:10E9300001960E94D78664EA75E0C7010E9460854F
:10E94000882321F1F801128A118A80E090E19587ED
:10E95000848784E890E0948B838B81E0868780E0D5
:10E9600090E2908B8787D58A81E090E026960FB65B
:10E97000F894DEBF0FBECDBFDF91CF911F910F91F5
:10E98000FF90EF90DF90BF90AF90089561EB75E03E
:10E99000C7010E946085882369F0F801128A118AF4
:10E9A000148A138A84E890E095878487168680E02D
:10E9B00090E3D7CF90E080E0D9CFEF92FF920F9312
:10E9C0001F93CF93DF9300D01F92CDB7DEB78C019A
:10E9D0007B01FB0184858830A8F08FE094E0F8018A
:10E9E000918380831282138214821582C8010F9052
:10E9F0000F900F900F90DF91CF911F910F91FF908B
:10EA0000EF90089580E591E00E9489A424E030E031
:10EA1000AE014F5F5F4F6CE070E0F70184850E94AC
:10EA2000C621BE016F5F7F4FC8010E940D8ADECFF5
:10EA3000EF92FF920F931F93CF93DF9300D000D0FC
:10EA4000CDB7DEB78091310B9091320B892B09F451
:10EA50006CC087E70E94069C8091310B9091320B2D
:10EA6000DC01ED91FC910088F189E02D70E060E01F
:10EA7000199510E000E08091310B9091320BDC0190
:10EA8000ED91FC9111971C962D913C910217130763
:10EA900040F40190F081E02D60E019950F5F1F4F69
:10EAA000EACF0088F189E02D70E060E019950AE274
:10EAB00013E08EE2E82E83E0F82E8091310B9091E6
:10EAC000320BF80161918F01DC01ED91FC91019015
:10EAD000F081E02D1995E016F10679F78091310B60
:10EAE0009091320BDC01ED91FC910488F589E02DC9
:10EAF00019956AE076E0CE0101960E941687CE0154
:10EB000001960E94F1AFCE0101960E94D78687E060
:10EB100090E00E94249F87E090E00E942E9F6FE289
:10EB200075E185E59BE00E94C8891092510B109217
:10EB3000500B80E090E190934C0B80934B0B84E85A
:10EB400090E09093530B8093520B81E080934D0B98
:10EB500080E090E290934F0B80934E0B82E780937E
:10EB6000540B8FE39BE00E944E158FE39BE00E94C5
:10EB70000F1A88EC90E026960FB6F894DEBF0FBE11
:10EB8000CDBFDF91CF911F910F91FF90EF9008952E
:10EB9000CF93DF93CDB7DEB72E970FB6F894DEBFD5
:10EBA0000FBECDBF80916207811121C180916207A4
:10EBB0008F5F8093620764E673E185E59BE00E94C6
:10EBC000C88985E59BE00E9441881092510B109204
:10EBD000500B80E090E190934C0B80934B0B84E8BA
:10EBE00090E09093530B8093520B81E080934D0BF8
:10EBF00080E090E290934F0B80934E0B82E78093DE
:10EC0000540B8FE39BE00E9437218B37910509F06D
:10EC1000C5C066E573E186E09CE00E94C88986E095
:10EC20009CE00E9441888091AC069091AD06892BB2
:10EC300021F081E090E00E94A1651C821B8283E8A4
:10EC400092E09A8389838FE39BE09E838D838FEF8D
:10EC50009FEF98878F83CE0101960E94FBA490932B
:10EC6000AD068093AC068FE39BE00E940F1A809163
:10EC7000AC069091AD06892B01F56AE473E18FE54E
:10EC80009BE00E94C8898FE59BE00E9441886AE072
:10EC900076E0CE0109960E941687CE0109960E9461
:10ECA000F1AFCE0109960E94D7868091620781500C
:10ECB0008093620790E080E019C067E373E185E527
:10ECC0009BE00E94C88985E59BE00E944188809175
:10ECD00062078150809362070E940E718091310B10
:10ECE0009091320B892B59F481E090E02E960FB66B
:10ECF000F894DEBF0FBECDBFDF91CF9108950E9483
:10ED00001B9C882389F382E70E94069C8091310B2B
:10ED10009091320BDC01ED91FC910088F189E02D9E
:10ED200060E670E019956091310B7091320B40E014
:10ED3000CE0109960E949B87BE01675F7F4F83E3E8
:10ED40009BE00E947585CE0109960E94D78680912E
:10ED5000310B9091320BDC01ED91FC910488F58927
:10ED6000E02D199569E173E186E09CE00E94C88975
:10ED700063E37BE0CE0109960E940D87BE01675FC9
:10ED80007F4F86E09CE00E94BA8986E09CE00E946A
:10ED90004188CE0109960E94D786A6CF8FE39BE0DB
:10EDA0000E942415892BA1F08FE39BE00E944E1551
:10EDB0006AE076E0CE0101960E941687CE010196A8
:10EDC0000E94F1AFCE0101960E94D7860E9472B0D8
:10EDD0008FE39BE00E940F1A66E273E185E59BE0FA
:10EDE0000E94C88985E59BE00E9441885ECF8FEF35
:10EDF0009FEF7CCFFF920F931F93CF93DF9300D0B1
:10EE000000D0CDB7DEB78C01BC01CE0101960E94C7
:10EE10000D87BE016F5F7F4F86E09CE00E94BA893C
:10EE200086E09CE00E944188CE0101960E94D78630
:10EE30006AE575E1CE0101960E94DF86BE016F5F33
:10EE40007F4FC8010E944585F82ECE0101960E9491
:10EE5000D786FF2069F0B801CE0101960E940D8788
:10EE6000CE0101960E94F1AFCE0101960E94D78695
:10EE700026960FB6F894DEBF0FBECDBFDF91CF91BF
:10EE80001F910F91FF9008954F925F926F927F9222
:10EE90008F929F92AF92BF92CF92DF92EF92FF92AA
:10EEA0000F931F93CF93DF93CDB7DEB7C859D10926
:10EEB0000FB6F894DEBF0FBECDBF8E010F5B1F4FA4
:10EEC000D8011D921C92FE01ED5BFF4F8EE1DF0128
:10EED0001D928A95E9F78091310B9091320B892B25
:10EEE00009F4CFC10E941B9C882309F4CAC182E7A0
:10EEF0000E94069C8091310B9091320BDC01ED91C8
:10EF0000FC910088F189E02D60E270E019954FE1F5
:10EF100050E0B8018091310B9091320B0E94609CBF
:10EF20007C018091310B9091320BDC01ED91FC91D1
:10EF30000488F589E02D1995E114F10409F4A1C1C3
:10EF4000F801EE0DFF1D108280913E0B1F928F93F2
:10EF500080913D0B1F928F9380913C0B1F928F935A
:10EF600080913B0B1F928F9380913A0B1F928F934E
:10EF70008091390B1F928F938DEB95E09F938F9328
:10EF80001F9280E48F93FE0131966F01FF93EF9300
:10EF90000E947FD869E476E185E59BE00E94C889FC
:10EFA000B80185E59BE00E947189B60185E59BE08B
:10EFB0000E94718985E59BE00E9441887E01F1E60F
:10EFC000EF0EF11CD70113961C921E92129788EE39
:10EFD00093E0A0E0B0E0F70184839583A683B78334
:10EFE00088E0848788EE93E0968785878BE392E0BC
:10EFF00091838083108A1786128B018B148A138A5F
:10F0000080E590E0968B858B118E61E675E186E058
:10F010009CE00E94C88963E37BE0CE0185589F4F46
:10F020000E940D87BE0165587F4F86E09CE00E94DC
:10F03000BA8986E09CE00E944188CE0185589F4FA6
:10F040000E94D7866CEE75E0CE0183579F4F0E94D9
:10F0500016876CEE75E0CE0185589F4F0E9416878B
:10F06000BE0165587F4FCE018B579F4F0E940D8781
:10F0700063E37BE0CE018B579F4F0E947386BE01F6
:10F0800063577F4F0E947386BC01CE018D569F4F00
:10F090000E940D87CE018B579F4F0E94D786CE01CD
:10F0A00085589F4F0E94D786CE0183579F4F0E945D
:10F0B000D7868EEE95E0CB57DF4F99838883C5586E
:10F0C000D040C757DF4F19821882C958D040C55762
:10F0D000DF4F19821882CB58D040CD56DF4F888140
:10F0E0009981C359D040C957DF4F99838883C75846
:10F0F000D04063E476E186E09CE00E94C8890E94EB
:10F10000CB28AB01BC012AE086E09CE00E94F58799
:10F1100086E09CE00E94418864E670E080E090E038
:10F120000E9479A98AEF96E7D70150969C938E9317
:10F130001F976CE478E884E391E90E942ACD8C0162
:10F140000FB6F894DEBF0FBECDBF892B09F4F4C013
:10F1500083E090E00E94E7C9D8011D969C938E93AE
:10F160001C97FC01F182E0821282C7010E94F6170F
:10F17000882319F0C7010E94D370D70153966D916F
:10F180007C9154975596AD90BC906115710509F42A
:10F190008FC0CE0185589F4F0E940D8AA501BE01E8
:10F1A00065587F4FC7010E94E973181619060CF0C5
:10F1B000C0C0D7015196BC9051975296AC90DF9247
:10F1C000CF928CEB95E19F938F931F930F930E94A7
:10F1D000B1CDDF92CF9287EB95E19F938F931F93F1
:10F1E0000F930E94B1CDD8011C96ED91FC9181E066
:10F1F0008283DF92CF9284EB95E19F938F931F934D
:10F200000F930E94B1CDD8011C96ED91FC91128212
:10F21000AF92BF928EE795E19F938F931F930F93C9
:10F220000E94B1CD0FB6F894DEBF0FBECDBFB12C9A
:10F2300085E7C82E85E1D82E8B2D94E08902F00158
:10F240001124A5E8B0E0AC0FBD1FEA0FFB1F8081C1
:10F2500091810097A9F12281338121153105C9F3EC
:10F260003F932F939F938F93DF92CF921F930F9390
:10F270000E94B1CDB3940FB6F894DEBF0FBECDBFE0
:10F28000DBCF40E250E06BE776E1C8010E9457CC4B
:10F290006DE576E185E59BE00E94C889B80185E5CA
:10F2A0009BE00E94718985E59BE00E9441884CCEDD
:10F2B000F70161897289A501C7010E949D1875CF68
:10F2C00089EB95E19F938F931F930F930E94B1CD8C
:10F2D000D70158961C921E925797D8011C96ED9113
:10F2E000FC91C080D1800F900F900F900F9043E35E
:10F2F000A42EB12CD601ED91FC910084F185E02D76
:10F30000C601199541975CF4B1E0AB1AB10839F028
:10F3100064E170E080E090E00E9479A9EBCFD60133
:10F32000ED91FC910084F185E02DC601199541977E
:10F3300034F4C8010E940D9110E000E05AC06AE068
:10F3400076E0CE0183579F4F0E941687912CA12C07
:10F35000D601ED91FC910688F789E02DC60119953B
:10F360008823E1F1BDE0AB1201C0A92CD601ED91DB
:10F37000FC910688F789E02DC60119958111BBC063
:10F38000D601ED91FC910084F185E02DC60119951F
:10F39000892B09F4C2C0D601ED91FC910284F3855A
:10F3A000E02DC6011995B82EBAE08B1709F4B7C045
:10F3B000EDE08E1709F4B3C0FFEF8F1709F4ADC06D
:10F3C000682FCE0183579F4F0E9402869A2CAB2C48
:10F3D000BFCFBAE0BB12FACFAB12F8CFCC24C394A4
:10F3E000D12CCE0183579F4F0E94D786CD2809F498
:10F3F000A3CFD7015796ED90FC9065E376E186E0C8
:10F400009CE00E94C889B70186E09CE00E94399F79
:10F4100086E09CE00E94418864E670E080E090E035
:10F420000E9479A90115110509F465C1B8ECEB1624
:10F43000F10409F03EC169E276E185E59BE00E94B6
:10F44000C88964EF71E080E090E00E9479A9EF96AE
:10F450001FAE1EAEEF97C158DF4F19821882CF57EB
:10F46000D0408FEF9FEFCF57DF4F99838883C158EC
:10F47000D0408DE692E0ED969FAF8EAFED97CD57E1
:10F48000DF4F19830883C358D040F89490E080E0A0
:10F490000E94A1658111CEC06DE176E18FE59BE010
:10F4A0000E94C8898FE59BE00E944188C8010E94A4
:10F4B0000D9124EFE22EFF24F394CE018D569F4F41
:10F4C0000E94D786C701C856DF4F0FB6F894DEBF3B
:10F4D0000FBECDBFDF91CF911F910F91FF90EF90A5
:10F4E000DF90CF90BF90AF909F908F907F906F9064
:10F4F0005F904F900895D601ED91FC910084F185C5
:10F50000E02DC6011995892B09F03ACF64E670E029
:10F5100080E090E00E9479A929CFBB24BA946CEFD7
:10F5200075E089E69BE00E947189BE0163577F4FB9
:10F5300089E69BE00E94BA8989E69BE00E944188A7
:10F540006CE675E1CE0185589F4F0E94DF86BE01B3
:10F5500065587F4FCE0183579F4F0E944585982E57
:10F56000CE0185589F4F0E94D786992099F1CF569A
:10F57000DF4F28813981C159D04049E050E0BE01B8
:10F5800063577F4FCE0185589F4F0E942787ED9686
:10F590008EAD9FADED97412C512C3201009719F0A3
:10F5A0000E94D2CB2B014201CE0185589F4F0E9471
:10F5B000D7864114510429F0D70158965C924E9297
:10F5C0005797B40189E69BE00E94399F89E69BE04A
:10F5D0000E944188F7018784908881149104D1F0BA
:10F5E000CF56DF4F88819981C159D040892B91F046
:10F5F000BE0163577F4FCE0185589F4F0E940D87F4
:10F60000CE0185589F4FF4011995CE0185589F4F23
:10F610000E94D7866AE076E0CE0183579F4F0E9412
:10F62000A786FFEFBF12D5CEC8010E940D91D12C45
:10F63000C12CD7CECE0185589F4F0E94FBA490933A
:10F64000AD068093AC067894C8010E940D9180911C
:10F65000AC069091AD06892BD1F46AE076E0CE013C
:10F6600083579F4F0E941687CE0183579F4F0E945A
:10F67000F1AFCE0183579F4F0E94D78666E076E1B7
:10F680008FE59BE00E94C889F12CE12C16CF0E94E7
:10F690000E7180915F07882329F00E947A9E71FF86
:10F6A0000E94841B6FEF75E185E59BE00E94C8898D
:10F6B00004CFE0E3EE16E1E0FE0651F46BEE75E1F7
:10F6C00085E59BE00E94C889C8010E940D91F5CE96
:10F6D00063ED75E18FE59BE00E94C889C8010E9437
:10F6E0000D91B7018FE59BE00E94399F8FE59BE06C
:10F6F0000E944188E2CE60EC75E186E09CE00E94C9
:10F70000C889EE24EA94FE2CD8CE4F925F926F9275
:10F710007F928F929F92AF92BF92CF92DF92EF92A1
:10F72000FF920F931F93CF93DF93CDB7DEB7C157EF
:10F73000D1090FB6F894DEBF0FBECDBF8C014B01CF
:10F74000F42E4AE050E06F2D86E09CE00E94458850
:10F750006FE47FE086E09CE00E94C889B401CE019E
:10F7600001965C010E940D87B50186E09CE00E9435
:10F77000BA8986E09CE00E944188C5010E94D78634
:10F7800092E0F91280C16DE47FE0C5010E94DF863E
:10F79000D40114962D913C9115978D819E81281747
:10F7A000390711F58D919C9169817A81009759F003
:10F7B0006115710509F064C1232B09F4A3C1DC01B3
:10F7C0008C9190E00DC06115710509F49BC1232B4C
:10F7D00009F498C1FB01808190E091958195910990
:10F7E000FF24F394892B09F0F12CC5010E94D786E0
:10F7F000FF2009F4D3C240E06DE271E0C8010E942D
:10F80000E9B080905A0790905B0766E47FE0CE01F4
:10F8100084599F4F0E94DF866FE37FE0CE018A59B3
:10F820009F4F0E94DF86CE01865A9F4F0E9415236C
:10F83000A096FFACA0976F96EFAC6F976E96DFAC7B
:10F840006E976D96CFAC6D976AE076E0CE018196AB
:10F850000E941687BE016F5D7F4FC5010E940D8714
:10F860006C2DC5010E9428866FEF75E00E945986B5
:10F870006D2D0E9428866FEF75E00E9459866E2DCF
:10F880000E9428866FEF75E00E9459866F2D0E94B6
:10F890002886BC01CE01805A9F4F0E940D87C5016A
:10F8A0000E94D786CE0181960E94D7866AE37FE0C8
:10F8B000CE018C5A9F4F0E94DF866E01EEE4CE0E81
:10F8C000D11C6AE076E0C6010E94168791E3E92E1A
:10F8D0009BE0F92E27E3622E2BE0722E2601D70142
:10F8E00018966C9170E084E0759567958A95E1F7BC
:10F8F000C5010E94DA9B4D815E8169817A81C201D6
:10F900000E94D685C5010E94D786F70160856F7079
:10F9100070E0C5010E94DA9B4D815E8169817A8128
:10F92000C2010E94D685C5010E94D786FFEFEF1A5B
:10F93000FF0A6E147F0499F664E37FE0CE01885BD2
:10F940009F4F0E94DF8662E27FE0CE0181960E9497
:10F95000DF86BE016F5D7F4FCE01805C9F4F0E94AE
:10F960000D872696EEACFFAC269788E1E80EF11CD9
:10F97000B701CE01805C9F4F0E94AE858111C5C04A
:10F98000CE01805C9F4F0E941686BE01685B7F4F50
:10F99000CE01805C9F4F0E947386B6010E947386E1
:10F9A000BE016C5A7F4F0E947386BE01605A7F4F22
:10F9B0000E947386BE016A597F4F0E9473867C0144
:10F9C0004AE0B50180E590E00E949CCCF5010190F1
:10F9D0000020E9F73197AF014A195B09B501C7016A
:10F9E0000E94D685811103C0C7010E941686BE0100
:10F9F00064597F4FC7010E947386B4010E945986E3
:10FA0000BC01C8010E94BA89C8010E944188CE0188
:10FA1000805C9F4F0E94D786CE0181960E94D78638
:10FA2000CE01885B9F4F0E94D786C2010E94D78675
:10FA3000CE018C5A9F4F0E94D786CE01805A9F4F8D
:10FA40000E94D786CE018A599F4F0E94D786CE0149
:10FA500084599F4F0E94D786C8010E94418864E65E
:10FA600070E080E090E00E9479A9D801ED91FC91CE
:10FA70000488F589E02DC801199501E010E0EDC07A
:10FA80000E9437D8ADCEB1E0FB1220C262E07FE029
:10FA9000C5010E94DF86B501C4010E944585582E2C
:10FAA000C5010E94D786552009F4D8C1EE2009F47B
:10FAB00073C166E070E0C4010E9413A74AE0B80178
:10FAC000CE01885B9F4F0E949B87409166075091B3
:10FAD0006707F40160817181CE0181960E94FB3C31
:10FAE000CE0181960E94773B811122C000E911E08E
:10FAF000CE0181960E943741CE01885B9F4F0E94C4
:10FB0000D786ABC0FF24F39470CE22962EAD3FADC6
:10FB1000229726968EAD9FAD269769E07FE0820FF3
:10FB2000931F0E9429CC2696FFAEEEAE26972DCFCE
:10FB30002A966EAD7FAD2A97CE0181960E94C0A114
:10FB4000892BA1F224961CAE1DAE1EAE1FAE2497CB
:10FB500028961CAE1DAE1EAE1FAE289722968FAD06
:10FB60002297807F22968FAF229740E050E3BE011C
:10FB70006F5D7F4FCE01805C9F4F0E94024000E08E
:10FB800020E030E340E250E0B501CE01805C9F4FC1
:10FB90000E94801EBC01C6010E94B18608EC10E1E3
:10FBA000A7CFEE2009F4F8C066E070E0C4010E941F
:10FBB00013A74091660750916707D4016D917C911E
:10FBC000CE0181960E94FB3CCE0181960E94773B3C
:10FBD00000E911E08823E9F18BA5873061F4CE01BB
:10FBE00081960E94D74361E0892B09F462E0CE013F
:10FBF00081960E94D01924961CAE1DAE1EAE1FAE7B
:10FC0000249728961CAE1DAE1EAE1FAE28972296D6
:10FC10008FAD2297807F22968FAF229740E050E3EE
:10FC2000BE016F5D7F4FCE01805C9F4F0E940240FE
:10FC300000E020E030E340E250E0B501CE01805C1E
:10FC40009F4F0E94801EBC01C6010E94B18608EC35
:10FC500010E1CE0181960E943741C801CF58DF4F95
:10FC60000FB6F894DEBF0FBECDBFDF91CF911F91CD
:10FC70000F91FF90EF90DF90CF90BF90AF909F904B
:10FC80008F907F906F905F904F900895F401608106
:10FC900071810E94CB9A7C01892B09F0C5C004E9CF
:10FCA00011E0DBCFEE2009F477C069E070E0C40119
:10FCB0000E9413A74AE0B801C5010E949B8741E05A
:10FCC00050E060EB74E0C4010E94D6854D815E81F6
:10FCD00069817A81C4010E94D68565EE7EE086E066
:10FCE0009CE00E94C889B401CE0181960E940D87D4
:10FCF000BE016F5D7F4F86E09CE00E94BA8986E07E
:10FD00009CE00E944188CE0181960E94D7866DEDCD
:10FD10007EE0CE0181960E94DF86F4018481958188
:10FD20002DA13EA182179307E1F4892B91F1E08088
:10FD3000F18069A07AA0D7018D917D01882349F1D6
:10FD4000082E000C990B0E94BCD76C01F301819125
:10FD50003F01082E000C990B0E94BCD7C816D9068B
:10FD600051F3CE0181960E94D786552031F041E0B3
:10FD700068EC70E0C8010E94E9B0D4018D919C91BB
:10FD80000E948E8E009711F484E991E08C01C501E8
:10FD9000B6CE55245394E5CF01E982CF6BEF7EE0D8
:10FDA000C5010E94DF86B501C4010E944585F82E79
:10FDB000C5010E94D786F110F4CE65EF7EE0C50143
:10FDC0000E94DF86B501C4010E944585F82EC50159
:10FDD0000E94D786FF2009F479C0EE20E9F265E0A1
:10FDE00070E0C4010E9413A76FEF75E0C4010E9488
:10FDF0006085882339F0E0906607F0906707E1148A
:10FE0000F10491F46AE076E0C4010E9460858111FA
:10FE100007C08091660790916707009709F036CF79
:10FE2000E090AC06F090AD0640E068EC70E2C801EE
:10FE30000E94E9B0C8010E9441881C821B8283E8AD
:10FE400092E09A8389831E830D838FEF9FEF9887BB
:10FE50008F83B701C5010E9476A001CE6BEE7EE0D4
:10FE6000C5010E94DF86B501C4010E944585F82EB8
:10FE7000C5010E94D786F11015CF60ED7EE0C50167
:10FE80000E94DF86B501C4010E944585182FC50177
:10FE90000E94D78600E0112309F4DFCE80E00E94A3
:10FEA0001A9F68EA7EE085E59BE00E94C88985E5A7
:10FEB0009BE00E9441886AE076E0C5010E941687B7
:10FEC000C5010E94F1AFC5010E94D78600E0D6CDE2
:10FED0000895FC01248135816217730748F48081FD
:10FEE0009181009729F0860F971FFC01808108956A
:10FEF00080E008950895AF92BF92CF92DF92EF9283
:10FF0000FF920F931F93CF93DF936C017B018B01C3
:10FF1000040F151FEB015E01AE18BF08C017D10713
:10FF200059F06991D601ED91FC910190F081E02D9D
:10FF3000C6011995892B79F7C501DF91CF911F91E2
:10FF40000F91FF90EF90DF90CF90BF90AF9008950A
:10FF5000FC01A089B1898C91A689B78982FD0FC067
:10FF60009C91818D8F5F8F73228D821749F0A18DB7
:10FF7000AE0FBF2FB11D5D969C93818F08958C911C
:10FF80000895FC01538D448D252F30E0842F90E09F
:10FF9000821B930B541710F0CF9608950197089584
:10FFA000FC01918D828D981761F0A28DAE0FBF2F4D
:10FFB000B11D5D968C91928D9F5F9F73928F90E0A3
:10FFC00008958FEF9FEF0895FC01918D828D981712
:10FFD00031F0828DE80FF11D858D90E008958FEF4F
:10FFE0009FEF0895FC01918D228D892F90E0805C18
:10FFF0009F4F821B91098F739927089580ED98E098
:020000021000EC
:100000000E94F27F21E0892B09F420E0822F0895DD
:100010008DE699E00E94F27F21E0892B09F420E02F
:10002000822F08958AE09AE00E94F27F21E0892BD6
:1000300009F420E0822F089589E69BE00E94F27F78
:1000400021E0892B09F420E0822F0895FC01A48D82
:10005000A80FB92FB11DA35ABF4F2C91848D90E0EA
:1000600001968F739927848FA689B7892C93A089CD
:10007000B1898C91837080648C93938D848D981357
:1000800006C00288F389E02D80818F7D80830895EA
:10009000EF92FF920F931F93CF93DF93EC0181E0D8
:1000A000888F9B8D8C8D98131AC0E889F98980817F
:1000B00085FF15C09FB7F894EE89FF896083E889B2
:1000C000F98980818370806480839FBF81E090E0A4
:1000D000DF91CF911F910F91FF90EF900895F62E31
:1000E0000B8D10E00F5F1F4F0F731127E02E8C8DCB
:1000F0008E110CC00FB607FCFACFE889F989808110
:1001000085FFF5CFCE010E942680F1CFEB8DEC0F5D
:10011000FD2FF11DE35AFF4FF0829FB7F8940B8F2C
:10012000EA89FB8980818062CFCFCF93DF93EC0196
:10013000888D8823B9F0AA89BB89E889F9898C91CF
:1001400085FD03C0808186FD0DC00FB607FCF7CF8B
:100150008C9185FFF2CF808185FFEDCFCE010E948B
:100160002680E9CFDF91CF91089580E090E0892B40
:1001700029F00E941C8081110E94000080E090E024
:10018000892B29F00E94128081110E94000080E0DA
:1001900090E0892B29F00E94088081110E940000C4
:1001A00080E090E0892B29F00E94FE7F81110C9461
:1001B00000000895DC01ED91FC910190F081E02DAB
:1001C00019948FEF9FEF0895FC01628973898489E8
:1001D00095890895EF920F931F93CF93DF93FC01BE
:1001E000248D222341F0213051F1DF91CF911F91D5
:1001F0000F91EF9008952289338944895589868922
:100200009789A08DB18D821B930BA40BB50B892F01
:100210009A2FAB2FBB278C010F5F1F4F6281738119
:1002200084819581CFB7F894DCB7E1E0ECBFEE2490
:10023000E394E2E0FEEF1995DCBFCFBFD6CFF0E04C
:10024000E0E0DF91CF911F910F91EF901994FC01A5
:10025000138E128E41110CC082899389A489B589AD
:10026000868B978BA08FB18F148E81E090E00895DC
:1002700090E080E00895CF92DF92EF92FF92CF93CB
:10028000DF93DC01CB01642FCFB7F8946D01EE242E
:10029000FF24CBBEDCB741E04CBFA901E1E0FEEF9B
:1002A0001995DCBFCFBFDF91CF91FF90EF90DF902A
:1002B000CF900895CF93DF93FC01248D211110C0BE
:1002C000EC01828D938D892B49F066897789808D29
:1002D000918D30E020E045E00E943B811B8E1A8E1C
:1002E000DF91CF9108951F93CF93DF93FC01248D6D
:1002F000211145C0162FEC01828D938D892B49F475
:1003000066897789808D918D30E020E043E00E94FE
:100310003B814A8D5B8DCA0181709927FE01E80FF0
:10032000F91F158F892B69F02D8D3E8D6E897F8980
:10033000888D998D640F751F811D911D41E00E946C
:100340003B818A8D9B8D01969B8F8A8F8115914071
:10035000B1F46E897F89888D998D30E020E045E089
:100360000E943B811B8E1A8E8E899F89A88DB98D24
:100370009F5FAF4FBF4F8E8B9F8BA88FB98F81E050
:1003800090E0DF91CF911F910895DC01ED91FC91F8
:100390000280F381E02D40E01994FB0144815581F6
:1003A00022813381215031094217530750F4A08133
:1003B000B181A40FB51F8C9384819581019695839B
:1003C000848380E00895CF93DF93EC01E881F98185
:1003D0000284F385E02DCE0119950196B9F7DF91DE
:1003E000CF910895FC01A285B3851097A9F0868569
:1003F0009785029788F0CD010196938782876C9349
:10040000868597850197978786870284F385E02DF7
:10041000108281E090E0089590E080E00895FC0172
:10042000868197818F3F980729F02FEF3FEF378321
:1004300026830895A085B185109789F02485358598
:100440002115310561F0CD010196918780878C914E
:100450002150310935872487082E000C990B089507
:10046000FC0186819781019639F481E024853585E8
:10047000232B19F480E0089581E00895CF92DF9254
:10048000EF92FF920F931F93CF93DF937C016A014A
:100490008B01D0E0C0E0CC15DD0581F0D701ED91F6
:1004A000FC910284F385E02DC70119958F3F9807D1
:1004B00029F0F80181938F012196EDCFCE01DF91D4
:1004C000CF911F910F91FF90EF90DF90CF90089503
:1004D000CF93C62FDC01ED91FC910088F189E02DCE
:1004E0001995DC01ED91FC910190F081E02D6C2FCC
:1004F000CF911994062E000C770BFC01778366834D
:100500000895CF93DF93EC018E819F81019611F5C1
:10051000E881F9810088F189E02DCE011995DC018F
:10052000ED91FC910084F185E02D1995892BB1F0B6
:10053000E881F9810284F385E02DCE01199581329D
:10054000910534F3E881F9810684F785E02D682F61
:10055000CE01199581E0DF91CF91089580E0FBCF26
:10056000FC0120812EBD9B012150310941F05181B8
:100570000DB407FEFDCF4EB55EBD4193F5CF615082
:100580007109860F971F0DB407FEFDCF2EB5FC0134
:1005900020830895E0916907F0916A078081909126
:1005A0006807892B80830895E0916907F0916A07B5
:1005B00090818091680780958923808308958EBDFE
:1005C00000000DB407FEFDCF8EB5089590E0209198
:1005D000BA08233339F40C96982F990F990F990F75
:1005E00080E008954896F8CFEF92FF920F931F9303
:1005F000CF93DF93EC018B017A010E94ABA9688B4A
:10060000798B8A8B9B8B8C819D81DC01ED91FC9198
:100610000280F381E02DA701B801DF91CF911F91F6
:100620000F91FF90EF9019941F93CF93DF93EC01FC
:10063000162F0E94ABA9688B798B8A8B9B8B8C8140
:100640009D81DC01ED91FC910190F081E02D612F05
:10065000DF91CF911F911994CF92DF92EF92FF9289
:10066000CF93DF93EC018E819F818F3F980759F0E4
:100670002FEF3FEF3F832E83DF91CF91FF90EF90DD
:10068000DF90CF9008950E94ABA96B017C01A4EF8D
:10069000CA0EA1E0DA1EE11CF11CE881F981008894
:1006A000F189E02DCE011995DC01ED91FC910084DA
:1006B000F185E02D1995892B39F40E94ABA96C15B1
:1006C0007D058E059F0548F3E881F9810088F18951
:1006D000E02DCE011995DC01ED91FC910284F385AA
:1006E000E02DDF91CF91FF90EF90DF90CF901994A4
:1006F0000E94B7D70F931F93CF93DF938C01CDEA5E
:10070000D7E0688179816115710529F0C8010E94DF
:1007100037D8892B29F00B80DC81C02D209789F7F1
:10072000CE01DF91CF911F910F9108950C9483CA50
:10073000CF92DF92EF92FF920F931F93CF93DF93AD
:100740006C018B0186E090E00E94E7C9EC01909378
:10075000B3078093B207F60101900020E9F7CF01BB
:100760008C199D090E94E7C97C01B6010E9440D8FE
:10077000F60101900020E9F73197EC19FD09EE0D23
:10078000FF1D1082F982E8821B830A838091F007A3
:100790009091F1079D838C83D093F107C093F0076C
:1007A000DF91CF911F910F91FF90EF90DF90CF904D
:1007B0000895FC01868197818F3F980729F02FEFDC
:1007C0003FEF378326830895808591850C9475CDFE
:1007D0007F928F929F92AF92BF92CF92DF92EF92D1
:1007E000FF920F931F93CF93DF93CDB7DEB7A697FA
:1007F0000FB6F894DEBF0FBECDBF8C01762E942EBF
:10080000852E20E2A22ECE0101967C01DC01EA2D8C
:100810001D92EA95E9F76801F3E4CF0ED11C8FE051
:1008200094E09AA389A38FEF8BA38CA38DA38EA3AF
:1008300043E450E0BE016F5D7F4FC6010E94582225
:10084000019609F4BFC081E089838A8386E0B82ECF
:10085000BB821C82D80114966D917D918D919C91E3
:1008600017970E94DED36D837E838F839887898656
:100870009A8680E890E09C878B874CE150E0B70136
:10088000C6010E94ED21FE0137968AE1DF011D922B
:100890008A95E9F74801B8E08B0E911CF401D70165
:1008A00001900D92BA94E1F740E150E0B701C60122
:1008B0000E94ED21F7011192AA94E9F796E0A92E82
:1008C000B12C40E250E0B701C6010E94ED21F1E0F9
:1008D000AF1AB108B1F783E6898392E89A8393E56A
:1008E0009B838C8385E38D8381E08E837F829DE370
:1008F000988797E099878A8786E0F401DE011B9646
:1009000001900D928A95E1F78CE0898B8A8B61E0EA
:1009100076E0CE0143960E9440D8D8011B966C9198
:10092000CE0149960E94EEA5F8016485CE014B9652
:100930000E94EEA5D8011D966C91CE014D960E94A5
:10094000EEA54EE150E0B701C6010E94ED21B3E0F3
:100950007B121EC082E3898384E08A83F801968536
:100960009B8397859C8390899D8391899E8396E341
:100970009F838887828D8987838D8A87848D8B87E3
:10098000858D8C874CE050E0B701C6010E94ED21B7
:1009900087E3898386E08A8391E09B8393E09C834D
:1009A0008D838FE08E838AE38F838BE388878FEF3D
:1009B000898749E050E0B701C6010E94ED21C601D8
:1009C0000E942722A6960FB6F894DEBF0FBECDBFB9
:1009D000DF91CF911F910F91FF90EF90DF90CF901B
:1009E000BF90AF909F908F907F90089590E080E0AF
:1009F0000C94A321CF93DF93C4E1D0E00E94F6844E
:100A0000882361F061E070E080E090E00E9479A9C5
:100A10002197A1F780E0DF91CF91089581E0FBCF8E
:100A2000FF920F931F93CF93DF931F921F92CDB727
:100A3000DEB7F82E22E030E0AE014F5F5F4F66E296
:100A400070E00E94C62109811A8110270127102712
:100A500022E030E0AE014F5F5F4F66E270E08F2D25
:100A60000E94C62189819A8198278927982708178B
:100A7000190749F4C8010F900F90DF91CF911F9192
:100A80000F91FF9008958C01E3CFFB0144815581C4
:100A9000FC01248135812417350778F0808191810C
:100AA000009759F0FB01608171816115710529F092
:100AB0000E9457D821E0892B09F020E0822F089569
:100AC000FC0124813581232B39F421E0FB01808155
:100AD000882349F020E007C0808191810E9437D8A7
:100AE00021E0892BB9F7822F08950F931F93CF939D
:100AF000DF938C01EB01FC01808191810097E1F093
:100B00006881798161157105A9F0428153812C8139
:100B10003D814217530770F00E9440D88C819D811F
:100B2000F801958384831D821C82DF91CF911F91F0
:100B30000F9108950E9483CA88819981F801918359
:100B400080838A819B81938382838C819D8195831D
:100B50008483198218821B821A82E5CF0F931F9318
:100B6000CF93DF93EC0188819981009759F02A8116
:100B70003B812617370730F081E0DF91CF911F913D
:100B80000F9108958B016F5F7F4F0E94D6D600971B
:100B900059F0998388831B830A832C813D81232B01
:100BA00059F7FC011082E8CF80E0E7CFEF92FF9287
:100BB0000F931F93CF93DF936115710541F480E08C
:100BC000DF91CF911F910F91FF90EF900895411504
:100BD0005105B1F07B01EC010C811D81040F151F43
:100BE000B8010E94AE85882351F3288139818C8118
:100BF0009D81B701820F931F0E9440D81D830C83F3
:100C000081E0DECFCF93DF931F921F92CDB7DEB787
:100C100069831A8241E050E0BE016F5F7F4F0E94FE
:100C2000D6850F900F90DF91CF910895CF93DF93EA
:100C3000EC0188819981009711F00E9483CA198282
:100C400018821D821C821B821A82DF91CF91089527
:100C5000EF92FF920F931F93CF93DF9300D01F92D9
:100C6000CDB7DEB77C01862F4AE08E010F5F1F4FA4
:100C7000B80190E00E949CCCF80101900020E9F7B7
:100C80003197AF01401B510BB801C7010E94D685B7
:100C9000811103C0C7010E941686C7010F900F90F3
:100CA0000F900F90DF91CF911F910F91FF90EF90D8
:100CB0000895CF93DF93EC016115710539F4CE01EE
:100CC0000E941686CE01DF91CF910895FB0101901D
:100CD0000020E9F73197AF01461B570B0E94D685DC
:100CE000882369F3EFCFCF93DF93EC01FB014481BD
:100CF0005581608171810E94D685811103C0CE012A
:100D00000E941686CE01DF91CF910895EF92FF9257
:100D10000F931F93CF93DF93EC017B018A01BA01FC
:100D20000E94AE8581110BC0CE010E941686CE01B5
:100D3000DF91CF911F910F91FF90EF9008951D8348
:100D40000C83B701888199810E9440D8F0CFFB01C4
:100D500001900020E9F73197AF01461B570B0C9427
:100D60008686CF93DF93EC016115710531F00E9407
:100D7000A786CE01DF91CF9108950E941686F9CF04
:100D8000CF93DF93EC01FB018617970749F0608151
:100D900071816115710541F0448155810E948686FB
:100DA000CE01DF91CF9108950E941686F9CFFC0104
:100DB00080819181009711F00C9483CA0895EF927D
:100DC000FF920F931F93CF93DF93EC018B01198256
:100DD00018821B821A821D821C82CB010E9430CC99
:100DE0007C01BC01CE010E94AE85811109C0CE01FB
:100DF000DF91CF911F910F91FF90EF900C94168689
:100E0000FD82EC82B80188819981DF91CF911F9199
:100E10000F91FF90EF900C9429CCFC01118210826D
:100E200013821282158214820C94C086FC011182F6
:100E300010821382128215821482FB01019000201D
:100E4000E9F73197AF01461B570B0C948686AF929A
:100E5000BF92CF92DF92EF92FF920F931F93CF93A7
:100E6000DF935C016B017A0189012417350720F4B7
:100E70008F2D7901042F182F6AE076E0C5010E94BA
:100E80001687D6011496CD91DC91EC16FD06C8F4B8
:100E90000C171D0708F4E801D601ED91FC9111979C
:100EA000EC0FFD1F108110826D917C916E0D7F1DE6
:100EB000C5010E94B186F60180819181C80FD91FBA
:100EC0001883C501DF91CF911F910F91FF90EF9093
:100ED000DF90CF90BF90AF9008950F931F93CF9363
:100EE000DF93EC010E94ABA9688779878A879B878B
:100EF000E881F9810284F385E02DCE01199597FFF1
:100F000015C00E94ABA9088519852A853B85601B01
:100F1000710B820B930B0C811D812E813F81601719
:100F200071078207930720F38FEF9FEFDF91CF9137
:100F30001F910F910895EF92FF920F931F93CF93FC
:100F4000DF93EC017B01042F6AE076E00E941687B4
:100F5000C7010E946D87002E000C110B97FD0BC07E
:100F60000817190741F0682FCE010E940286C701B9
:100F70000E946D87F3CFCE01DF91CF911F910F912A
:100F8000FF90EF900895CF92DF92EF92FF920F9330
:100F90001F93CF93DF936C017A018B01D0E0C0E007
:100FA000C6010E946D8797FD07C0F80181938F01EC
:100FB0002196EC16FD06A1F7CE01DF91CF911F918E
:100FC0000F91FF90EF90DF90CF900895FB0101907B
:100FD0000020E9F73197AF01461B570BDC01ED917B
:100FE000FC910280F381E02D19948F929F92AF9231
:100FF000BF92EF92FF920F931F93CF93DF93CDB7E2
:10100000DEB7A1970FB6F894DEBF0FBECDBF7C014F
:10101000FA01CB0119A2223008F42AE08E010F5DFB
:101020001F4F822E912CB12CA12CBF01A501940140
:101030000E945FD3F901CA016A300CF5605DD801E6
:101040006E938D01232B242B252B79F790E080E0E4
:10105000109721F0BD01C7010E94E687A1960FB647
:10106000F894DEBF0FBECDBFDF91CF911F910F91DE
:10107000FF90EF90BF90AF909F908F900895695C24
:10108000DECF68E076E00C94E687242F462F50E010
:1010900070E060E00C94F587EF92FF920F931F933E
:1010A000CF93DF93009751F4CFEFDFEFCE01DF91C5
:1010B000CF911F910F91FF90EF900895DC011C9646
:1010C000ED90FC90F70100811181D801ED91FC9128
:1010D0000688F789E02DC8011995882329F3D801DE
:1010E000ED91FC910084F185E02DC8011995D8019E
:1010F000ED91FC91892B61F30284F385E02DC80109
:101100001995EC01019681F2F801818D882339F05F
:101110004AE050E06C2F89E69BE00E944588D701A9
:1011200012968C91882311F2C532D10509F0BECFF9
:10113000D801ED91FC910084F185E02DC80119954D
:1011400002975CF0D801ED91FC910688F789E02DBB
:10115000C80119958111ECCFA7CFD1E0C0E0D8012B
:10116000ED91FC910284F385E02DC80119958F3F24
:10117000980709F499CF9C01215431092A3131058E
:1011800070F48D2F8295807F829FC00D1124D11124
:1011900004C00C2E000CDD0B89CFD0E0E0CF9C0109
:1011A000215631092A31310560F3C0978A30910503
:1011B00070F79D2F9295907F989FC00D1124E7CFD7
:1011C000DC01ED91FC910190F081E02D1994CF921A
:1011D000DF92EF92FF920F931F93CF93DF9321152E
:1011E000310581F4DC01ED91FC910190F081E02D5D
:1011F000642FDF91CF911F910F91FF90EF90DF90BF
:10120000CF9019942A30310501F52AE077FF1DC0EF
:101210006A017B01EC016DE20E94E0888C014427A9
:101220005527BA014C195D096E097F092AE0CE01E4
:101230000E94F587800F911FDF91CF911F910F9131
:10124000FF90EF90DF90CF900895DF91CF911F91A5
:101250000F91FF90EF90DF90CF900C94F5878F92D5
:101260009F92AF92BF92CF92DF92EF92FF920F9335
:101270001F93CF93DF937C018B014C0182E0880E9A
:10128000911C5701E5E0AE0EB11CD0E0C0E0F401C6
:1012900061914F014AE050E0C8010E9445886C010D
:1012A0006EE2C8010E94E0888C0D9D1DC80FD91FF9
:1012B0008A149B0461F74AE050E0F7016581C80198
:1012C0000E9445888C0F9D1FDF91CF911F910F9138
:1012D000FF90EF90DF90CF90BF90AF909F908F9056
:1012E00008956115710511F00C94E68790E080E097
:1012F00008950F931F93CF93DF93EC016BE076E09B
:1013000089E69BE00E9471894A855B856C857D85B5
:101310008A819B81AC81BD81481B590B6A0B7B0B79
:101320008E859F85A889B989481B590B6A0B7B0B51
:101330002AE089E69BE00E94F58789E69BE00E940F
:1013400041886A857B858C859D850A811B812C81DE
:101350003D81601B710B820B930B0E851F852889C5
:101360003989601B710B820B930BDF91CF911F9119
:101370000F910895DB0114964D915C9115976D9135
:101380007C91DC01ED91FC910280F381E02D1994B8
:10139000EF92FF920F931F93CF93DF938C017B010A
:1013A000D0E0C0E0F701EC0FFD1F6491662361F00F
:1013B000D801ED91FC910190F081E02DC8011995C3
:1013C000892B11F02196EECFCE01DF91CF911F91A5
:1013D0000F91FF90EF9008950F931F93CF93DF939A
:1013E000EC010E94C8898C01CE010E944188800FC7
:1013F000911FDF91CF911F910F9108958091580710
:1014000081110AC089E69BE00E94418863E27CE189
:1014100089E69BE00C94C8890895DC018FE094E094
:101420008D939D9384E0FB0101900D928A95E1F7E5
:1014300008953F924F925F926F927F928F929F9208
:10144000AF92BF92CF92DF92EF92FF920F931F93D2
:10145000CF93DF93CDB7DEB7EA970FB6F894DEBF30
:101460000FBECDBF7C012A013B0169010E94ABA9DF
:101470004B015C0187010D5B1F4FC8010E94C21622
:1014800018161906ACF00E94ABA9681979098A09E7
:101490009B09461657066806790608F468C10E943B
:1014A000BD7061E070E080E090E00E9479A9E5CF36
:1014B00042E250E0BE016F5F7F4FC8010E944D16AF
:1014C00089818230D1F0312C832DEA960FB6F894C1
:1014D000DEBF0FBECDBFDF91CF911F910F91FF9067
:1014E000EF90DF90CF90BF90AF909F908F907F90C4
:1014F0006F905F904F903F900895F801848995898F
:101500008334910501F76D817E818F8198850E94DA
:10151000DED34B015C01F60180829182A282B3820C
:1015200046E050E0B701685F7F4FCE014D960E94C4
:10153000E6D7892B41F6F70180819181A281B381A1
:1015400088169906AA06BB0608F4BDCF848195814A
:10155000A681B78188159905AA05BB0508F4B3CF04
:1015600089899A89AB89BC8986879787A08BB18B3B
:101570004EEC50E070E060E0C8010E944D16312C46
:10158000C701829698AB8FA7F701B696FAABE9AB85
:1015900008969CAB8BAB67019AE1C90ED11CBD9636
:1015A000FEABEDABC701429698AF8FABFD97FAAF9C
:1015B000E9AF4701FEE18F0E911CF801818D928DFC
:1015C000181619060CF080CFC8010E946C168333E0
:1015D000910509F4B2C014F58130910509F464C095
:1015E00044F4892B51F3C8010E946C16AC015527B5
:1015F00075C08330910509F462C00697A1F7C80150
:101600000E946C16B82E44E050E0B401C8010E945C
:101610004D16EB2DE450FF0BAF0160C08A339105EE
:1016200009F45FC084F585339105B1F1C697D9F609
:10163000C8010E946C165C01B601CE0189960E9419
:101640000D8A8BA59CA5ADA5BEA5892B8A2B8B2BBE
:10165000B1F0EDA9FEA94080518062807380B6018F
:10166000CE0183960E940D8A8DA19EA1AFA1B8A53F
:10167000A501481659066A067B0609F0B8CF44E072
:1016800050E0B60118C08B33910509F440C08F3F7C
:10169000910509F492CFA7CFC8010E946C16C8012A
:1016A0000E946C16382E89CFC8010E946C1644E047
:1016B00050E06FA978ADC8010E944D167ECFC801D9
:1016C0000E946C16B82E44E050E069AD7AADC801B6
:1016D0000E944D168B2D8450990BAC0170E060E098
:1016E000EACFC8010E946C1644E050E069A97AA9CB
:1016F000C8010E944D16F70166A177A180A591A5AA
:101700000E94DED366A377A380A791A756CFC80116
:101710000E946C1644E050E06BA97CA9C8010E94AD
:101720004D16F70162A573A584A595A50E94DED389
:1017300062A773A784A795A740CFC8010E946C1623
:1017400044E050E06FA578A9C8010E944D16F7014A
:1017500062A173A184A195A10E94DED362A373A3A9
:1017600084A395A366A777A780AB91AB26CF33243C
:101770003A94AACE2F923F924F925F926F927F92AD
:101780008F929F92AF92BF92CF92DF92EF92FF9291
:101790000F931F93CF93DF9300D000D0CDB7DEB768
:1017A0008C010E9458CB2FEC37E040E050E00E94C3
:1017B00081D3DC01CB010196A11DB11DF801848309
:1017C0009583A683B78380839183A283B3835801D3
:1017D000F3E4AF0EB11CC5010E94171664E470E07B
:1017E000C5010E949117882309F445C10E94ABA945
:1017F0002B013C01480182E4880E911C48EEC42E66
:1018000043E0D42EE12CF12C52E0252E1E821D82C5
:10181000D4018C918330B1F1811166C0F8018481CB
:101820009581A681B7810196A11DB11D8483958301
:10183000A683B7830E94ABA9641975098609970925
:10184000A70196010E945FD3A90161E0C8010E942F
:10185000E88381E0D4018C938D819E810197C1F250
:101860000E94ABA96419750986099709D801D69613
:101870002D913D914D915C91D997261737074807D7
:10188000590720F6C5010E941716F8018481958139
:10189000A681B7810196A11DB11D84839583A6837E
:1018A000B7830E94ABA9F801FE966083718382839F
:1018B00093838D819E8126960FB6F894DEBF0FBE6E
:1018C000CDBFDF91CF911F910F91FF90EF90DF90EF
:1018D000CF90BF90AF909F908F907F906F905F90D0
:1018E0004F903F902F9008958430F1F4F801848157
:1018F0009581A681B7810196A11DB11D8483958331
:10190000A683B7830E94ABA9641975098609970954
:10191000A70196010E945FD3A90163E0C8010E945C
:10192000E883D4012C9298CF813051F5F80142AD73
:1019300053AD64AD75AD9E012F5F3F4FC8010E944E
:10194000198A382EF2E08F1390C089819A81AB8179
:10195000BC81F80184839583A683B7830E94ABA9D9
:101960006419750986099709A70196010E945FD33A
:10197000A90163E0C8010E94E883D4013C926CCFC6
:10198000823009F069CFF80142AD53AD64AD75AD59
:101990009E012F5F3F4FC8010E94198A382EF5E043
:1019A0008F135DC0E3E0D401EC93F80182A193A111
:1019B000A4A1B5A1892B8A2B8B2B41F484E893E059
:1019C000A0E0B0E082A393A3A4A3B5A3F80186A1ED
:1019D00097A1A0A5B1A5892B8A2B8B2B61F482A19D
:1019E00093A1A4A1B5A1B695A7959795879586A330
:1019F00097A3A0A7B1A7F80182A593A5A4A5B5A513
:101A0000892B8A2B8B2BA9F482A193A1A4A1B5A128
:101A1000AC01BD0123E076956795579547952A95CA
:101A2000D1F7841B950BA60BB70B82A793A7A4A78E
:101A3000B5A7F80186A197A1A0A5B1A586A797A7EC
:101A4000A0ABB1AB82A593A5A4A5B5A582AB93AB82
:101A5000A4ABB5AB81E090E09E838D83FDCE96E094
:101A6000891303C0D4011C92F7CEBFEF3B12F4CE12
:101A7000F4011082F1CE1E821D821BCF1F920F92A5
:101A80000FB60F9211240BB60F922F933F934F93E3
:101A90005F936F937F938F939F93AF93BF93EF93D6
:101AA000FF9380ED98E00E942680FF91EF91BF9117
:101AB000AF919F918F917F916F915F914F913F91E6
:101AC0002F910F900BBE0F900FBE0F901F90189587
:101AD0001F920F920FB60F9211240BB60F922F93F5
:101AE0003F934F935F936F937F938F939F93AF93A6
:101AF000BF93EF93FF9380ED98E00E94A87FFF9142
:101B0000EF91BF91AF919F918F917F916F915F9175
:101B10004F913F912F910F900BBE0F900FBE0F90E2
:101B20001F9018951F920F920FB60F9211240BB6AB
:101B30000F922F933F934F935F936F937F938F9366
:101B40009F93AF93BF93EF93FF938DE699E00E942D
:101B50002680FF91EF91BF91AF919F918F917F91DF
:101B60006F915F914F913F912F910F900BBE0F900E
:101B70000FBE0F901F9018951F920F920FB60F92E5
:101B800011240BB60F922F933F934F935F936F9354
:101B90007F938F939F93AF93BF93EF93FF938DE6C4
:101BA00099E00E94A87FFF91EF91BF91AF919F9123
:101BB0008F917F916F915F914F913F912F910F90F6
:101BC0000BBE0F900FBE0F901F9018951F920F9293
:101BD0000FB60F9211240BB60F922F933F934F9392
:101BE0005F936F937F938F939F93AF93BF93EF9385
:101BF000FF938AE09AE00E942680FF91EF91BF91C7
:101C0000AF919F918F917F916F915F914F913F9194
